:100000000C9478030C9497030C9497030C94970327
:100010000C9497030C9497030C9497030C949703F8
:100020000C9497030C9497030C9488560C94BF512E
:100030000C94D1640C9497030C9497030C9497033D
:100040000C9497030C9497030C9497030C949703C8
:100050000C944B180C9497030C9497030C949703EF
:100060000C9497030C9497030C9497030C949703A8
:100070000C9497030C9497030C9497030C94970398
:100080000C9497030C9497030C9497030C94970388
:100090000C9497030C9497036E616E00696E660072
:1000A000456E676C697368005452414E5356455211
:1000B00054455200506F77657220436F6E74726FB3
:1000C0006C00506F776572204D6F64756C650050E1
:1000D0007265737320746865004F464620627574BC
:1000E000746F6E005072657373204F4646006167EF
:1000F00061696E00456E74657220342044696769D9
:10010000742050494E00444320494E004143204949
:100110002F4F00504D20252D32640054253032647D
:1001200058004C4E20256400524C59202564005440
:10013000455354004D41494E0053455455500052CB
:1001400065626F6F74207468652055493F00286FA1
:100150006E6C79207468652055492900504D7320D4
:1001600077697468204572726F72733A004348452C
:100170004D495354525900543133580053657475E6
:100180007000436C6F636B005365742054696D6538
:10019000005465737473004175746F00544C6F772D
:1001A00000544C6F773A00544869676800506F7785
:1001B00065720044432050777200414320507772AB
:1001C00000205553422052455345542020202041C1
:1001D00055544F00414C41524D0052455345540037
:1001E00059454152004D4F00444159004852004D7D
:1001F000494E00555000444F574E00555020313065
:1002000000444F574E203130005550203100444FAC
:10021000574E2031005550202E3100444F574E206C
:100220002E310053415645005642413A0056424253
:100230003A004942413A004942423A005635303A82
:1002400000563530413A00563530423A0056313981
:10025000303A0056494E3A0049494E3A0050494E0C
:100260003A0049523A2000504D00414300487A007C
:10027000564100503A0050663A0043616E63656C27
:1002800000537769746368204F4646004F4E004F15
:1002900046460054696C6C00444320494E0041437B
:1002A00020492F4F004C4F434B004F4B00424154CD
:1002B000004241545445525900534F4C00534F4C47
:1002C00041520048594400485944524F00574E4447
:1002D0000057494E4400475249440053594E434841
:1002E0000047454E45524154004E4F4E450050493F
:1002F0004E005550444154450053455420555050EC
:10030000455200534554204C4F5745520043544CDE
:10031000204C494D4954004C494D495400535552C5
:10032000474500504F55540046414E005042410051
:100330005042420056353000426174746572792033
:1003400042616E6B733A00416D702D487273004DBF
:10035000696E732F42616E6B004C454144004E69DB
:100360004344004C495448004E694D4800434F4EA9
:10037000535452554354494F4E005745540041473A
:100380004D0047454C0041626F7274005265626FC8
:100390006F74004572726F727300414343004348AB
:1003A0004700566572004C494E45530052454C413A
:1003B0005953004B574800204F50454E00434C4F77
:1003C00053450053434845442000454E41424C4567
:1003D000440044495341424C4500494E20004F558A
:1003E00054004F4E20004F46460043484152474973
:1003F0004E47200044495343484152474500204658
:10040000554C4C00454D5054590020564241002057
:10041000564242004E4F4E4520202000534F4C4143
:1004200052202000485944524F20200057494E4442
:1004300020202000475249442020200053594E4399
:1004400048202000313256003234560033365600F0
:10045000464C4F4154494E47004348415247494E4C
:1004600047004F50454E202000434C4F5345440019
:10047000564F5554204241440056313930204241B4
:1004800044004E4F204552524F520006A0FF090132
:10049000A1010902A10006A1FF0903090415802595
:1004A0007F350045FF750895088102090509061585
:1004B00080257F350045FF750895089102C0C01260
:1004C000011001FFFFFF082509222200010102039C
:1004D0000109022900010100C0320904000002FFE5
:1004E000FFFF0009211101000122340007058203EA
:1004F000400001070501034000010403090424032F
:100500004800650061007200740020005400720011
:1005100061006E0073007600650072007400650073
:100520007200000026034800540032003000300002
:10053000300020005400720061006E0073007600ED
:100540006500720074006500720000001C03540016
:1005500052003000300030003100300030003300F5
:10056000310032003300340000008E008E0287001C
:100570008700840287028702840289008B008D0035
:1005800089028B028D0288008A008C0088028A0210
:100590008C020B000F000B020F020A000E000A0271
:1005A0000E0209000D0009020D0208000C000802ED
:1005B0000C0207008100830007028102830206000B
:1005C0008000820006028002820285028502850286
:1005D000850202000500020205020100040001027A
:1005E0000402CF08CF08CF08CF0ACF0ACF0A0000F5
:1005F00003000002030200407A10F35A00A0724E7A
:1006000018090010A5D4E80000E87648170000E4B7
:100610000B54020000CA9A3B000000E1F5050000FF
:1006200080969800000040420F000000A086010064
:100630000000102700000000E80300000000640034
:10064000000000000A00000000000100000000009F
:100650002C76D888DC674F0823DFC1DFAE59E1B1C3
:10066000B796E5E3E453C63AE651997696E8E6C2D2
:100670008426EB898C9B62ED407C6FFCEFBC9C9FD9
:1006800040F2BAA56FA5F490055A2AF75C936B6CFB
:10069000F9676DC11BFCE0E40D47FEF520E6B500EF
:1006A000D0ED902E0300943577050080841E08005D
:1006B00000204E0A000000C80C333333330F986E0D
:1006C00012831141EF8D2114893BE65516CFFEE6CA
:1006D000DB18D1844B381BF77C1D901DA4BBE42490
:1006E000203284725E228100C9F124ECA1E53D270D
:1006F00011241FBECFEFD0E2DEBFCDBF1CE0A0E0D3
:10070000B1E0E8E6FBE801E00BBF02C007900D9204
:10071000A838B107D9F71EE1A8E8BCE001C01D92D6
:10072000AA32B107E1F70E9450640C94B2C50C9450
:1007300000008091880C882311F4409A0895419A12
:1007400008958091880C882311F440980895419869
:1007500008958093880C08950E94990300C00E9418
:10076000A10308951F93662311F0429A01C0429895
:1007700043983C9A3D9A3E9A3F9A479846984598A6
:10078000449887FD479A182F86FD469A15FD459A8D
:1007900014FD449A0E94AC034798469845984498A3
:1007A00013FD479A12FD469A11FD459A10FD449A91
:1007B0000E94AC03449A459A469A479A1F9108951D
:1007C0001F93882311F0429A01C04298439A3C98A3
:1007D0003D983E983F980E94990300C0349B02C008
:1007E00010E101C010E03599106236991064379914
:1007F00010680E94A10300C00E94990300C03499B0
:1008000011603599126036991460379918600E940A
:10081000A103812F1F910895CF93DF93C8EED3E0FA
:1008200004C0219739F00E94486480E00E94E003F0
:1008300087FDF7CF84E090E00197F1F780E00E9418
:10084000E00390E0DF91CF9108950E940C0481E0D5
:100850000E94E00308951F93182F0E940C04812F1B
:1008600061E00E94B2031F9108951F93182F0E9408
:100870000C04812F60E00E94B2031F910895DF9263
:10088000EF92FF920F931F93CF93DF93D82E109286
:10089000880C3A9A3B9A389A399A3C9A3D9A3E9AF1
:1008A0003F9A80E09DE70197F1F7C0E0D0E0E12CAE
:1008B00087E2F82E00E810E0C093880C459A449A2D
:1008C0000E94AC03C7010197F1F70E94AC03C80175
:1008D0000197F1F70E94AC03C8010197F1F7449822
:1008E0000E94AC03C8010197F1F788E20E94350429
:1008F00088E00E94350481E00E94350486E00E9471
:1009000035048D2D0E9435042196C230D105A1F603
:10091000DF91CF911F910F91FF90EF90DF9008959D
:100920001092880C662319F091E09093880C8770E0
:10093000880F880F880F805C0E943504089564300A
:1009400008F063E070E0FB01E050FF4F908190936E
:10095000880C80586C5F7E4FFB019081890F0E944C
:10096000350408951F93182F0E940C041A3049F47F
:10097000803410F080E001C080E480580E9435048B
:1009800004C0812F61E00E94B2031F9108950F936C
:100990001F93DF93CF930F92CDB7DEB78C0106C0C4
:1009A0000F5F1F4F69830E94B2046981662329F09B
:1009B000F80180816150882399F70F90CF91DF91E2
:1009C0001F910F910895CF93DF93EC0102C00E9415
:1009D000B20489918823D9F7DF91CF9108959EBD04
:1009E0000DB407FEFDCF3EB58EBD0DB407FEFDCFA5
:1009F0002EB5932F80E030E0282B392BC9010895C4
:100A0000E4E6F0E080818B7F808384B1866084B9E6
:100A100089E58CBD8DB58EB508958EBD0DB407FEEC
:100A2000FDCF8EB50895FC01862F972F2FEF07C0BD
:100A30002EBD0DB407FEFDCF3EB5319301971816BC
:100A40001906B4F30895262F372F0AC0FC01408100
:100A50004EBD0DB407FEFDCF01964EB5215030407E
:100A6000121613069CF308950E94EF0408950F9345
:100A70001F93CF93DF93EC01062F172F08C080E060
:100A800090E00E94EF048993999301501040101652
:100A90001106ACF3DF91CF911F910F9108950F9341
:100AA0001F93CF93DF93EC01062F172F06C0899178
:100AB00099910E94EF040150104010161106BCF3EA
:100AC000DF91CF911F910F910895E0912E1EF0912B
:100AD0002F1EE65DF14E8081089580912E1E90912B
:100AE0002F1E019797FF02C083E090E0865D914E34
:100AF000FC01808108952AE23EE1E0912E1EF091F2
:100B00002F1EE20FF31F9081290F311DF901808301
:100B1000089509966AE070E00E9417C37093970CDD
:100B20006093960C089580E060E041E00E941C64B0
:100B300008958AE090E09093970C8093960C0E9421
:100B400057128091311B81508093311B8CE00E94A1
:100B50003504E0912E1EF0912F1EE65DF14EE081EE
:100B6000F0E0EE0FFF1FE85FFE4F0190F081E02DF7
:100B70000190F081E02D09958091311B8F5F80936A
:100B8000311B089580912E1E90912F1EFC01E65D71
:100B9000F14E22E02083019797FF02C083E090E0AE
:100BA00090932F1E80932E1EFC01E65DF14E8081F6
:100BB000882311F482E080830E9499050895E091D2
:100BC0002E1EF0912F1EE65DF14E80830E94990546
:100BD000089520912E1E30912F1E2F5F3F4F2430FD
:100BE000310514F020E030E030932F1E20932E1EAC
:100BF000265D314EF90180830E94990508958DE0AC
:100C00000E94E905089588E10E94E905089583E0BE
:100C10000E94E905089581E20E94E90508958CE0AB
:100C20000E94E905089582E00E94E9050895CF92A7
:100C3000DF92EF92FF920F931F93DF93CF930F9268
:100C4000CDB7DEB7982F6B0180E0692F49830E94F2
:100C50009F0400E010E04981E42EFF2407C00E94B9
:100C60002504F60181936F010F5F1F4F0E151F05BD
:100C7000B4F30F90CF91DF911F910F91FF90EF9000
:100C8000DF90CF900895CF93DF93682F80E00E948C
:100C90009F04CCEDDAE189910E94B2048AE1C03F61
:100CA000D807C9F7DF91CF9108950E94E304089512
:100CB0000F931F93DF93CF93CDB7DEB766970FB631
:100CC000F894DEBF0FBECDBF2DB73EB728503040E1
:100CD0000FB6F8943EBF0FBE2DBFEDB7FEB73196ED
:100CE0008E010F5F1F4FADB7BEB712961C930E93C8
:100CF000119725E130E033832283758364839783E2
:100D000086834E8B0E94B6C42DB73EB7285F3F4FF7
:100D10000FB6F8943EBF0FBE2DBFC8014E89642F99
:100D20000E94C70466960FB6F894DEBF0FBECDBF13
:100D3000CF91DF911F910F9108950F931F93DF9330
:100D4000CF93CDB7DEB766970FB6F894DEBF0FBE70
:100D5000CDBFADB7BEB71A970FB6F894BEBF0FBEE2
:100D6000ADBFEDB7FEB731968E010F5F1F4F1296E4
:100D70001C930E931197A5E1B0E0B383A283558332
:100D8000448366837783808791872E8B0E94B6C4C5
:100D9000EDB7FEB73A960FB6F894FEBF0FBEEDBFA3
:100DA000C8012E89622F0E94C70466960FB6F89478
:100DB000DEBF0FBECDBFCF91DF911F910F91089580
:100DC000EF92FF920F931F937A018B010E94B76BF2
:100DD0008091A30D9091A40DA091A50DB091A60DA9
:100DE00080938D0C90938E0CA0938F0CB093900CED
:100DF000C801B701675F7F4F8F4F9F4F2AE030E0F8
:100E000040E050E00E943EC32093910C3093920C3E
:100E10004093930C5093940C1F910F91FF90EF907F
:100E200008958091950C882329F09091661B93304A
:100E300009F084E040E050E0BA010E94E006089525
:100E4000823060F4E0912E1EF0912F1EE65DF14E8F
:100E5000808169E070E00E94ED290895843071F08E
:100E6000833071F48091910C9091920CA091930C2D
:100E7000B091940C0097A105B10511F40E941107DF
:100E80000895CF92DF92EF92FF920F931F9380917C
:100E9000631C882361F08091311B81508093311B4A
:100EA0000E9417398091311B8F5F8093311B0E9404
:100EB0006609882309F437C18091311B81508093E2
:100EC000311B80E190E00E947109882399F0E09144
:100ED0002E1EF0912F1EE65DF14EE081F0E0EE0F48
:100EE000FF1FE85FFE4F0190F081E02D0684F7853B
:100EF000E02D18C088E090E00E9471098823A9F0D5
:100F0000E0912E1EF0912F1EE65DF14EE081F0E0A3
:100F1000EE0FFF1FE85FFE4F0190F081E02D00888B
:100F2000F189E02D309709F0099582E090E00E9468
:100F30007109882399F0E0912E1EF0912F1EE65D35
:100F4000F14EE081F0E0EE0FFF1FE85FFE4F0190F1
:100F5000F081E02D0488F589E02D18C084E090E050
:100F60000E9471098823A9F0E0912E1EF0912F1E96
:100F7000E65DF14EE081F0E0EE0FFF1FE85FFE4F0F
:100F80000190F081E02D0288F389E02D309709F07F
:100F9000099580E091E00E947109882399F0E09121
:100FA0002E1EF0912F1EE65DF14EE081F0E0EE0F77
:100FB000FF1FE85FFE4F0190F081E02D0680F78172
:100FC000E02D4AC080E890E00E947109882399F0E2
:100FD000E0912E1EF0912F1EE65DF14EE081F0E0D3
:100FE000EE0FFF1FE85FFE4F0190F081E02D0084BF
:100FF000F185E02D31C080E490E00E9471098823E2
:1010000099F0E0912E1EF0912F1EE65DF14EE081E9
:10101000F0E0EE0FFF1FE85FFE4F0190F081E02D42
:101020000284F385E02D18C080E290E00E947109EF
:101030008823A9F0E0912E1EF0912F1EE65DF14E5F
:10104000E081F0E0EE0FFF1FE85FFE4F0190F081BE
:10105000E02D0484F585E02D309709F0099580E0B6
:1010600092E00E9471098823A9F0E0912E1EF09170
:101070002F1EE65DF14EE081F0E0EE0FFF1FE85F0E
:10108000FE4F0190F081E02D0480F581E02D309736
:1010900009F009958091661B833011F084E001C04E
:1010A0008CE048E853E160E070E00E94E00681E0F7
:1010B00090E00E947109882381F1E0912E1EF09149
:1010C0002F1EE65DF14EE081F0E0EE0FFF1FE85FBE
:1010D000FE4F0190F081E02D0688F789E02D3097D2
:1010E00011F009951AC08091661B8823B1F0809198
:1010F000950C8C3010F48C5F01C084E08093950CCB
:101100008091950C68E070E00E94ED298091950C2B
:1011100040E050E0BA010E94E0068091311B8F5FF1
:101120008093311B28C02091910C3091920C4091FA
:10113000930C5091940C2115310541055105D9F0BE
:101140008091A30D9091A40DA091A50DB091A60D35
:10115000E0908D0CF0908E0C00918F0C1091900C03
:101160008E199F09A00BB10B82179307A407B5072F
:1011700010F00E9411072091890C30918A0C409147
:101180008B0C50918C0C8091A30D9091A40DA0918B
:10119000A50DB091A60D281739074A075B07D1F1B5
:1011A0006C017D01C21AD30AE40AF50A4091960C3B
:1011B0005091970C60E070E0C416D506E606F7067D
:1011C00048F18093890C90938A0CA0938B0CB09378
:1011D0008C0CE0912E1EF0912F1EE65DF14EE08109
:1011E000F0E0EE0FFF1FE85FFE4F0190F081E02D71
:1011F00082819381009771F08091311B815080939F
:10120000311B0280F381E02D09958091311B8F5FA6
:101210008093311B1F910F91FF90EF90DF90CF9043
:10122000089588E090E064E04CE024E00E94FA2910
:101230008093950C80912E1C80FD07C080912E1EFE
:1012400090912F1E84309105B0F080E04AEF50E07D
:1012500060E070E00E94E00610922A1E10922B1EA1
:1012600010922C1E10922D1E10922F1E10922E1EC8
:101270000E940B2102C00E9411071092311B80E0D6
:101280000E94E905089520919C0C30919D0C282B1B
:10129000392B30939D0C20939C0C089580E0209175
:1012A000980C3091990C33702115310509F081E0CB
:1012B000089540E02091980C3091990C282339230F
:1012C0002115310509F041E0842F089580E0209137
:1012D0009A0C30919B0C33702115310509F081E097
:1012E000089540E020919A0C30919B0C28233923DB
:1012F0002115310509F041E0842F08950E94976778
:101300006091980C7091990C9093990C8093980C23
:101310002FB7F89440919C0C50919D0C10929D0C0D
:1013200010929C0C27FF01C078942091980C30916A
:10133000990C8627972782239323842B952B9093B0
:101340009B0C80939A0C242B352B3093990C209373
:10135000980C089580E092E09093990C8093980CFB
:101360000E947E0908958091F11A882321F481E07A
:101370008093F11A08951092F11A0895AF92BF92D6
:10138000CF92DF92EF92FF920F931F93DF93CF9351
:10139000CDB7DEB729970FB6F894DEBF0FBECDBF2D
:1013A0008091661B882309F481C180910D1C8F3FB9
:1013B00009F485C180910F1C8F3708F080C190918E
:1013C000F11A8091621B992351F50E944069609344
:1013D000F61A7093F71A8093F81A9093F91A80917D
:1013E000621B90E00E944C686093FA1A7093FB1A9B
:1013F0008093FC1A9093FD1A8091621B90E00E94EA
:10140000C6686093FE1A7093FF1A8093001B909336
:10141000011B8091621B90E00E940A682AC090E044
:101420000E947D696093F61A7093F71A8093F81AF8
:101430009093F91A8091621B90E00E9489686093F2
:10144000FA1A7093FB1A8093FC1A9093FD1A8091FC
:10145000621B90E00E9403696093FE1A7093FF1A6A
:101460008093001B9093011B8091621B90E00E946F
:10147000066860930A1B70930B1B80930C1B909360
:101480000D1B8091621B90E00E940E6860930E1B02
:1014900070930F1B8093101B9093111B6091F61A91
:1014A0007091F71A8091F81A9091F91A2091FA1A0E
:1014B0003091FB1A4091FC1A5091FD1A0E94D9C13B
:1014C000D62EC72EB82EA92EA6019501652F742FF2
:1014D000832F922F20E030E040EA50E40E94D5C1F3
:1014E00018165CF00F2EF0E0EF2EF0E0FF2EF0E08B
:1014F0000F2FF0E01F2FF02D33C06091FE1A709176
:10150000FF1A8091001B9091011BD601F5012B2F32
:101510003A2F4F2F5E2F0E948AC0E62EF72E082FFB
:10152000192F20E030E0A9010E9486C0882324F40E
:1015300017FB109517F91095C801B70120E030E0AE
:1015400040E85FE30E94D5C1181654F40F2EF0E076
:10155000EF2EF0E0FF2EF0E80F2FFFE31F2FF02D0E
:1015600083E060E00E949F04E091F11AF0E0EE0F4A
:10157000FF1FEF50F54E818192810E94E3048DE0C0
:1015800060E00E949F0460910E1B70910F1B809180
:10159000101B9091111B4AE551E026E00E949D0628
:1015A00080E061E00E949F046091F61A7091F71A42
:1015B0008091F81A9091F91A4AE551E026E00E94CC
:1015C0009D068BE061E00E949F048091621B90E089
:1015D000019660E671E042E00E9458068DE061E00D
:1015E0000E949F046091FA1A7091FB1A8091FC1A74
:1015F0009091FD1A4AE551E026E00E949D0683E0A5
:1016000062E00E949F046091FE1A7091FF1A80911F
:10161000001B9091011B45E651E027E00E949D06CA
:101620008BE062E00E949F04A6019501652F7C2D4E
:10163000832F9A2D45E651E027E00E949D0683E026
:1016400063E00E949F04C801B7014BE651E027E028
:101650000E949D068BE063E00E949F046091F61A51
:101660007091F71A8091F81A9091F91A20E030E001
:10167000A9010E9486C0882359F480E090E0DC0133
:1016800080930A1B90930B1BA0930C1BB0930D1B14
:1016900060910A1B70910B1B80910C1B90910D1B8C
:1016A0004BE651E028E00E949D0668C0CE010196FD
:1016B00066E372E00E9469C406E312E008C0CE014E
:1016C00001966EE372E00E9469C40EE312E083E0CB
:1016D00062E00E949F047E010894E11CF11CC70196
:1016E0000E9455068BE062E00E949F04C7010E94A1
:1016F000550683E063E00E949F04C7010E945506DF
:101700008BE063E00E949F04C7010E945506B80168
:101710006F5F7F4FC7010E9469C483E060E00E9451
:101720009F04E091F11AF0E0EE0FFF1FEF50F54E2D
:10173000818192810E94E3048DE060E00E949F0419
:10174000C7010E94550680E061E00E949F04C70126
:101750000E9455068BE061E00E949F048091621B0D
:1017600090E0019660E671E042E00E9458068DE04C
:1017700061E00E949F04C7010E94550629960FB69A
:10178000F894DEBF0FBECDBFCF91DF911F910F91B7
:10179000FF90EF90DF90CF90BF90AF900895EF92C1
:1017A000FF920F931F93CF93DF9381E08093F11A01
:1017B0008FE70E949B129093F31A8093F21A80E8AD
:1017C0000E949B129093F51A8093F41A84EF91E093
:1017D0000E948905CCEDDAE1CE0160E270E044E1DF
:1017E00050E00E9459C480E40E949B12BC01FC019D
:1017F00001900020E9F73197E81BF90BCE01AF010A
:101800000E9450C48AE30E949B12BC01FC0101901B
:101810000020E9F73197E81BF90B9E01295F3F4F44
:10182000C901AF010E9450C486E58093EF1A80E0A1
:1018300090E00E944306CE0160E270E044E150E097
:101840000E9459C48FE30E949B12BC01FC010190CD
:101850000020E9F73197E81BF90B9E01285F3F4F05
:10186000C901AF010E9450C481E48093EF1A81E066
:1018700090E00E944306CE0160E270E044E150E057
:101880000E9459C483E40E949B12BC01FC01019098
:101890000020E9F73197E81BF90BCE01AF010E9458
:1018A00050C487E58093E51A82E40E949B12BC0134
:1018B000FC0101900020E9F73197E81BF90B8E013C
:1018C0000E5E1F4FC801AF010E9450C482E090E03D
:1018D0000E944306CE0160E270E044E150E00E94C5
:1018E00059C484E40E949B12BC01FC0101900020B9
:1018F000E9F73197E81BF90BCE01AF010E9450C404
:1019000081E40E949B12BC01FC0101900020E9F7D8
:101910003197E81BF90BC801AF010E9450C483E066
:1019200090E00E9443060E94BE09DF91CF911F9173
:101930000F91FF90EF900895EF92FF920F931F93F6
:10194000DF93CF93CDB7DEB729970FB6F894DEBFFC
:101950000FBECDBF8091621B90E00E94B86A609379
:10196000F11A7093F21A8093F31A9093F41A8091FB
:10197000621B90E00E94B26A6093F51A7093F61AA7
:101980008093F71A9093F81A8091621B90E00E945E
:10199000046B6093F91A7093FA1A8093FB1A909370
:1019A000FC1A8091621B90E00E94FE6A6093FD1A0F
:1019B0007093FE1A8093FF1A9093001B8091621B14
:1019C00090E00E94AC6A6093011B7093021B8093AD
:1019D000031B9093041B8091621B90E00E94C66AD7
:1019E0006093051B7093061B8093071B9093081B45
:1019F0008091621B90E00E940E686093091B7093B7
:101A00000A1B80930B1B90930C1B8091661B8823F1
:101A100009F488C080910D1C8F3F09F48EC084E0CA
:101A200060E00E949F046091F11A7091F21A809117
:101A3000F31A9091F41A49E851E027E00E949D06BC
:101A40008CE060E00E949F046091F91A7091FA1A8C
:101A50008091FB1A9091FC1A49E851E027E00E941E
:101A60009D0684E061E00E949F046091F51A7091E8
:101A7000F61A8091F71A9091F81A49E851E027E098
:101A80000E949D068CE061E00E949F046091FD1A17
:101A90007091FE1A8091FF1A9091001B49E851E065
:101AA00027E00E949D0684E062E00E949F0460910E
:101AB000011B7091021B8091031B9091041B49E84C
:101AC00051E027E00E949D068CE062E00E949F04A6
:101AD0006091051B7091061B8091071B9091081B5C
:101AE00049E851E027E00E949D0680910F1C8F3746
:101AF00090F485E063E00E949F046091091B70915F
:101B00000A1B80910B1B90910C1B4FE851E026E0C3
:101B10000E949D0656C085E063E00E949F048FE30B
:101B200092E04DC0CE01019666E372E00E9469C466
:101B300096E3E92E92E0F92E0AC0CE0101966EE3FB
:101B400072E00E9469C48EE3E82E82E0F82E84E001
:101B500060E00E949F048E010F5F1F4FC8010E942A
:101B600055068CE060E00E949F04C8010E94550663
:101B700084E061E00E949F04C8010E9455068CE049
:101B800061E00E949F04C8010E94550684E062E063
:101B90000E949F04C8010E9455068CE062E00E94EA
:101BA0009F04C8010E945506B7016F5F7F4FC801AF
:101BB0000E9469C485E063E00E949F04C8010E94FE
:101BC000550682E163E00E949F048091621B90E0D1
:101BD000019665E971E042E00E94580629960FB629
:101BE000F894DEBF0FBECDBFCF91DF911F910F9153
:101BF000FF90EF900895EF92FF920F931F93CF9372
:101C0000DF9384EF91E00E948905CCEDDAE1CE010B
:101C100060E270E044E150E00E9459C483E30E9416
:101C20009B12BC01FC0101900020E9F73197E81BF1
:101C3000F90BCE01AF010E9450C416E51093E71ACC
:101C400001E40093EF1A80E090E00E944306CE0189
:101C500060E270E044E150E00E9459C484E30E94D5
:101C60009B12BC01FC0101900020E9F73197E81BB1
:101C7000F90BCE01AF010E9450C41093E71A0093F4
:101C8000EF1A81E090E00E944306CE0160E270E02E
:101C900044E150E00E9459C487E30E949B12BC01BA
:101CA000FC0101900020E9F73197E81BF90BCE0108
:101CB000AF010E9450C41093E71A0093EF1A82E01C
:101CC00090E00E944306CE0160E270E044E150E003
:101CD0000E9459C48AE30E949B12BC01FC0101903E
:101CE0000020E9F73197E81BF90BCE01AF010E9404
:101CF00050C41093E71A8FE30E949B12BC01FC01B1
:101D000001900020E9F73197E81BF90B2F96CE01DF
:101D1000AF010E9450C483E090E00E9443060E94FD
:101D20009C0CDF91CF911F910F91FF90EF90089540
:101D300081E00E94E90508951F938091A30D909181
:101D4000A40DA091A50DB091A60D2091F61A309189
:101D5000F71A4091F81A5091F91A821B930BA40BB1
:101D6000B50B893C9105A105B105F8F089E090E03B
:101D700060E048E220E00E94FA29182F80912E1C92
:101D800080FD06C0112321F0113011F01A3111F439
:101D90008EE008C00E946D05181719F40E94C20554
:101DA00008C0812F0E94E90504C081EF9AE10E94DA
:101DB000C3491F9108950F931F93CF93DF93CCEDE9
:101DC000DAE1CE0160E270E044E150E00E9459C4E3
:101DD00081E00E949B12BC01FC0101900020E9F708
:101DE0003197E81BF90B04E110E098012E1B3F0B23
:101DF000369527952C0F3D1FC901AF010E9450C495
:101E000080E090E00E944306CE0160E270E044E191
:101E100050E00E9459C481E090E00E94430683E0B4
:101E200090E00E94430680E00E949B12BC01FC01EE
:101E300001900020E9F73197E81BF90B98012E1B60
:101E40003F0B369527952C0F3D1FC901AF010E940E
:101E500050C482E090E00E94430686E70E949B12F5
:101E60002DB73EB7245130400FB6F8943EBF0FBE99
:101E70002DBFEDB7FEB73196ADB7BEB71296DC9366
:101E8000CE93119725E130E03383228322EB31E0BA
:101E9000358324839783868382E090E091878087CF
:101EA00089E290E09387828780E190E0958784873C
:101EB0001787068780E290E0918B808B82E190E02B
:101EC000938B828B0E94B6C42DB73EB72C5E3F4FDA
:101ED0000FB6F8943EBF0FBE2DBF80E063E00E94B6
:101EE0009F04CE010E94550681EF9AE10E94054AA7
:101EF0008091A30D9091A40DA091A50DB091A60D78
:101F00008093F61A9093F71AA093F81AB093F91ADF
:101F1000DF91CF911F910F91089581E00E94E90513
:101F200008958091621B8093651B8091691B80934B
:101F3000681B0E94070608950F931F93DF93CF93AA
:101F4000CDB7DEB728970FB6F894DEBF0FBECDBF72
:101F50008091A30D9091A40DA091A50DB091A60D17
:101F60002091F81A3091F91A4091FA1A5091FB1AFF
:101F7000821B930BA40BB50B853F21E0920720E059
:101F8000A20720E0B20720F081E090E00E94430920
:101F900081EF9AE10E94C3498DB79EB708970FB6AB
:101FA000F8949EBF0FBE8DBFEDB7FEB731968E0180
:101FB0000F5F1F4FADB7BEB712961C930E931197CC
:101FC00088E090E0938382838091F61A9091F71ACB
:101FD000958384838091621B90E00196978386832A
:101FE0000E94B6C4F80101900020E9F78DB79EB7B2
:101FF00008960FB6F8949EBF0FBE8DBFC8018E1B0A
:102000009F0B45969695879561E00E949F04C801B5
:102010000E94550628960FB6F894DEBF0FBECDBFBE
:10202000CF91DF911F910F910895EF92FF920F933F
:102030001F93CF93DF938091A30D9091A40DA09156
:10204000A50DB091A60D8093F81A9093F91AA0935C
:10205000FA1AB093FB1A8BE00E949B129093F71A26
:102060008093F61ACCEDDAE1CE0160E270E044E153
:1020700050E00E9459C481E00E949B12BC01FC0107
:1020800001900020E9F73197E81BF90B04E110E01B
:1020900098012E1B3F0B369527952C0F3D1FC9012C
:1020A000AF010E9450C480E090E00E944306CE0140
:1020B00060E270E044E150E00E9459C481E090E0A9
:1020C0000E94430687E10E949B12BC01FC01019023
:1020D0000020E9F73197E81BF90BCE01AF010E9410
:1020E00050C480E10E949B12BC01FC0101900020C1
:1020F000E9F73197E81BF90B98012E1B3F0B36953A
:1021000027952C0F3D1FC901AF010E9450C48AE1E1
:102110000E949B12BC01FC0101900020E9F731975D
:10212000E81BF90B0E1B1F0B0C0F1D1FC801AF0185
:102130000E9450C482E090E00E944306CE0160E21B
:1021400070E044E150E00E9459C48BE10E949B1270
:10215000BC01FC0101900020E9F73197E81BF90B65
:102160009E012E5F3F4FC901AF010E9450C488E11C
:102170000E949B12BC01FC0101900020E9F73197FD
:10218000E81BF90BCE1BDF0B6296CE01AF010E945C
:1021900050C483E090E00E94430681EF9AE10E94E0
:1021A000054ADF91CF911F910F91FF90EF90089515
:1021B0000F931F93CF93DF93CCEDDAE1CE0160E272
:1021C00070E044E150E00E9459C481E00E949B12FB
:1021D000BC01FC0101900020E9F73197E81BF90BE5
:1021E00004E110E098012E1B3F0B369527952C0F2C
:1021F0003D1FC901AF010E9450C480E090E00E94E1
:102200004306CE0160E270E044E150E00E9459C410
:1022100081E090E00E944306CE0160E270E044E17C
:1022200050E00E9459C48FE00E949B12BC01FC0147
:1022300001900020E9F73197E81BF90B0E1B1F0BEB
:10224000169507950C0F1D1FC801AF010E9450C4C1
:1022500082E090E00E944306CE0160E270E044E13B
:1022600050E00E9459C483E090E00E94430681EF51
:102270009AE10E94054ADF91CF911F910F91089535
:102280000F931F93DF93CF930F92CDB7DEB70E94CA
:10229000D8108CE10E949B128C0180E062E00E94C9
:1022A0009F04C8010E94E30480E20E949B12182F41
:1022B000E82FF92FDF010D900020E9F7EA1B8E2FA0
:1022C0008B5E62E099830E949F04812F99810E9416
:1022D000E3048EE10E949B128C0182E063E00E9485
:1022E0009F04C8010E94E30481E20E949B12182F00
:1022F000E82FF92FDF010D900020E9F7EA1B8E2F60
:102300008D5E63E099830E949F04812F99810E94D2
:10231000E3040E9457128BE00E949B129093F71ADD
:102320008093F61A0F90CF91DF911F910F9108952E
:1023300080E20E94E905089586E20E94E905089579
:1023400084E20E94E905089583E20E94E905089568
:1023500082E20E94E905089585E20E94E905089558
:1023600081E20E94E90508958BE10E94E905089544
:102370000F931F93DF93CF93CDB7DEB728970FB698
:10238000F894DEBF0FBECDBF81EF9AE10E94C34932
:102390008DB79EB708970FB6F8949EBF0FBE8DBF3E
:1023A000EDB7FEB731968E010F5F1F4FADB7BEB7C9
:1023B00012961C930E93119788E090E0938382838A
:1023C0008091F61A9091F71A958384838091621B0D
:1023D00090E00196978386830E94B6C4F80101902D
:1023E0000020E9F78DB79EB708960FB6F8949EBF08
:1023F0000FBE8DBFC8018E1B9F0B45969695879586
:1024000061E00E949F04C8010E94550628960FB6FD
:10241000F894DEBF0FBECDBFCF91DF911F910F911A
:1024200008950F931F93DF93CF930F92CDB7DEB72D
:1024300080916B1B882311F480E205C080916C1B96
:10244000882321F48CE10E94DF052BC00E94D81064
:102450008FE30E949B128C0182E063E00E949F0444
:10246000C8010E94E30486E10E949B12182FE82F06
:10247000F92FDF010D900020E9F7EA1B8E2F8D5E0A
:1024800063E099830E949F04812F99810E94E30455
:102490000E9457128BE00E949B129093F71A809330
:1024A000F61A0F90CF91DF911F910F91089510921E
:1024B0009F0D10929E0D80E091E0EEE9FCE0DF01BF
:1024C0009C011D9221503040E1F708950F931F9316
:1024D000CF93DF93BC0120919E0D30919F0D890118
:1024E0000256134F8EEF90E0821B930BEB01099085
:1024F0000020E9F72197C61BD70B8C179D0708F41E
:10250000EC01C801AE010E9470C480919E0D9091B3
:102510009F0D01968C0F9D1FFC01E256F34F108218
:10252000019690939F0D80939E0DC801DF91CF91EE
:102530001F910F9108956F927F928F929F92AF9209
:10254000BF92CF92DF92EF92FF920F931F93DF9390
:10255000CF93CDB7DEB72B970FB6F894DEBF0FBE83
:10256000CDBF8B3908F0A3C0E0909E0DF0909F0D79
:102570002FEFE216F10411F008F099C0870102561E
:10258000134F6FEFC62ED12CCE18DF089091A00DFF
:10259000992309F464C0282F30E04091A10D509197
:1025A000A20D2417350708F05AC0C901880F991FDA
:1025B00088509048BE016F5F7F4F42E00E94F75005
:1025C00089819A8136E1C316D10414F024E102C056
:1025D0002C2D215040EF842E4FE7942E880E991E0B
:1025E0005801CC2433E0632E712C6C0E7D1E28C064
:1025F000D22E293010F098E0D92EC401B3014D2D10
:102600002B870E94F750F30180E090E04D2D50E0C1
:102610002B850FC03081D5013C9331910196332336
:1026200029F4FC01EC0DF11D6F0112C00894A11CEE
:10263000B11C8417950774F3CD0C2D19840E951ECB
:102640002223B1F6D5011C92DD240894C11CD11CB3
:10265000CE0CDF1CD0929F0DC0929E0D2AC0E82F99
:10266000F0E0EE0FFF1FEA5BFD4F20813181211565
:102670003105E9F080E090E005C0F801E80FF91FAE
:1026800040830196F901E80FF91F4491442319F0A2
:102690008C159D0594F3F801E80FF91F108201963F
:1026A0008E0D9F1D90939F0D80939E0D02C00CE791
:1026B00013E0C8012B960FB6F894DEBF0FBECDBF56
:1026C000CF91DF911F910F91FF90EF90DF90CF900E
:1026D000BF90AF909F908F907F906F9008950F93D1
:1026E0001F93DF93CF9300D000D0CDB7DEB780EF3C
:1026F0009FE78E010F5F1F4FB80144E00E94F75023
:10270000C80161E372E00E9460C49C0180E0211571
:10271000310509F481E08093A00D882349F0809170
:10272000F67F9091F77F61EA7DE042E00E94F750EA
:102730000F900F900F900F90CF91DF911F910F91FD
:1027400008958CE094E00E94D367BC018091F21A56
:10275000882321F064601092F21A04C06B7F81E03C
:102760008093F21A8CE094E00E94A46B08958CE0B0
:1027700094E00E94D3672091F11A222329F0BC0132
:102780006E7F1092F11A05C081E08093F11A61E02A
:1027900070E08CE094E00E94A46B0895CF93DF93E7
:1027A0008CE094E00E94D367EC01C2608CE094E07E
:1027B000BE010E94A46B8FE79AE1A6E08150904091
:1027C000A040E1F700C00000BE016D7F8CE094E006
:1027D0000E94A46BDF91CF9108950E9456560E94EB
:1027E0006B560895EF92FF920F931F93CF93DF9351
:1027F000CCEDDAE1CE0160E270E044E150E00E940D
:1028000059C46091F51A7091F61ADB01FD0101902F
:102810000020E9F73197EA1BFB0BCE01AF010E94C4
:1028200050C48091F21A882329F06091FB1A7091AC
:10283000FC1A04C06091FD1A7091FE1AFB01019010
:102840000020E9F73197E61BF70B20EF3AE1CCEDDA
:10285000DAE12E1B3F0BC901AF010E9450C480E09A
:1028600090E00E944306CE0160E270E044E150E057
:102870000E9459C46091F71A7091F81ADB01FD01AA
:1028800001900020E9F73197EA1BFB0BCE01AF0165
:102890000E9450C48091F11A882329F06091FB1A9C
:1028A0007091FC1A04C06091FD1A7091FE1AFB0130
:1028B00001900020E9F73197E61BF70B04E110E0E7
:1028C00098012E1B3F0BCCEDDAE12C0F3D1FC90107
:1028D000AF010E9450C481E090E00E944306CE0107
:1028E00060E270E044E150E00E9459C46091F71A40
:1028F0007091F81ADB01FD0101900020E9F7319792
:10290000EA1BFB0BCE01AF010E9450C46091F91A83
:102910007091FA1ADB01FD0101900020E9F731976F
:10292000EA1BFB0B0E1B1F0B0C0F1D1FC801AF0179
:102930000E9450C482E090E00E944306CE0160E213
:1029400070E044E150E00E9459C46091F31A709124
:10295000F41ADB01FD0101900020E9F73197EA1B31
:10296000FB0B2EEE3AE12E1B3F0BC901AF010E947B
:1029700050C483E090E00E944306DF91CF911F9105
:102980000F91FF90EF90089582E20E949B12909326
:10299000F41A8093F31A8BE10E949B129093F61A1B
:1029A0008093F51A83E20E949B129093F81A809309
:1029B000F71A84E20E949B129093FA1A8093F91AF4
:1029C0008DE70E949B129093FC1A8093FB1A8EE76E
:1029D0000E949B129093FE1A8093FD1A8CE094E063
:1029E0000E94D367282F21702093F11A969587951E
:1029F00096958795809581708093F21A0E94F213C4
:102A000008958091A30D9091A40DA091A50DB09172
:102A1000A60D8093F21A9093F31AA093F41AB09330
:102A2000F51A8091F11A882311F484E001C08150D5
:102A30008093F11A08958091A30D9091A40DA09117
:102A4000A50DB091A60D8093F21A9093F31AA0935E
:102A5000F41AB093F51A8091F11A843018F010929C
:102A6000F11A08958F5F8093F11A08958091A30D54
:102A70009091A40DA091A50DB091A60D8093F21A8E
:102A80009093F31AA093F41AB093F51A0E94565635
:102A90000E946B560895CF93DF93CCEDDAE1CE011F
:102AA00060E270E044E150E00E9459C48DB79EB7E7
:102AB0000E970FB6F8949EBF0FBE8DBFEDB7FEB751
:102AC0003196ADB7BEB71296DC93CE93119786E9D7
:102AD00093E09383828380915B1B90915C1B958331
:102AE000848380915D1B90E001969783868380911B
:102AF0005E1B8087118680915F1B82871386809181
:102B0000601B848715860E94F4C48DB79EB70E960D
:102B10000FB6F8949EBF0FBE8DBF80E090E00E947C
:102B200043068091A30D9091A40DA091A50DB091A5
:102B3000A60D2091F21A3091F31A4091F41A509197
:102B4000F51A821B930BA40BB50B853F21E092076E
:102B500020E0A20720E0B20720F081E090E00E9490
:102B60004309DF91CF9108958BE59BE10E947E1D83
:102B70001092611B0E944B150895EF92FF92CF9324
:102B8000DF938091A30D9091A40DA091A50DB0911C
:102B9000A60D8093F21A9093F31AA093F41AB093AF
:102BA000F51A8BE59BE10E947E1D1092611B0E942D
:102BB0004B15CCEDDAE1CE0160E270E044E150E08B
:102BC0000E9459C481E090E00E94430682E30E9483
:102BD0009B12BC01FC0101900020E9F73197E81B32
:102BE000F90B9E012E1B3F0B2C5E3F4FC901AF011D
:102BF0000E9450C482E090E00E944306CE0160E251
:102C000070E044E150E00E9459C48BE10E949B12A5
:102C1000BC01FC0101900020E9F73197E81BF90B9A
:102C20009E012E5F3F4FC901AF010E9450C489E150
:102C30000E949B12BC01FC0101900020E9F7319732
:102C4000E81BF90BCE1BDF0B6296CE01AF010E9491
:102C500050C483E090E00E944306DF91CF91FF9043
:102C6000EF9008958CED9AE160E270E044E150E06D
:102C70000E9459C48091F11A8230B9F0833018F45F
:102C8000813029F40BC08330B9F08430E1F06091D9
:102C9000321B7091331B21E030E01BC06091341B6C
:102CA0007091351B26E030E014C06091361B7091A6
:102CB000371B29E030E00DC06091381B7091391B43
:102CC0002EE030E006C060913A1B70913B1B20E182
:102CD00030E0FB0101900020E9F73197E61BF70B8C
:102CE0002452354EC901AF010E9450C481E090E0EA
:102CF0000E94430608950E944B150E9432160895C3
:102D00008091A30D9091A40DA091A50DB091A60D59
:102D10008093F21A9093F31AA093F41AB093F51AD1
:102D200084E59BE10E947E1D8BE59BE10E94E61AF3
:102D30009091581B80915F1B9817B9F49091571B85
:102D400080915E1B981789F49091561B80915D1BB2
:102D5000981759F42091541B3091551B80915B1B9F
:102D600090915C1B2817390719F083E080931111AB
:102D70000895EF92FF92CF93DF938091A30D9091EE
:102D8000A40DA091A50DB091A60D8093F21A909379
:102D9000F31AA093F41AB093F51A8BE59BE10E9405
:102DA0007E1D1092611B84E08093F11A0E944B15E6
:102DB0000E943216CCEDDAE1CE0160E270E044E12F
:102DC00050E00E9459C48AE20E949B12BC01FC019F
:102DD00001900020E9F73197E81BF90BCE01AF0114
:102DE0000E9450C482E30E949B12BC01FC0101902E
:102DF0000020E9F73197E81BF90B9E012E1B3F0BD2
:102E00002C5E3F4FC901AF010E9450C482E090E0A8
:102E10000E944306CE0160E270E044E150E00E946F
:102E200059C48BE20E949B12BC01FC01019000205E
:102E3000E9F73197E81BF90B9E012E5F3F4FC9015F
:102E4000AF010E9450C488E10E949B12BC01FC01AA
:102E500001900020E9F73197E81BF90BCE1BDF0B3F
:102E60006296CE01AF010E9450C483E090E00E94C0
:102E700043060E94571285E20E949B129093331BD7
:102E80008093321B86E20E949B129093351B8093A5
:102E9000341B87E20E949B129093371B8093361B52
:102EA00088E20E949B129093391B8093381B89E221
:102EB0000E949B1290933B1B80933A1BDF91CF9112
:102EC000FF90EF9008950E94571285E20E949B1296
:102ED0009093331B8093321B86E20E949B12909347
:102EE000351B8093341B87E20E949B129093371B03
:102EF0008093361B88E20E949B129093391B80932B
:102F0000381B89E20E949B1290933B1B80933A1BD3
:102F10008EE00E94E90508958091A30D9091A40D83
:102F2000A091A50DB091A60D8093F21A9093F31A7B
:102F3000A093F41AB093F51A8091F11A8230E1F05F
:102F4000833018F4813029F412C0833031F1843099
:102F500071F180915B1B90915C1B27E08A3D920789
:102F600088F1019790935C1B80935B1B08958BE520
:102F70009BE10E94D619089580915E1B823048F42F
:102F80008BE59BE10E94D6198BE59BE10E94C91855
:102F900001C0815080935E1B089580915F1B882340
:102FA00011F487E101C0815080935F1B08958091E7
:102FB000601B882321F48BE38093601B089581506C
:102FC0008093601B08958BE59BE10E94DB188BE5E5
:102FD0009BE10E94C91890915E1B891718F4981BF9
:102FE00090935E1B08951F938091A30D9091A40D63
:102FF000A091A50DB091A60D8093F21A9093F31AAB
:10300000A093F41AB093F51A8091F11A8230D1F09E
:10301000833018F4813029F412C0833029F18430D0
:1030200071F180915B1B90915C1B27E08F3E9207B2
:1030300080F5019690935C1B80935B1B2AC00E94D5
:10304000E31727C010915E1B8BE59BE10E94C91816
:10305000181720F00E94E31781E003C080915E1BE7
:103060008F5F80935E1B15C080915F1B873118F0C6
:1030700010925F1B0EC08F5F80935F1B0AC0809110
:10308000601B8B3318F01092601B03C08F5F80931E
:10309000601B1F9108951F920F920FB60F9211247B
:1030A0008F939F93AF93BF938091A30D9091A40DA5
:1030B000A091A50DB091A60D0196A11DB11D809303
:1030C000A30D9093A40DA093A50DB093A60D88ED2C
:1030D0008093850083EF80938400BF91AF919F918F
:1030E0008F910F900FBE0F901F901895DC01CB01B0
:1030F0002EE0B695A795979587952A95D1F78F716C
:103100009070A070B07088319105A105B10520F0D4
:1031100087E190E0A0E0B0E00895BB27A92F982FA9
:10312000872F8F739070A070B0708C339105A105BC
:10313000B10520F08BE390E0A0E0B0E0089510929C
:10314000800082E08093810088ED8093850083EF8A
:10315000809384001092870010928600109289005C
:103160001092880010928B0010928A0010928D00AD
:1031700010928C0081E080936F00089510926F0090
:10318000089520E083709070009709F421E0822F69
:103190000895FC01928120813181E92FF0E0ED5109
:1031A000FC4F8081913031F423703070211531054E
:1031B00009F48DE10895FC0182818B3070F08081EB
:1031C000918127E08F3E920710F080E008950196EC
:1031D00091838083128281E008958F5F828381E0F2
:1031E0000895FC01828120813181A82FB0E0AD518A
:1031F000BC4F9C91813031F4237030702115310522
:1032000009F49DE18381860F8383981710F081E094
:103210000895891B8383CF010E94DB18089567E01E
:1032200070E00E94F118089561E070E00E94F118CA
:1032300008958F929F92AF92BF92DF92EF92FF928A
:103240000F931F93DF93CF93CDB7DEB727970FB6BA
:10325000F894DEBF0FBECDBF8C01DE011196FC01DC
:1032600087E001900D928150E1F7A980BA80DB8060
:10327000EC80FD80F8012481CB01820F911D9C011F
:1032800068E170E00E9417C3862E972E88E1869F22
:10329000802D1124281B248306C0C8010E94141904
:1032A00008948108910881149104B9F7F80180818C
:1032B0009181A816B90659F48281D81641F4838108
:1032C000E81629F480E090E02481F21611F081E004
:1032D00090E027960FB6F894DEBF0FBECDBFCF911A
:1032E000DF911F910F91FF90EF90DF90BF90AF9013
:1032F0009F908F900895AF92BF92DF92EF92FF92CE
:103300000F931F93DF93CF93CDB7DEB727970FB6F9
:10331000F894DEBF0FBECDBF8C01DE011196FC011B
:1033200087E001900D928150E1F7A980BA80DB809F
:10333000EC80FD80F8012581CB01820F911D9C015D
:103340008C33910570F06CE370E00E9417C38CE33E
:10335000689F802D1124281B2583C8010E941919FC
:1033600002C0F8018583F80180819181A816B90611
:1033700059F48281D81641F48381E81629F480E05B
:1033800090E02481F21611F081E090E027960FB6CC
:10339000F894DEBF0FBECDBFCF91DF911F910F918B
:1033A000FF90EF90DF90BF90AF900895FC01828175
:1033B000882379F48081918127E08A3D920710F477
:1033C00080E008950197918380838BE0828381E080
:1033D00008958150828381E00895CF93DF93EC01BB
:1033E0008B818830D8F4CE010E94D619813011F03B
:1033F00080E017C08A8128813981E82FF0E0ED5103
:10340000FC4F9081813031F42370307021153105EB
:1034100009F49DE18B818750890F01C087508B8310
:1034200081E0DF91CF910895CF93DF93EC018B8101
:103430008230B0F4CE010E94D6198823A1F09A817F
:1034400028813981E92FF0E0ED51FC4F80819130E6
:1034500041F4237030702115310519F48DE101C05C
:1034600081508B8381E0DF91CF910895EF92FF929D
:103470000F931F93FC016081718189ED97E020E03B
:1034800030E0A9010FC0DC01A370B070109729F4DF
:1034900022593E4F4F4F5F4F04C023593E4F4F4F6D
:1034A0005F4F01968617970770F3E280A3EEB3E0B3
:1034B00080E0637070700DC09C91813021F46115C3
:1034C000710509F49DE1290F311D411D511D8F5FCB
:1034D00011968E1589F77381858190E0A0E0B0E0A8
:1034E000BA2FA92F982F8827E480FF2400E010E04E
:1034F0006EE0EE0CFF1C001F111F6A95D1F78E299C
:103500009F29A02BB12B6681660F660FE62EFF2444
:1035100000E010E08E299F29A02BB12B270F311D31
:10352000411D511D203060E2360760E0460760E033
:10353000560720F02FEF3FE140E050E063E1220F1B
:10354000331F441F551F6A95D1F7282B392B4A2B5F
:103550005B2BB901CA011F910F91FF90EF90089565
:103560000895CF92DF92EF92FF920F931F938AE01C
:1035700090E040E050E0BA010EEF1FEF2FEF3FEF79
:10358000CC24DD2476010E94632A1F910F91FF90C5
:10359000EF90DF90CF900895DF93CF9300D000D0CD
:1035A000CDB7DEB769837A838B839C8380E094E018
:1035B000BE016F5F7F4F42E050E00E94156B0F909D
:1035C0000F900F900F90CF91DF910895EF92FF929F
:1035D0000F931F930E94361A7B018C010E94CC1A14
:1035E000C801B7014AE050E00E94252A8091A30D4E
:1035F0009091A40DA091A50DB091A60D8093A70D5B
:103600009093A80DA093A90DB093AA0D1F910F91AF
:10361000FF90EF900895EF92FF920F931F93DF9327
:10362000CF93CDB7DEB728970FB6F894DEBF0FBEA5
:10363000CDBF05E0E02EF12CEC0EFD1E8E010F5FDC
:103640001F4F80E094E0B70142E050E00E94B16774
:1036500080E094E0B80142E050E00E94B167298127
:103660003A814B815C818D819E81AF81B88528171D
:1036700039074A075B0728F3B901CA0128960FB634
:10368000F894DEBF0FBECDBFCF91DF911F910F9198
:10369000FF90EF9008952F923F924F925F926F921A
:1036A0007F928F929F92AF92BF92CF92DF92EF92D2
:1036B000FF920F931F93DF93CF93CDB7DEB7289779
:1036C0000FB6F894DEBF0FBECDBF182F0E940B1BA4
:1036D0002B013C01113009F426C10E94B11A9B0153
:1036E000AC015B016C01F3E1D694C794B794A79445
:1036F000FA95D1F7D301C201E3E1B695A795979565
:103700008795EA95D1F789549F4FAF4FBF4F8A15E0
:103710009B05AC05BD0508F001C1112319F401E0BA
:1037200010E019C1E090A30DF090A40D0091A50D3B
:103730001091A60D8091A70D9091A80DA091A90DB3
:10374000B091AA0DE81AF90A0A0B1B0BDA01C9019C
:103750007EE0B695A795979587957A95D1F78F7165
:103760009070A070B07088319105A105B10520F06E
:1037700087E190E0A0E0B0E0282E3324BB27A52FFE
:10378000942F832F8F739070A070B0708C3391053D
:10379000A105B10520F08BE390E0A0E0B0E0482E59
:1037A0005524307040705070203F3105410551055F
:1037B00020F02FEE30E040E050E0622F70E078879C
:1037C0006F83C801B70120E036ED43E850E00E9466
:1037D0003EC329833A834B835C8369817A818B81E1
:1037E0009C8120E036ED43E850E00E94ECC2E61AEE
:1037F000F70A080B190BC801B70120E43EE745E0C2
:1038000050E00E943EC33E832D83390188249924D1
:10381000C401B30120E43EE745E050E00E94ECC261
:10382000E61AF70A080B190BC401B30120E737E1C8
:1038300040E050E00E94ECC2A8019701261B370B24
:10384000480B590BCA01B90129E130E040E050E0D2
:103850000E943EC36F817885620F731F78876F83E4
:10386000603F710538F0605F704078876F8308941F
:10387000411C511CC801B70120E737E140E050E08E
:103880000E943EC3240D351D2C33310528F02C53E6
:1038900030400894211C311C8D819E81820D931D26
:1038A0008831910530F048970894A11CB11CC11CC7
:1038B000D11C422E552466247724762C652C542C5A
:1038C00044247F81272F30E040E050E0422A532AF1
:1038D000642A752A29813A814B815C81A20EB31E2C
:1038E000C41ED51E33E1AA0CBB1CCC1CDD1C3A95B2
:1038F000D1F74A285B286C287D2890E0A0E0B0E052
:103900002EE0880F991FAA1FBB1F2A95D1F7482ABE
:10391000592A6A2A7B2A01E010E007C0112319F412
:1039200000E010E018C000E010E0C301B2014AE07E
:1039300050E00E94252A8091A30D9091A40DA091A2
:10394000A50DB091A60D8093A70D9093A80DA093FF
:10395000A90DB093AA0DC80128960FB6F894DEBF42
:103960000FBECDBFCF91DF911F910F91FF90EF90D0
:10397000DF90CF90BF90AF909F908F907F906F908F
:103980005F904F903F902F9008956F927F928F920B
:103990009F92AF92BF92CF92DF92EF92FF920F93DE
:1039A0001F93CF93DF937B018C01EA015B016C01D4
:1039B00033E1D694C794B794A7943A95D1F787E0AA
:1039C000DA011D928A95E9F789ED97E09C01237051
:1039D00030702115310529F42EE631E040E050E049
:1039E00004C02DE631E040E050E0BC016F5F7F4F46
:1039F000A216B306C406D50630F0A21AB30AC40A4A
:103A0000D50ACB01E3CF998388831A829A812881D2
:103A10003981E92FF0E0ED51FC4F8081913031F494
:103A2000237030702115310509F48DE1682E77245B
:103A3000882499246A147B048C049D0440F4CE01EC
:103A40000E94DB18A618B708C808D908DFCF9A2D3E
:103A5000AB828A1528F4981B9B83CE010E94DB1849
:103A6000D801C7012EE0B695A795979587952A9519
:103A7000D1F78F719070A070B07088319105A10559
:103A8000B10520F087E190E0A0E0B0E08C83BB2797
:103A9000A12F902F8F2D8F739070A070B0708C33EA
:103AA0009105A105B10520F08BE390E0A0E0B0E026
:103AB0008D838FEF90E0A0E0B0E0E822F9220A23A6
:103AC0001B2390EFE916F1040105110528F0AFEE74
:103AD000EA2EF12C012D112DE694E694EE82DF9171
:103AE000CF911F910F91FF90EF90DF90CF90BF90FB
:103AF000AF909F908F907F906F900895CF93DF93BA
:103B0000EC010E940B1BAE010E94C51CDF91CF91FE
:103B100008958091A30D9091A40DA091A50DB09151
:103B2000A60D2091F11A3091F21A4091F31A50919A
:103B3000F41A821B930BA40BB50B2091F51A2230BB
:103B400048F4893E23E0920720E0A20720E0B20774
:103B500048F408958D3221E0920720E0A20720E08A
:103B6000B20710F00E94C205089584E094E00E941C
:103B7000D367BC01707F84E094E00E94A46B0E9434
:103B8000C2050895EF92FF920F931F93CF93DF9397
:103B900084E094E00E94D367BC01707F84E094E0ED
:103BA0000E94A46B8091A30D9091A40DA091A50DEE
:103BB000B091A60D8093F11A9093F21AA093F31A84
:103BC000B093F41A1092F51ACCEDDAE1CE0160E26E
:103BD00070E044E150E00E9459C484E00E949B12CE
:103BE000BC01FC0101900020E9F73197E81BF90BBB
:103BF0008E010C5F1F4FC801AF010E9450C480E0CE
:103C000090E00E944306CE0160E270E044E150E0A3
:103C10000E9459C485E00E949B12BC01FC010190E6
:103C20000020E9F73197E81BF90BC801AF010E94AA
:103C300050C481E090E00E944306CE0160E270E053
:103C400044E150E00E9459C485E40E949B12BC01EB
:103C5000FC0101900020E9F73197E81BF90BCE0138
:103C6000AF010E9450C482E090E00E944306CE0162
:103C700060E270E044E150E00E9459C483E090E0CB
:103C80000E94430686EB96E060E00E948E4980E049
:103C900060E00E946B49DF91CF911F910F91FF90DF
:103CA000EF9008951F93182F1295107F8EEC98E0D7
:103CB00060E0712F40E050EF0E94CF6B8EED98E0F6
:103CC00060E0712F40E050EF0E94CF6B1F9108958C
:103CD00080E00E94521E85E094E00E94D367BC0100
:103CE000607F85E094E00E94A46B0895EF92FF92BC
:103CF000CF93DF9384E094E00E94D367BC01707F90
:103D00007A6084E094E00E94A46B8091F51A8F5F42
:103D10008093F51A813009F066C08091A30D9091CF
:103D2000A40DA091A50DB091A60D8093F11A9093CA
:103D3000F21AA093F31AB093F41A0E94681E80E05E
:103D40000E9435648CED9AE160E270E044E150E05D
:103D50000E9459C486E00E949B12BC01FC010190A4
:103D60000020E9F73197E81BF90BC0EEDAE1CE014C
:103D7000AF010E9450C480E090E00E944306CE0153
:103D8000049760E270E044E150E00E9459C487E08B
:103D90000E949B12BC01FC0101900020E9F73197C1
:103DA000E81BF90BCE01AF010E9450C481E090E006
:103DB0000E944306CE01049760E270E044E150E0C7
:103DC0000E9459C482E090E00E94430683E090E0A4
:103DD0000E94430686EB96E060E00E948E4980E0F8
:103DE00060E00E946B49DF91CF91FF90EF900895C2
:103DF0000E94681E84E00E9435640E94C2050895F6
:103E000085E094E00E94D367BC01607F656085E037
:103E100094E00E94A46B82E00E94521E0E94C205A0
:103E20000895EF92FF92CF93DF938CED9AE160E2D9
:103E300070E044E150E00E9459C483E00E949B126C
:103E4000BC01FC0101900020E9F73197E81BF90B58
:103E5000C0EEDAE1CE01AF010E9450C480E090E0F4
:103E60000E94430681E160E00E949F048091621BF2
:103E700090E001966FEE73E042E00E945806CE019A
:103E8000049760E270E044E150E00E9459C48DE183
:103E90000E949B12BC01FC0101900020E9F73197C0
:103EA000E81BF90BCE01AF010E9450C485E094E0FD
:103EB0000E94D3678F7090708530910511F481E86E
:103EC00001C082E80E949B12BC01FC01019000200D
:103ED000E9F73197E81BF90BC6EEDAE1CE01AF0145
:103EE0000E9450C481E090E00E9443062A97CE01D0
:103EF00060E270E044E150E00E9459C485E40E9411
:103F00009B12BC01FC0101900020E9F73197E81BEE
:103F1000F90BCE01AF010E9450C487E40E949B12AE
:103F2000BC01FC0101900020E9F73197E81BF90B77
:103F300020EF3AE12E1B3F0BC901AF010E9450C494
:103F400082E090E00E944306CE0160E270E044E12E
:103F500050E00E9459C488E40E949B12BC01FC01FD
:103F600001900020E9F73197E81BF90B2DEE3AE1BB
:103F70002E1B3F0BC901AF010E9450C483E090E0AB
:103F80000E94430686EB96E060E00E948E4980E046
:103F900060E00E946B49DF91CF91FF90EF90089510
:103FA00081E00E944B1B82E06BE57BE10E942BAB22
:103FB0008AE10E94DF05089589E10E94DF050895E6
:103FC000EF92FF920F931F93DF93CF93CDB7DEB79E
:103FD00028970FB6F894DEBF0FBECDBF8091A30D1A
:103FE0009091A40DA091A50DB091A60D8093F11A0A
:103FF0009093F21AA093F31AB093F41A1092F51A50
:104000000CED1AE1C80160E270E044E150E00E946A
:1040100059C482E00E949B12BC01FC010190002067
:10402000E9F73197E81BF90B98012B5F3F4FC90166
:10403000AF010E9450C480E090E00E944306C80196
:1040400060E270E044E150E00E9459C48DB79EB731
:104050000A970FB6F8949EBF0FBE8DBFEDB7FEB79F
:1040600031967E010894E11CF11CADB7BEB71296E3
:10407000FC92EE92119788E090E09383828384EF24
:1040800093E09583848382E090E09783868389E23E
:1040900090E0918780870E94B6C4F70101900020CC
:1040A000E9F73197EE19FF099801285F3F4F8DB767
:1040B0009EB70A960FB6F8949EBF0FBE8DBFC9017A
:1040C000B701AF010E9450C481E090E00E94430616
:1040D000C80160E270E044E150E00E9459C485E408
:1040E0000E949B12BC01FC0101900020E9F731976E
:1040F000E81BF90BC801AF010E9450C486E40E947E
:104100009B12BC01FC0101900020E9F73197E81BEC
:10411000F90B98012E1B3F0B2C5E3F4FC901AF01DD
:104120000E9450C482E090E00E944306C80160E211
:1041300070E044E150E00E9459C48FE10E949B125C
:10414000BC01FC0101900020E9F73197E81BF90B55
:104150000E1B1F0B0E5E1F4FC801AF010E9450C403
:1041600083E090E00E94430686EB96E060E00E94C8
:104170008E4980E060E00E946B4928960FB6F89463
:10418000DEBF0FBECDBFCF91DF911F910F91FF908A
:10419000EF900895E091FA1AF0E0E05DF14E808131
:1041A0008F3F11F481E309C0893311F481E405C024
:1041B000863411F480E301C08F5F808308952091DD
:1041C000FA1A30E0F901E05DF14E80818F3F11F085
:1041D000803329F4205D314E86E4F90105C0813435
:1041E00011F489E301C08150808308958091FA1A07
:1041F000882311F0815001C083E08093FA1A08955A
:104200008091FA1A833020F48F5F8093FA1A089510
:104210001092FA1A08958FEF8093301E8093311E0A
:104220008093321E8093331E089580E09091081B86
:10423000992309F481E08093081B089580E0909110
:10424000091B992309F481E08093091B0895AF921B
:10425000BF92CF92DF92EF92FF920F931F93CF9373
:10426000DF938091091BC82FD0E0CC0FDD1FCC0F4E
:10427000DD1FCF50D54E6D817E818F81988520E0E6
:1042800030E040E85FE30E9422C06D837E838F832D
:1042900098878091091BC82FD0E0CC0FDD1FCC0F71
:1042A000DD1FCF50D54EAD80BE80CF80D884E0904A
:1042B000021BF090031B0091041B1091051BC6010B
:1042C000B501A80197010E94D5C11816B4F4C80120
:1042D000B7012091FE1A3091FF1A4091001B5091B6
:1042E000011B0E9421C09B01AC01C601B5010E94C7
:1042F00021C06D837E838F83988781E080930B1B21
:1043000080910C1B863099F085E080930C1B809186
:10431000A30D9091A40DA091A50DB091A60D809331
:104320000D1B90930E1BA0930F1BB093101BDF91DE
:10433000CF911F910F91FF90EF90DF90CF90BF90A2
:10434000AF900895AF92BF92CF92DF92EF92FF921B
:104350000F931F93CF93DF938091091BC82FD0E059
:10436000CC0FDD1FCC0FDD1FCF50D54E6D817E8170
:104370008F81988520E030E040E85FE30E9421C013
:104380006D837E838F8398878091091BC82FD0E02F
:10439000CC0FDD1FCC0FDD1FCF50D54EAD80BE80C2
:1043A000CF80D884E090FE1AF090FF1A0091001B95
:1043B0001091011BC601B501A80197010E9486C09A
:1043C0008823B4F46091021B7091031B8091041B3D
:1043D0009091051BA80197010E9421C09B01AC018F
:1043E000C601B5010E9422C06D837E838F839887AA
:1043F00081E080930B1B80910C1B883099F087E043
:1044000080930C1B8091A30D9091A40DA091A50DFC
:10441000B091A60D80930D1B90930E1BA0930F1BC4
:10442000B093101BDF91CF911F910F91FF90EF90F0
:10443000DF90CF90BF90AF900895AF92BF92CF9290
:10444000DF92EF92FF920F931F93CF93DF938091B0
:10445000091BC82FD0E0CC0FDD1FCC0FDD1FCF50C4
:10446000D54E6D817E818F8198852DEC3CEC4CEC96
:104470005DE30E9421C06D837E838F839887809146
:10448000091BC82FD0E0CC0FDD1FCC0FDD1FCF5094
:10449000D54EAD80BE80CF80D884E090FE1AF090DB
:1044A000FF1A0091001B1091011BC601B501A80164
:1044B00097010E9486C08823B4F46091021B70911A
:1044C000031B8091041B9091051BA80197010E947A
:1044D00021C09B01AC01C601B5010E9422C06D83C1
:1044E0007E838F83988781E080930B1B80910C1BC8
:1044F0008C3099F08BE080930C1B8091A30D9091F0
:10450000A40DA091A50DB091A60D80930D1B9093C5
:104510000E1BA0930F1BB093101BDF91CF911F9127
:104520000F91FF90EF90DF90CF90BF90AF900895E4
:10453000AF92BF92CF92DF92EF92FF920F931F93B1
:10454000CF93DF938091091BC82FD0E0CC0FDD1FE4
:10455000CC0FDD1FCF50D54E6D817E818F81988528
:104560002DEC3CEC4CEC5DE30E9422C06D837E831D
:104570008F8398878091091BC82FD0E0CC0FDD1F57
:10458000CC0FDD1FCF50D54EAD80BE80CF80D884FC
:10459000E090021BF090031B0091041B1091051B7F
:1045A000C601B501A80197010E94D5C18823B4F0C6
:1045B000C801B7012091FE1A3091FF1A4091001BEB
:1045C0005091011B0E9421C09B01AC01C601B501A5
:1045D0000E9421C06D837E838F83988781E08093C2
:1045E0000B1B80910C1B8A3099F089E080930C1B87
:1045F0008091A30D9091A40DA091A50DB091A60D51
:1046000080930D1B90930E1BA0930F1BB093101B58
:10461000DF91CF911F910F91FF90EF90DF90CF909E
:10462000BF90AF900895E091091BF0E0EE0FFF1FDF
:10463000EF50F54E858196812091FC1A3091FD1A3C
:104640008217930714F4019604C08091FA1A90918E
:10465000FB1A9683858381E080930B1B90910C1B42
:10466000923091F080930C1B8091A30D9091A40D3A
:10467000A091A50DB091A60D80930D1B90930E1BDC
:10468000A0930F1BB093101B0895E091091BF0E05D
:10469000EE0FFF1FEF50F54E858196812091FA1A9B
:1046A0003091FB1A2817390714F4019704C0809140
:1046B000FC1A9091FD1A9683858381E080930B1BF1
:1046C00080910C1B843099F083E080930C1B8091C7
:1046D000A30D9091A40DA091A50DB091A60D80936E
:1046E0000D1B90930E1BA0930F1BB093101B0895EE
:1046F00086EF9AE160E37EE144E050E00E9443C42B
:104700000097C1F120E030E08091331E863411F42F
:1047100021E030E080E090E04091321E463411F418
:1047200081E090E02823392390E08091311E863487
:1047300009F491E080E04091301E463409F481E0B4
:10474000892390E082239323009761F48FEF809375
:10475000301E8093311E8093321E8093331E109240
:10476000FA1A089580E39EE160E070E044E050E0D2
:104770000E941B2A0E94C20508958091301E8F3F1F
:1047800061F48091311E8F3F41F48091321E8F3F42
:1047900021F48091331E8F3F89F080E39EE160E039
:1047A00070E044E050E00E941B2A8FEF8093301E9F
:1047B0008093311E8093321E8093331E82E00E94CC
:1047C000E90508958AE00E94E905089584E00E94C1
:1047D000E90508958CED9AE160E270E044E150E073
:1047E0000E9459C48BE58093DC1A8091301E8F3F64
:1047F00009F480E28093DD1A8091311E8F3F09F425
:1048000080E28093DE1A8091321E8F3F09F480E2AD
:104810008093DF1A8091331E8F3F09F480E28093EA
:10482000E01A8DE58093E11A81E090E00E94430652
:104830008091FA1A8F5F61E00E949F048EE00E94CF
:10484000350408958DE50E949B129093121B80936E
:10485000111B8CE50E949B129093141B8093131BD9
:104860000895EF92FF920F931F93CF93DF938FEFF3
:104870008093301E8093311E8093321E8093331EAE
:104880001092FA1ACCEDDAE1CE0160E270E044E178
:1048900050E00E9459C488E00E949B12BC01FC01B8
:1048A00001900020E9F73197E81BF90B04E110E0D3
:1048B00098012E1B3F0B369527952C0F3D1FC901E4
:1048C000AF010E9450C480E090E00E9443060E9425
:1048D000EA23CE0160E270E044E150E00E9459C456
:1048E0008AE20E949B12BC01FC0101900020E9F7C2
:1048F0003197E81BF90BCE01AF010E9450C48DE443
:104900000E949B12BC01FC0101900020E9F7319745
:10491000E81BF90B0E1B1F0B0C0F1D1FC801AF016D
:104920000E9450C482E090E00E944306CE0160E203
:1049300070E044E150E00E9459C48BE20E949B1257
:10494000BC01FC0101900020E9F73197E81BF90B4D
:104950009E012E5F3F4FC901AF010E9450C48CE4FD
:104960000E949B12BC01FC0101900020E9F73197E5
:10497000E81BF90BCE1BDF0B6296CE01AF010E9444
:1049800050C483E090E00E944306DF91CF911F91D5
:104990000F91FF90EF900895CF93DF93CCEDDAE184
:1049A000CE0160E270E044E150E00E9459C481E031
:1049B0000E949B12BC01FC0101900020E9F7319795
:1049C000E81BF90B24E130E02E1B3F0B36952795B1
:1049D0002C0F3D1FC901AF010E9450C480E090E040
:1049E0000E944306CE0160E270E044E150E00E9484
:1049F00059C481E090E00E944306DF91CF91089571
:104A000080E061E041E00E941C6408958BE00E9418
:104A1000DF0508958091FB1A882319F084E10E9434
:104A2000DF05089582E10E94DF0508958FE00E946E
:104A3000DF0508950F931F93DF93CF93CDB7DEB7B4
:104A400028970FB6F894DEBF0FBECDBF8DB79EB7C7
:104A500008970FB6F8949EBF0FBE8DBFEDB7FEB797
:104A600031968E010F5F1F4FADB7BEB712961C93E4
:104A70000E93119788E090E0938382838091321B9C
:104A80009091331B958384838091651B90E0019600
:104A9000978386830E94B6C4F80101900020E9F74D
:104AA0008DB79EB708960FB6F8949EBF0FBE8DBF08
:104AB000C8018E1B9F0B45969695879561E00E94D5
:104AC0009F04C8010E94550628960FB6F894DEBFD1
:104AD0000FBECDBFCF91DF911F910F9108950E941E
:104AE0001A2581EF9AE10E94C3490895EF92FF923F
:104AF000CF93DF930E94CC24CCEDDAE1CE0160E2CB
:104B000070E044E150E00E9459C48AE50E949B1283
:104B1000BC01FC0101900020E9F73197E81BF90B7B
:104B2000CE01AF010E9450C481E10E949B12BC01E2
:104B3000FC0101900020E9F73197E81BF90B24E113
:104B400030E02E1B3F0B369527952C0F3D1FC901DA
:104B5000AF010E9450C482E090E00E944306CE0163
:104B600060E270E044E150E00E9459C48BE10E9491
:104B70009B12BC01FC0101900020E9F73197E81B72
:104B8000F90B9E012E5F3F4FC901AF010E9450C437
:104B90008BE50E949B12BC01FC0101900020E9F70B
:104BA0003197E81BF90BCE1BDF0B6296CE01AF01EC
:104BB0000E9450C483E090E00E94430681EF9AE196
:104BC0000E94054A0E9457128BE00E949B1290930C
:104BD000331B8093321B0E946F25DF91CF91FF9092
:104BE000EF9008951F930E941A258091651B6EE037
:104BF0000E94CB69192F8091651B6CE00E94CB69E4
:104C00009295917012951170910F9093FB1A8CED03
:104C10009AE160E270E044E150E00E9459C4609182
:104C2000341B7091351BDB01FD0101900020E9F779
:104C30003197EA1BFB0B2EED3AE1C901AF010E944F
:104C400050C48091FB1A8823A1F06091361B7091AB
:104C5000371BDB01FD0101900020E9F73197EA1BCA
:104C6000FB0B2EEE3AE12E1B3F0BC901AF010E9458
:104C700050C483E090E00E94430681EF9AE10E94D5
:104C8000C3491F910895EF92FF92CF93DF9386EF70
:104C90009AE160E070E044E050E00E94592A80917F
:104CA000F61A8F3FB9F48091F71A8F3F99F48091EB
:104CB000F81A8F3F79F48091F91A8F3F59F481E304
:104CC00091E3DC018093F61A9093F71AA093F81AF7
:104CD000B093F91A86EF9AE160E37EE144E050E098
:104CE0000E9443C4009779F00E946D05823021F440
:104CF0008BE00E94DF056EC083E00E947B058BE0A5
:104D00000E94E90567C00E94CC24CCEDDAE1CE0117
:104D100060E270E044E150E00E9459C48AE40E94DD
:104D20009B12BC01FC0101900020E9F73197E81BC0
:104D3000F90B7E01CE01AF010E9450C481E10E94B7
:104D40009B12BC01FC0101900020E9F73197E81BA0
:104D5000F90BC4E1D0E09E012E1B3F0B3695279541
:104D60002E0D3F1DC901AF010E9450C486E10E9473
:104D70009B12BC01FC0101900020E9F73197E81B70
:104D8000F90BCE1BDF0BCE0DDF1DCE01AF010E9454
:104D900050C482E090E00E94430681EF9AE10E94B5
:104DA000054A0E9457128BE00E949B129093331B7E
:104DB0008093321B8BE40E949B129093351B80934F
:104DC000341B8FE40E949B129093371B8093361BF9
:104DD0000E94F225DF91CF91FF90EF900895EF921E
:104DE000FF920F931F93CF93DF9380910C1B882327
:104DF00009F4B5C00E944E09882309F4B0C080911F
:104E00000C1B873040F48530A8F4813008F4A7C02B
:104E1000833068F009C08B3018F48930A8F40FC0D3
:104E20008D3008F09CC015C0C5E4D3E20AC0C3E1D0
:104E3000D3E202C0C7E2D1E280E091E00EC0C2EA54
:104E4000D1E280E890E009C0C8E9D2E280E290E0D7
:104E500004C0CDE1D2E280E490E00E9459098823A9
:104E600009F47FC080910C1B863009F450C0873054
:104E700088F4833009F1843030F48130E9F08230F5
:104E800009F06DC044C0843009F441C0853009F098
:104E900066C012C0893081F08A3030F4873061F00A
:104EA000883009F05CC033C08B3031F08B3078F142
:104EB0008C3009F054C02BC08091A30D9091A40DAB
:104EC000A091A50DB091A60D20910D1B30910E1B48
:104ED00040910F1B5091101B7C018D01E21AF30AC7
:104EE000040B150BA8019701253631054105510525
:104EF000C0F180930D1B90930E1BA0930F1BB093DA
:104F0000101B80910C1B8F5F80930C1B2AC080911B
:104F1000A30D9091A40DA091A50DB091A60D209187
:104F20000D1B30910E1B40910F1B5091101B7C01EB
:104F30008D01E21AF30A040B150BA80197012B301F
:104F400031054105510568F080930D1B90930E1BB0
:104F5000A0930F1BB093101BFE01099502C0109285
:104F60000C1BDF91CF911F910F91FF90EF9008954F
:104F70008091621B882311F48091AF0D8150809342
:104F8000621B81E080936A1B08958091651B8823D2
:104F900011F48BE001C081508093651B81E0809308
:104FA0006A1B08958091621B8F5F9091AF0D8917E6
:104FB00018F01092621B02C08093621B81E0809304
:104FC0006A1B08958091651B8F5F8C3018F01092DA
:104FD000651B02C08093651B81E080936A1B089566
:104FE0001092621B81E080936A1B089581E0809398
:104FF000621B80936A1B089582E08093621B81E0AC
:1050000080936A1B089583E08093621B81E0809304
:105010006A1B089590916B1B992359F08091691B2D
:10502000882321F491509093691B089581508093B7
:10503000691B08958091681B882311F481E001C0E9
:1050400081508093681B08958091691B8F5F9091B8
:105050006B1B891718F01092691B08958093691BC8
:1050600008958091681B8F5F823018F01092681B42
:1050700008958093681B08951092691B089580918C
:105080006B1B882319F081E08093691B0895809140
:10509000641B882311F483E001C081508093641B5A
:1050A00008958091641B8F5F843018F01092641B08
:1050B00008958093641B08958091631B882311F4E5
:1050C00085E001C081508093631B08958091631B2C
:1050D0008F5F863018F01092631B08958093631BD6
:1050E00008951092661B8091B00D8823F1F485E03D
:1050F00090E060E04CE02CE00E94FA2980936C1B69
:1051000091E090936B1B843008F484E08093AF0DA2
:1051100090E001972091621B30E0281739070CF4CA
:10512000C9018093621B1092691B0E9488900E94A3
:10513000275E08951F93182F8230E8F48091621B38
:1051400064E070E00E94ED298091691B66E070E0E8
:105150000E94ED298091B00D882389F080916C1B0D
:1051600065E070E00E94ED2980916B1B67E070E0C4
:105170000E94ED2904C0843011F40E947128812F0F
:105180000E94FC5B812F0E94A7871F91089580E7F2
:1051900098E00E94D3679F708F339105E9F18034C6
:1051A0009105A0F48730910589F18830910538F494
:1051B0008130910549F183309105E1F523C08F30AD
:1051C000910531F18F319105A9F524C021E08F3F80
:1051D000920741F122E08030920738F48F37910531
:1051E000E9F08F3F910531F51BC027E08F3F920713
:1051F000E9F02FE08F3F9207D9F023E08F3F92072D
:10520000C9F412C082E0089581E0089583E0089512
:1052100084E0089585E0089586E0089587E0089584
:1052200088E0089589E008958AE008958BE0089564
:105230008CE0089580E0089585E094E00E94D367B3
:105240008F7090708530910509F09CC08091661B2D
:105250008130D9F0813010F08430B0F18091A30D0D
:105260009091A40DA091A50DB091A60D8093AB0DCA
:105270009093AC0DA093AD0DB093AE0D81E08093F3
:10528000661B82E00E94356408950E94575F8091FA
:10529000A30D9091A40DA091A50DB091A60D209104
:1052A000AB0D3091AC0D4091AD0D5091AE0D821B08
:1052B000930BA40BB50B86399105A105B10508F434
:1052C00063C082E08093661B0E94C72880936C1B9A
:1052D00080E798E00E94D36781E080936B1B809306
:1052E000B00D80916C1B843008F484E08093AF0D86
:1052F00090E001972091621B30E0281739070CF4E9
:10530000C9018093621B1092691B8091661B8330D8
:1053100050F58091A30D9091A40DA091A50DB09191
:10532000A60D2091AB0D3091AC0D4091AD0D50917B
:10533000AE0D821B930BA40BB50B843F21E09207AB
:1053400020E0A20720E0B20770F083E08093661BA4
:105350000E94DE4A81E090E00E941BA30E94544E0E
:1053600083E00E9435640E94575F0E94734B0E9445
:10537000B0B20E948B5C0E94E7880E9478500E9425
:10538000969008950E947128089584E090E060E06E
:105390004BE020E00E94FA298093621B91E09093F9
:1053A0006A1B8093651B86E090E060E041E020E0AE
:1053B0000E94FA298093691B8093681B0E947128C0
:1053C0000E94DE4A81E090E00E941BA30E94544E9E
:1053D0000E94655C0E94E78808951F93282FCB01E7
:1053E0001FB7F894622F0E94A4C517FF01C07894DC
:1053F0001F9108951F93DF93CF9300D00F92CDB7E5
:10540000DEB71FB7F8942B834A8369830E9492C545
:105410002B814A81698117FF01C07894861718F0A3
:10542000481708F0282F822F0F900F900F90CF91E0
:10543000DF911F9108951F931FB7F8940E949AC59A
:1054400017FF01C078941F910895DF93CF9300D088
:1054500000D0CDB7DEB769837A838B839C83BA0192
:10546000CE01019644E050E00E941B2A0F900F905D
:105470000F900F90CF91DF910895DF93CF9300D0DD
:10548000CDB7DEB79A838983CE01019642E050E022
:105490000E941B2A0F900F90CF91DF91089544E056
:1054A00050E00E941B2A089544E050E00E941B2A0D
:1054B00008951F931FB7F8940E9482C517FF01C07B
:1054C00078941F9108954F925F926F927F928F927E
:1054D0009F92AF92BF92CF92DF92EF92FF920F9383
:1054E0001F93DF93CF9300D000D0CDB7DEB7FC0180
:1054F0002A013B0148015901CE010196BF0144E058
:1055000050E00E94592A89819A81AB81BC8184151F
:105510009505A605B70538F088169906AA06BB06B4
:1055200010F06C017D01B601C7010F900F900F9034
:105530000F90CF91DF911F910F91FF90EF90DF902F
:10554000CF90BF90AF909F908F907F906F905F9023
:105550004F900895EF92FF920F931F93DF93CF9395
:1055600000D000D0CDB7DEB7FC017B018A01CE01AF
:105570000196BF0142E050E02B833C830E94592AF0
:1055800089819A812B813C818E159F0520F0081717
:10559000190708F09C01C9010F900F900F900F9010
:1055A000CF91DF911F910F91FF90EF9008950F938E
:1055B0001F93DF93CF9300D000D0CDB7DEB7BC01EF
:1055C0008E010F5F1F4FC80144E050E00E94592A2E
:1055D00089818F3F91F4F8013196D80111968C9111
:1055E00011978F3F51F4DF01119681818F3F29F48C
:1055F00011968C9111978F3F51F089819A81AB81DF
:10560000BC812A2F220F2B2F221F2F3F19F480E05D
:1056100090E0DC01682F792F8A2F9B2F0F900F903D
:105620000F900F90CF91DF911F910F9108952F92BE
:105630003F924F925F926F927F928F929F92AF9222
:10564000BF92CF92DF92EF92FF920F931F93DF935F
:10565000CF9300D000D0CDB7DEB7FC011A012B01EB
:1056600038014901560167017E010894E11CF11CD3
:10567000C701BF0144E050E00E94592A89818F3F51
:1056800091F4F7013196D70111968C9111978F3FC4
:1056900051F4DF01119681818F3F29F411968C918D
:1056A00011978F3FE1F0E980FA800B811C81802FF8
:1056B000880F812F881F8F3F91F0C801B701A20189
:1056C00091010E9486C087FD0AC0C801B701A401EC
:1056D00093010E94D5C1181614F0570168016A2D74
:1056E0007B2D8C2D9D2D0F900F900F900F90CF91B3
:1056F000DF911F910F91FF90EF90DF90CF90BF90BF
:10570000AF909F908F907F906F905F904F903F9061
:105710002F900895DC01EC91F0E02FEF3FEF22C0D5
:10572000432F50E0322F2227422B532B4E275F2747
:10573000242F22952F7030E024273527A901542FDC
:1057400044275295507F422753279A01307075E0C5
:10575000220F331F7A95E1F724273527DC01EC91DE
:10576000F0E0615001966623D9F62093C80D30937E
:10577000C90DC9010895AF92BF92CF92DF92EF9207
:10578000FF920F931F93DF93CF93CDB7DEB72A9786
:105790000FB6F894DEBF0FBECDBF8C015B01DC01FC
:1057A0008C91843309F404C2853308F58B3009F4F5
:1057B0007EC08C3070F4843009F44BC0853018F40E
:1057C0008823D1F136C0853009F450C0863089F580
:1057D00050C0813309F44CC1823318F4803349F549
:1057E00016C1823309F46EC1833319F592C1813435
:1057F00009F49DC3823460F4863309F4D9C1863339
:1058000008F439C2873309F436C2803491F4DAC21D
:10581000803609F457C0813630F4803509F4F3C37B
:10582000813539F4B3C5813609F480C0803D09F46F
:10583000E1C5EE24FF2429C6FB0110828FEF81838E
:1058400080E081938F5F8733E1F767E3E62EF12CE9
:105850001CC6DB01F80187E001900D928150E1F751
:1058600085EAD50117968C9317970CC6FB018083A8
:1058700009C6DB018C9382E011968C93119789E223
:1058800012968C93129780E213968C93139782E171
:1058900014968C93149780E115968C93159784E158
:1058A00016968C93169717961C921797EBC5F801CE
:1058B0006181D5018C9311966C9385E040E00E9444
:1058C0001C64E0C585E094E00E94D367BC0160627F
:1058D00085E094E00E94A46BF8012181628170E070
:1058E00080E090E0CB0177276627C380DD24EE249B
:1058F000FF24FE2CED2CDC2CCC246C297D298E2958
:105900009F29C480DD24EE24FF246C297D298E2963
:105910009F296093B20D7093B30D8093B40D909353
:10592000B50DA8014B5F5F4F0E94FB9685E094E0A8
:105930000E94D367BC01606285E094E00E94A46B82
:10594000D80111962C911197E22EFF24E5E0F0E0AA
:10595000EE0EFF1E12968C9190E0A0E0B0E0DC010C
:1059600099278827F801438150E060E070E0762FA6
:10597000652F542F4427842B952BA62BB72B4481BE
:1059800050E060E070E0842B952BA62BB72B809322
:10599000B20D9093B30DA093B40DB093B50DD50196
:1059A00085E001900D928150E1F76091B20D709108
:1059B000B30D8091B40D9091B50DA5014B5F5F4F74
:1059C000222311F548875A870E9453960E940D960C
:1059D000082F6091B20D7091B30D8091B40D90912C
:1059E000B50D48855A8524E60E947896D50116960D
:1059F0000C93169717960C93179718960C93189765
:105A000019960C93199741C50E9478963EC5F801E6
:105A1000E180328120E0838190E0822B932B909370
:105A2000B70D8093B60DB8016C5F7F4F4E2D0E946D
:105A30006A518091B60D9091B70D97FD19C08E0DEA
:105A4000911DF0E681309F0798F081E08093F21D70
:105A50008091A30D9091A40DA091A50DB091A60DDC
:105A60008093641C9093651CA093661CB093671C84
:105A7000D80111964C911197E42EFF24E5E0F0E057
:105A8000EE0EFF1E12963C91129720E013968C9119
:105A9000139790E0822B932B9093B70D8093B60DC4
:105AA0008D919D910D90BC91A02DF50181939193C5
:105AB000A193B193BF018091B60D9091B70D0E9453
:105AC000F750E3C4D80111966C9111976031B0F092
:105AD0006C3109F0D0C412968C9112978C31C9F4B4
:105AE00013968C9113978330A1F4C801029661EF4D
:105AF00072E04EE150E00E941B2A0BC070E0660F7E
:105B0000771F660F771F62567D4FC80102960E946D
:105B1000542AF8018081D5018C93818111968C9350
:105B200011978181803120F18C3109F0A4C48EEB72
:105B30009AE161EF72E04EE150E00E94592A8FE253
:105B40009CE161EF72E04EE150E00E94592AD501DC
:105B50001296EFE2FCE18CE101900D928150E1F7A9
:105B6000F501E180FF2484E090E0E80EF91E8DC489
:105B700090E0880F991F880F991FFC01E357FB4F96
:105B8000C080D180E280F38082569D4F40E050E09B
:105B900068E472EC00E010E028E432E40E94172B85
:105BA000D50112966D937D938D939C9315976AC43E
:105BB000F8016181862F829586958695837090E0A5
:105BC000823091050CF057C43081262F26952695FA
:105BD0002695343329F5277030E0243031050CF058
:105BE0004AC4677070E0633071050CF044C4660FFE
:105BF000771F660F771FE6EAF0E08E9FA0018F9F68
:105C0000500D9E9F500D1124640F751F6A5A7E4FD0
:105C100054E0220F331F5A95E1F7620F731F27C01C
:105C2000277030E0263031050CF025C4677070E035
:105C3000643071050CF01FC4660F771F660F771F65
:105C4000E6EAF0E08E9FA0018F9F500D9E9F500DC1
:105C50001124640F751F6D567E4FC901B4E0880F83
:105C6000991FBA95E1F7820F931F680F791FC8013A
:105C700002960E94542AD8018C91F50180831196D6
:105C80008C911197818311969C911197692F629540
:105C900066956695637070E0623071050CF0EBC339
:105CA0008C918453492F469546954695823008F04D
:105CB00043C0477050E0443051050CF0DCC397708E
:105CC000E92FF0E0E330F1050CF0D5C39F01220F7E
:105CD000331F220F331FA6EAB0E06A9FC0016B9FFB
:105CE000900D7A9F900D1124280F391F2A5A3E4F8C
:105CF000CA0144E0880F991F4A95E1F7EE0FFF1F94
:105D0000EE0FFF1FE353FB4FC080D180E280F38092
:105D1000820F931F40E050E068E472EC00E010E076
:105D200028E432E40E94172BD50112966D937D93DF
:105D30008D939C93159742C0477050E046305105B3
:105D40000CF099C39770E92FF0E0E430F1050CF006
:105D500092C3CF01880F991F880F991FA6EAB0E060
:105D60006A9F90016B9F300D7A9F300D1124820F36
:105D7000931F8D569E4F9A01B4E0220F331FBA95A0
:105D8000E1F7240F351FEE0FFF1FEE0FFF1FE75245
:105D9000FB4FC080D180E280F380820F931F40E0F0
:105DA00050E068E472EC00E010E028E432E40E9485
:105DB000172BF5016283738384839583E6E0EE2ECF
:105DC000F12C63C3D8011196EC901197E6941296CA
:105DD0003C91129720E013968C91139790E0822BC0
:105DE000932B9093B70D8093B60DB4E082309B0750
:105DF00050F48E0D911DE4E081309E0720F084E583
:105E00009BE10E947E1DB8016C5F7F4F8091B60DB3
:105E10009091B70D4E2D50E00E94156B8093C80DE8
:105E20009093C90D2091B60D3091B70DF4E020305C
:105E30003F07A0F521E02093B10D8093B80D90931A
:105E4000B90DF8017EEBC72E7DE0D72E8281D601F9
:105E50008D936D013196B8ECCB16BDE0DB06B1F742
:105E6000C6010A9764E00E948A2B8093C80D909324
:105E7000C90D2091B60D2093BA0D2091B70D209336
:105E8000BB0D8093BC0D9093BD0D86E294E0B601EE
:105E9000605170404CE050E00E94156B8091B60D4F
:105EA0009091B70DE4E082309E0708F040C08E0D5F
:105EB000911DF4E081309F07D0F181E08093F21DC5
:105EC0008091A30D9091A40DA091A50DB091A60D68
:105ED0008093641C9093651CA093661CB093671C10
:105EE0008BE59BE10E947E1D9091581B80915F1B6A
:105EF0009817B9F49091571B80915E1B981789F4FD
:105F00009091561B80915D1B981759F42091541B5A
:105F10003091551B80915B1B90915C1B28173907B2
:105F200019F084E08093111181E080939D1BD801CA
:105F300011964C911197469512963C91129720E03C
:105F400013968C91139790E0822B932B9093B70D1F
:105F50008093B60D8D919D910D90BC91A02DF50172
:105F600080839183A283B383842F880F8183B501BB
:105F70006C5F7F4F8091B60D9091B70D50E00E94FD
:105F8000B1678093C80D9093C90DD5011196EC901F
:105F900011972091B10D213071F58093B80D909338
:105FA000B90DF5010EEB1DE08281D8018D938D01B5
:105FB0003196BDE0083C1B07B9F7C8010A9764E0B9
:105FC0000E948A2B8093C80D9093C90D2091B60D25
:105FD0002093BA0D2091B70D2093BB0D8093BC0D7B
:105FE0009093BD0D82E394E0B801605170404CE0A5
:105FF00050E00E94156BFF24E4E0F0E0EE0EFF1E7F
:106000001092B10D42C285EA95EADB018D939C9313
:10601000F80180819181A281B381FB01808391830A
:10602000A283B383D80111968C911197853A09F414
:1060300094C0863A30F4882351F08E3109F022C2A0
:1060400031C08A3C69F08E3F09F01CC21AC0F801C9
:10605000828193810E94430964E0E62EF12C15C2EF
:10606000D80112968C91129713966C910E94D4725B
:10607000482F4E7FF801828163810E949D728FE4D8
:106080006DC0D80112968C91129713966C910E9454
:10609000D472482F4160F801828163810E949D7211
:1060A00083E45CC0D80112968C91129756EA859FC2
:1060B000C001112413966C9131E1639FB00111244A
:1060C000860F971F8E569E4F60E04BE022E0398787
:1060D0005A870E94FA29982FF80182816381988754
:1060E0000E94D472E82ED80112966C9112971396E2
:1060F0008C91139739855A859885E1FE14C0659F68
:10610000B0011124839F90011124620F731F6E56FA
:106110007E4F892F8D700E94ED294E2D4D70F80114
:106120008281638116C0659FB0011124839F900115
:106130001124620F731F6E567E4F892F82600E945A
:10614000ED294E2D4260D80112968C91129713962C
:106150006C910E949D7284E501C08EE4F8019181EA
:10616000D50111969C9311979FE516969C931697CF
:1061700022812F5C17962C93179718969C9318974B
:1061800023812F5C19962C9319971A969C931A9732
:106190001B968C931B975FE2E52E1C96EC924DE0CC
:1061A000C42ED12CCA0CDB1CCE0101960E947E1D90
:1061B000EDB7FEB770970FB6F894FEBF0FBEEDBFF8
:1061C0003196ADB7BEB71296DC92CE92119789EE9A
:1061D00094E09383828389819A81958384838B81E0
:1061E00090E00196978386838C81808711868D81CC
:1061F000828713868E81848715868F81868717868E
:106200000E94F4C4F501E1A232E2C32ED12CCA0CE3
:10621000DB1C8DB79EB740960FB6F8949EBF0FBE9D
:106220008DBFC8010296D80112966C9112971396F1
:106230004C910E94AF7BEDB7FEB73A970FB6F8943A
:10624000FEBF0FBEEDBF2DB73EB72F5F3F4FD282CF
:10625000C18288E090E0D90113969C938E931297A7
:1062600088E095E015969C938E931497F8018285AB
:106270009385A485B585F90186839783A087B18727
:106280000E94B6C4D5019996EC92C5018A962DB7A5
:106290003EB72F5F3F4FEDB7FEB79283818387E014
:1062A00090E0D90113969C938E9312978EE095E01F
:1062B00015969C938E931497F80182819381A48103
:1062C000B581F90186839783A087B1870E94B6C400
:1062D000D501D096EC92EDB7FEB73A960FB6F8948A
:1062E000FEBF0FBEEDBFD80195968C919597950195
:1062F0002E5C3F4F882321F081E3F50181AB04C080
:1063000080E3D501D1968C93D9018FE28D93F8016A
:1063100084A1AD014F5F5F4F882331F081E3D90144
:1063200011968C93119703C080E3F9018183FA01E0
:106330008FE28193D80196968C9196977F0108946D
:10634000E11CF11C8A3050F081E3DA0111968C9344
:10635000D80196968C9196978A5D09C080E3DA0100
:1063600011968C93D80196968C919697805D818337
:10637000F70131968FE2808326E0E22EF12CEE0EBB
:10638000FF1EEA18FB08F501E5827FC0DB018C9354
:1063900011961C9211978091311B882321F092E075
:1063A000E92EF12C72C0F80111811F70DB011196EA
:1063B0001C931197EE24FF2400E015C010FF0BC0C2
:1063C000602F70E06E5F7F4F6A0D7B1DC70144E157
:1063D0000E9417060C5E0894E11CF11CB4E0EB1659
:1063E000F10419F01695112349F7E02EFF24E2E09D
:1063F000F0E03EC0D80112963C91129720E013962F
:10640000EC901397FF24E22AF32AF092B70DE09262
:10641000B60D11960C9111970695FB018083802F84
:10642000880F8183F282E38284E0C82ED12CC60ECD
:10643000D71E15C0102F093008F018E0C701B601AB
:10644000412F50E00E94B167011B812F90E0880F1F
:10645000991FC80ED91E80E190E0E80EF91E0023B6
:1064600049F7D5011196EC901197FF24E4E0F0E094
:10647000EE0EFF1E0AC087E0D5018C9384E01196D2
:106480008C931197B8E0EB2EF12CC7012A960FB62A
:10649000F894DEBF0FBECDBFCF91DF911F910F915A
:1064A000FF90EF90DF90CF90BF90AF9008950E9443
:1064B000EF2680E060E00E949F04E091091BF0E07D
:1064C000EE0FFF1FEF5EF44E808191810E94550612
:1064D00083E061E00E949F04E0910A1BF0E0EE0F70
:1064E000FF1FEE5CF44E808191810E945506089555
:1064F0000E9457328BE061E00E949F04E091091BEB
:10650000F0E0EE0FFF1FEF50F54E8581968164E1BC
:1065100075E046E00E94580681E161E00E949F0418
:1065200081E40E94B2040895CF93DF9310920C1B74
:10653000CCEDDAE1CE0160E270E044E150E00E948F
:1065400059C48EE50E949B12BC01FC010190002001
:10655000E9F73197E81BF90B2AE030E02E1B3F0BDF
:1065600036952795265F3F4F2C0F3D1FC901AF0180
:106570000E9450C480E090E00E944306CE0160E299
:1065800070E044E150E00E9459C481E090E00E9434
:106590004306DF91CF9108950E94222489E50E944D
:1065A0009B129093331B8093321B83E30E949B12B8
:1065B0009093351B8093341B85E30E949B1290932C
:1065C000371B8093361B84E30E949B129093391BE8
:1065D0008093381B86E30E949B1290933B1B809311
:1065E0003A1B89E80E949B1290933D1B80933C1BB1
:1065F0008AE80E949B1290933F1B80933E1B8BE87E
:106600000E949B129093411B8093401B8DE80E9437
:106610009B129093431B8093421B8CE80E949B1219
:106620009093451B8093441B0895EF92FF92CF9364
:10663000DF930E9494328AE20E949B12BC01FC010B
:1066400001900020E9F73197E81BF90BCCEDDAE176
:10665000CE01AF010E9450C482E090E00E94430648
:10666000CE0160E270E044E150E00E9459C48BE248
:106670000E949B12BC01FC0101900020E9F73197B8
:10668000E81BF90B2296CE01AF010E9450C483E0B3
:1066900090E00E9443060E9457120E94CC32DF9184
:1066A000CF91FF90EF900895EF92FF92CF93DF93F9
:1066B0000E9494328EE20E949B12BC01FC01019068
:1066C0000020E9F73197E81BF90BCCEDDAE1CE01B8
:1066D000AF010E9450C480E30E949B12BC01FC01E8
:1066E00001900020E9F73197E81BF90B9E012E1B62
:1066F0003F0B2C5E3F4FC901AF010E9450C482E0A6
:1067000090E00E944306CE0160E270E044E150E078
:106710000E9459C48FE20E949B12BC01FC010190AF
:106720000020E9F73197E81BF90B9E012E5F3F4FE0
:10673000C901AF010E9450C481E30E949B12BC01B9
:10674000FC0101900020E9F73197E81BF90BCE1B03
:10675000DF0B6296CE01AF010E9450C483E090E04F
:106760000E9443060E9457120E94CC32DF91CF91C3
:10677000FF90EF90089580E10E94E90508951F932E
:1067800080910B1B882309F49CC080910A1B8230E6
:1067900051F1833020F4813009F093C007C0833079
:1067A00009F44AC0843009F08CC063C04091F61AE5
:1067B0005091F71A6091F81A7091F91A8091651B3F
:1067C00090E020E00E94736D4091FA1A5091FB1AFC
:1067D0006091FC1A7091FD1A8091651B90E020E099
:1067E0000E94596D6EC01091651B2091F61A309170
:1067F000F71AB901882777FD8095982F0E9425C147
:10680000AB01BC01812F90E020E00E94F86C109158
:10681000651B2091F81A3091F91AB901882777FD84
:106820008095982F0E9425C1AB01BC01812F90E07B
:1068300020E00E94C96C45C04091F61A5091F71AA9
:106840006091F81A7091F91A8091651B90E020E030
:106850000E943F6D4091FA1A5091FB1A6091FC1A08
:106860007091FD1A8091651B90E020E00E94256DDB
:1068700028C01091651B2091F61A3091F71AB901C2
:10688000882777FD8095982F0E9425C1AB01BC0118
:10689000812F90E020E00E949C6C1091651B20915C
:1068A000F81A3091F91AB901882777FD8095982F49
:1068B0000E9425C1AB01BC01812F90E020E00E9425
:1068C0006D6C1F91089580910A1B823009F183300D
:1068D00020F4813009F099C006C08330F1F1843092
:1068E00009F093C06EC08091651B90E060E00E944B
:1068F0007D6A6093F61A7093F71A8093F81A909352
:10690000F91A8091651B90E060E00E94716A39C0BD
:106910008091651B90E060E00E94426A0E94F2C094
:106920007093F71A6093F61A8091651B90E060E00F
:106930000E942B6A0E94F2C07093F91A6093F81AB1
:1069400084ED9EEF9093FB1A8093FA1A8CE291E00B
:106950009093FD1A8093FC1A08958091651B90E036
:1069600060E00E94656A6093F61A7093F71A80934C
:10697000F81A9093F91A8091651B90E060E00E94EC
:10698000596A6093FA1A7093FB1A8093FC1A9093D9
:10699000FD1A80E090E0DC018093FE1A9093FF1ACC
:1069A000A093001BB093011B80E090E0A6E9B2E445
:1069B0008093021B9093031BA093041BB093051BB1
:1069C00008958091651B90E060E00E94146A0E9427
:1069D000F2C07093F71A6093F61A8091651B90E0ED
:1069E00060E00E94FD690E94F2C07093F91A609302
:1069F000F81A84ED9EEF9093FB1A8093FA1A8CE2BA
:106A000091E09093FD1A8093FC1A0895CF93DF9341
:106A10000E94BF3380910A1B833049F0843069F0B3
:106A2000823019F0CFE0D0E00DC081E007C082E0F5
:106A300080930A1BC1E1D0E005C083E080930A1B6C
:106A4000C0E1D0E00E94633410920B1B1092091B2E
:106A50008C2F0E94E905DF91CF910895CF93DF93AA
:106A60000E94BF3380910A1B833061F0843081F033
:106A7000823011F082E007C083E080930A1BC0E1FE
:106A8000D0E00AC084E080930A1BC1E1D0E004C0DA
:106A900010920A1BC3E0D0E00E94633410920B1BDB
:106AA0001092091B8C2F0E94E905DF91CF91089568
:106AB0000E9457328BE061E00E949F04E091091B25
:106AC000F0E0EE0FFF1FEE0FFF1FEF50F54E658158
:106AD00076818781908548E155E027E00E949D06F8
:106AE00082E161E00E949F0486E50E94B20408955D
:106AF000413051F4662311F46EE001C06CE040E0D7
:106B000050E120E030E009C0662311F46EE001C0DE
:106B10006CE040E050E020E030E10E94F26B08952C
:106B2000E091081BF0E0EF50F54E158A6091651B6F
:106B30008BE1689FB00111249091081B8DE0989F14
:106B4000C0011124680F791F615F7F4F80E00E94B0
:106B5000ED298091651B6091081B40E00E9478350B
:106B60000895E091081BF0E0EF50F54E84E0858B2E
:106B70006091651B8BE1689FB00111249091081B07
:106B80008DE0989FC0011124680F791F615F7F4FCE
:106B900084E00E94ED298091651B6091081B44E010
:106BA0000E9478350895E091081BF0E0EF50F54E13
:106BB00083E0858B6091651B8BE1689FB001112498
:106BC0009091081B8DE0989FC0011124680F791FD8
:106BD000615F7F4F83E00E94ED298091651B60918A
:106BE000081B43E00E9478350895E091081BF0E00F
:106BF000EF50F54E82E0858B6091651B8BE1689FBD
:106C0000B00111249091081B8DE0989FC0011124C0
:106C1000680F791F615F7F4F82E00E94ED298091AC
:106C2000651B6091081B42E00E9478350895E09151
:106C3000081BF0E0EF50F54E81E0858B6091651BFD
:106C40008BE1689FB00111249091081B8DE0989F03
:106C5000C0011124680F791F615F7F4F81E00E949E
:106C6000ED298091651B6091081B41E00E947835F9
:106C70000895CF93DF938091081B882329F0C0915A
:106C8000381BD091391B04C0C091341BD091351BE7
:106C90008FE060E00E949F04CE010E94E304E09137
:106CA000081BF0E0EF50F54EE589F0E0EE0FFF1F16
:106CB000E45CF44EC081D1818DE061E00E949F04CC
:106CC000CE010E94550681EF9AE10E94C349DF91EF
:106CD000CF910895FF920F931F93082FF62E6623EE
:106CE00011F06CE001C06EE00E94CB69192F129583
:106CF00011702BE1029F90011124215F3F4F8DE025
:106D00004F2D489FC0011124820F931F60E044E083
:106D100020E00E94FA29813011F4812F02C0111164
:106D200081E01F910F91FF900895EF92FF920F93D2
:106D30001F93CF93DF938091651B60E00E946A36BA
:106D40008093061B8091651B61E00E946A368093E8
:106D5000071B1092081B81E080930A1B10920B1BEB
:106D60001092091B0E946334CCEDDAE1CE0160E29F
:106D700070E044E150E00E9459C489E00E949B12F7
:106D8000BC01FC0101900020E9F73197E81BF90BE9
:106D900004E110E098012E1B3F0B369527952C0F30
:106DA0003D1FC901AF010E9450C480E090E00E94E5
:106DB0004306CE0160E270E044E150E00E9459C415
:106DC00081E090E00E9443068EE40E949B12BC0189
:106DD000FC0101900020E9F73197E81BF90BCE0187
:106DE000AF010E9450C489E50E949B12BC01FC01C6
:106DF00001900020E9F73197E81BF90B98012E1B51
:106E00003F0B369527952C0F3D1FC901AF010E94FE
:106E100050C483E50E949B12BC01FC01019000203C
:106E2000E9F73197E81BF90B0E1B1F0B0C0F1D1F09
:106E3000C801AF010E9450C482E090E00E94430666
:106E4000CE0160E270E044E150E00E9459C481E567
:106E50000E949B12BC01FC0101900020E9F73197D0
:106E6000E81BF90B9E012E5F3F4FC901AF010E9445
:106E700050C485E50E949B12BC01FC0101900020DA
:106E8000E9F73197E81BF90BCE1BDF0B6296CE01B9
:106E9000AF010E9450C483E090E00E9443060E942C
:106EA00057120E94CC3281EF9AE10E94054ADF918D
:106EB000CF911F910F91FF90EF9008959091F11A4B
:106EC000892F882311F48BE001C08150E82FF0E076
:106ED000EB5AF34E2081222331F08093F11A81E0A6
:106EE0008093F21A0895891761F708959091F11A25
:106EF000892F8F5F8C3008F080E0E82FF0E0EB5AAC
:106F0000F34E2081222331F08093F11A81E08093A7
:106F1000F21A0895891769F70895AF92BF92CF9238
:106F2000DF92EF92FF920F931F93DF93CF93CDB732
:106F3000DEB72A970FB6F894DEBF0FBECDBF8091A3
:106F4000631C8823F1F48091A30D9091A40DA0916E
:106F5000A50DB091A60D2091F31A3091F41A40912D
:106F6000F51A5091F61A821B930BA40BB50B893CB2
:106F70009105A105B10510F00E94C2051092F21A08
:106F8000DEC08091F21A882309F4D9C08CED9AE111
:106F900060E270E044E150E00E9459C400E010E07B
:106FA00020E030E05E010894A11CB11C48E0C42E32
:106FB000D12C96E6E92E95E0F92EF801EB5AF34E26
:106FC0008081882399F18DB79EB708970FB6F89402
:106FD0009EBF0FBE8DBFEDB7FEB73196ADB7BEB742
:106FE0001296BC92AE921197D382C282F582E4824D
:106FF000C80101969783868329873A870E94B6C481
:1070000029853A85F901E452F54E89819A81918367
:1070100080832D5F3F4F8DB79EB708960FB6F894CB
:107020009EBF0FBE8DBF233131052CF40F5F1F4F64
:107030000C30110511F681E090E00E944306E091CA
:10704000F11AF0E0EB5AF34E8081882311F40E948C
:1070500076370CED1AE1C80160E270E044E150E0DF
:107060000E9459C4E091F11AF0E0EB5AF34E80818E
:1070700090E00E948290E82FF0E0EE0FFF1FE950B1
:10708000F54E60817181DB01FD0101900020E9F77F
:107090003197EA1BFB0BC801AF010E9450C4ADB78A
:1070A000BEB718970FB6F894BEBF0FBEADBFEDB711
:1070B000FEB731968E010F5F1F4F12961C930E93F1
:1070C000119788E090E0938382838AE695E0958328
:1070D00084838091F11A90E00196978386830E94C1
:1070E000B6C4F80101900020E9F73197E01BF10BDD
:1070F00020EF3AE12E1B3F0B8DB79EB708960FB6D7
:10710000F8949EBF0FBE8DBFC901B801AF010E94A8
:1071100050C483E090E00E9443061092F21A8091DE
:10712000A30D9091A40DA091A50DB091A60D8093F3
:10713000F31A9093F41AA093F51AB093F61A2A96BC
:107140000FB6F894DEBF0FBECDBFCF91DF911F9178
:107150000F91FF90EF90DF90CF90BF90AF90089588
:10716000EF92FF92CF93DF938BE08093F11A0E940E
:10717000763781E08093F21A8091A30D9091A40D4F
:10718000A091A50DB091A60D8093F31A9093F41AD7
:10719000A093F51AB093F61ACCEDDAE1CE0160E2D5
:1071A00070E044E150E00E9459C484E10E949B12C7
:1071B000BC01FC0101900020E9F73197E81BF90BB5
:1071C000CE01AF010E9450C480E090E00E944306CF
:1071D000CE0160E270E044E150E00E9459C481E0D9
:1071E00090E00E94430682E090E00E94430683E024
:1071F00090E00E9443060E9457128AE90E949B1267
:107200009093F81A8093F71A89E90E949B12909341
:10721000FA1A8093F91A88E90E949B129093FC1A3B
:107220008093FB1ADF91CF91FF90EF9008958091AA
:10723000621C882359F00E946505883221F481E0A0
:107240008093F21A089588E20E94E9050895EF926A
:10725000FF920F931F93DF93CF930F92CDB7DEB7BB
:107260008091A30D9091A40DA091A50DB091A60DB4
:107270002091CB0D3091CC0D4091CD0D5091CE0D84
:107280007C018D01E21AF30A040B150BA80197018A
:10729000253131054105510508F4B1C08093CB0D6E
:1072A0009093CC0DA093CD0DB093CE0D8091CA0DCF
:1072B000823009F45FC0833009F48CC0BE016F5F77
:1072C0007F4F813039F1198284EB9BE30E94BA5FD2
:1072D000198183E094E00E94D367BC016F737F73D0
:1072E000123071F0133018F4113071F40CC01330F7
:1072F00029F0143049F46068706806C0606804C002
:107300006068706401C0706483E094E00E94A46BC4
:1073100081E05DC019828AEC9AE30E94BA5F19810C
:1073200083E094E00E94D367BC01637F737F1430D5
:1073300091F0153038F4123061F0133050F4113000
:1073400099F409C0163061F0163038F0173061F446
:107350000AC06C6009C0646007C06460746004C0E7
:107360006C607C6001C07C6083E094E00E94A46B50
:1073700082E02DC0198280E19AE3BE016F5F7F4FEA
:107380000E94BA5F198183E094E00E94D367BC0138
:107390006F7C7F7C133081F0143028F4113051F071
:1073A000123081F405C0143051F0153059F409C081
:1073B000606108C0606306C06061706103C0706195
:1073C00001C0706383E094E00E94A46B83E080932B
:1073D000CA0D15C083E094E00E94D367BC016C7FA6
:1073E0007C7F8091631C882319F48091611C81113A
:1073F000716083E094E00E94A46B1092CA0D0F901C
:10740000CF91DF911F910F91FF90EF90089583E04E
:1074100094E060E070E00E94A46B1092CA0D0895A1
:10742000CF92DF92EF92FF920F931F93CF93DF9350
:10743000182F662319F421E030E0A2C0E42EE70102
:107440007E01F52EE701812F6EE00E94CB6994FF4B
:1074500043C0812F62E00E94CB6996FF02C001E029
:107460003CC0812F6EE00E94CB696C01812F63E0EC
:107470000E94CB69D4FE04C095FD02C002E02DC07D
:107480008091661B833041F5812F60E00E949958FE
:107490006B017C0120E030E040E450E40E9486C0B3
:1074A000882314F405E019C0C701B60120E030E0DC
:1074B00040EF50E40E9486C0882314F404E00DC01D
:1074C000C701B60120E030E040E751E40E9486C0E9
:1074D000882314F403E001C000E0812F6CE00E94D7
:1074E000CB6994FF43C0812F62E00E94CB6996FF75
:1074F00002C081E03CC0812F6EE00E94CB696C012C
:10750000812F63E00E94CB69D4FE04C095FD02C0C8
:1075100082E02DC08091661B833041F5812F60E0B1
:107520000E9499586B017C0120E030E040E450E477
:107530000E9486C0882314F485E019C0C701B601F3
:1075400020E030E040EF50E40E9486C0882314F42D
:1075500084E00DC0C701B60120E030E040E751E40F
:107560000E9486C0882314F483E001C080E0801765
:1075700008F4802F9881981708F4888320E030E081
:10758000C901DF91CF911F910F91FF90EF90DF9094
:10759000CF9008952F923F924F925F926F927F9279
:1075A0008F929F92AF92BF92CF92DF92EF92FF9213
:1075B0000F931F93DF93CF9300D000D0CDB7DEB7EA
:1075C000182F662319F421E030E0B6C01A0190E0CC
:1075D0000E94B86A4B015C01812F90E00E94046B0D
:1075E0006B017C01812F90E00E94B26A2B013C016B
:1075F000812F90E00E94FE6A69837A838B839C834B
:10760000C501B401A70196010E94D9C16B017C019B
:10761000C301B20129813A814B815C810E94D9C1A9
:107620009B01AC01C701B6010E9422C0D62EE72EF5
:10763000F82E092F20E030E04AEF53EC0E9486C07C
:10764000181614F003E070C06D2D7E2D8F2D902F35
:1076500020E030E048EC52EC0E9486C0181614F08E
:1076600004E062C06D2D7E2D8F2D902F20E030E83C
:107670004BEB54E40E94D5C1181614F407E054C033
:107680006D2D7E2D8F2D902F20E030E04AEF53E4BA
:107690000E94D5C1181614F406E046C06D2D7E2D4B
:1076A0008F2D902F20E030E048EC52E40E94D5C1AD
:1076B000181614F405E038C0812F62E00E94CB69EF
:1076C00095FD02C000E014C0812F90E00E94046B81
:1076D0006B017C01812F90E061E00E94426A9B0176
:1076E000AC01C701B6010E9486C087FD1CC001E045
:1076F000812F65E00E94CB6995FF16C0812F90E035
:107700000E94FE6A6B017C01812F90E061E00E9483
:10771000146A9B01AC01C701B6010E9486C087FDB7
:1077200002C001E001C002E0F1018081801710F485
:10773000F101008320E030E0C9010F900F900F901D
:107740000F90CF91DF911F910F91FF90EF90DF90FD
:10775000CF90BF90AF909F908F907F906F905F90F1
:107760004F903F902F900895EF92FF921F93CF93E9
:10777000DF93182F662319F421E030E032C0E42EA5
:10778000E7017E01F52EE701812F6BE00E94BA69C7
:1077900093FF02C084E01FC0812F6BE00E94BA6992
:1077A00092FF10C0812F6AE00E94BA6995FF12C053
:1077B000812F6BE00E94BA6994FD02C082E00BC089
:1077C00083E009C0812F6AE00E94BA6995FF02C078
:1077D00081E001C080E09881981708F4888320E058
:1077E00030E0C901DF91CF911F91FF90EF90089594
:1077F00083E10E94E905089580910B1B8823E1F144
:1078000080910A1B813019F08230B1F51BC0409184
:10781000F61A5091F71A6091F81A7091F91A80913E
:10782000651B90E00E94546C4091FA1A5091FB1A2B
:107830006091FC1A7091FD1A8091651B90E00E9486
:10784000396C08954091F61A5091F71A6091F81A20
:107850007091F91A8091651B90E00E94236C409111
:10786000FA1A5091FB1A6091FC1A7091FD1A8091DE
:10787000651B90E00E94086C089580910A1B81307E
:1078800019F08230B1F51BC08091651B90E00E9419
:10789000F5696093F61A7093F71A8093F81A90932B
:1078A000F91A8091651B90E00E94EC696093FA1AC6
:1078B0007093FB1A8093FC1A9093FD1A089580919F
:1078C000651B90E00E94E1696093F61A7093F71AC5
:1078D0008093F81A9093F91A8091651B90E00E94AA
:1078E000D2696093FA1A7093FB1A8093FC1A9093F2
:1078F000FD1A08950E94FC3B80910A1B823021F002
:1079000082E10E94E905089581E080930A1B0E94AC
:107910003D3C10920B1B1092091B08950E94FC3BEA
:1079200080910A1B823051F082E080930A1B0E94F2
:107930003D3C10920B1B1092091B089583E00E949E
:10794000E9050895CF93DF930E94EF2680E060E081
:107950000E949F04C1EFDAE1E091091BF0E070960C
:10796000EE0FFF1FEC0FFD1F808191810E945506D5
:1079700083E061E00E949F04E0910A1BF0E0EE0FBB
:10798000FF1FEE5CF44E808191810E9455068BE0D2
:1079900061E00E949F04E091091BF0E0EE0FFF1FE1
:1079A000EE0FFF1FEC0FFD1F6581768187819085AB
:1079B0004AE855E027E00E949D0682E161E00E94CE
:1079C0009F0486E50E94B204DF91CF910895EF9263
:1079D000FF92CF93DF9310920C1B80E090E0DC01CC
:1079E0008093FE1A9093FF1AA093001BB093011B83
:1079F00080E090E0A6E9B2E48093021B9093031B21
:107A0000A093041BB093051B0E94222489E50E94C9
:107A10009B129093331B8093321B88E30E949B122E
:107A20009093351B8093341B89E30E949B129093A3
:107A3000371B8093361BCCEDDAE1CE0160E270E0BB
:107A400044E150E00E9459C48EE50E949B12BC01A3
:107A5000FC0101900020E9F73197E81BF90B2AE0BF
:107A600030E02E1B3F0B36952795265F3F4F2C0F9E
:107A70003D1FC901AF010E9450C480E090E00E9408
:107A80004306CE0160E270E044E150E00E9459C438
:107A900081E090E00E9443068EE20E949B12BC01AE
:107AA000FC0101900020E9F73197E81BF90BCE01AA
:107AB000AF010E9450C480E30E949B12BC01FC01F4
:107AC00001900020E9F73197E81BF90B9E012E1B6E
:107AD0003F0B2C5E3F4FC901AF010E9450C482E0B2
:107AE00090E00E944306CE0160E270E044E150E085
:107AF0000E9459C48FE20E949B12BC01FC010190BC
:107B00000020E9F73197E81BF90B9E012E5F3F4FEC
:107B1000C901AF010E9450C481E30E949B12BC01C5
:107B2000FC0101900020E9F73197E81BF90BCE1B0F
:107B3000DF0B6296CE01AF010E9450C483E090E05B
:107B40000E944306DF91CF91FF90EF90089510922D
:107B5000061B6091651B8BE1689FB0011124625F79
:107B60007F4F80E00E94ED29089584E08093061BFA
:107B70006091651B8BE1689FB0011124625F7F4FAC
:107B800084E00E94ED29089583E08093061B6091B4
:107B9000651B8BE1689FB0011124625F7F4F83E01A
:107BA0000E94ED29089582E08093061B6091651B79
:107BB0008BE1689FB0011124625F7F4F82E00E94D9
:107BC000ED29089581E08093061B6091651B8BE190
:107BD000689FB0011124625F7F4F81E00E94ED2910
:107BE0000895CF93DF93E091061BF0E0EE0FFF1FA7
:107BF000E85CF44EC081D1818DE061E00E949F0479
:107C0000CE010E94550681EF9AE10E94C349DF919F
:107C1000CF910895EF92FF920F931F93CF93DF932D
:107C20009091651B8BE1989FC00111240E9660E036
:107C300044E020E00E94FA298093061B81E08093B3
:107C40000A1B10920B1B1092091B0E943D3CCCEDAD
:107C5000DAE1CE0160E270E044E150E00E9459C4F4
:107C60008AE00E949B12BC01FC0101900020E9F710
:107C70003197E81BF90B04E110E098012E1B3F0B34
:107C8000369527952C0F3D1FC901AF010E9450C4A6
:107C900080E090E00E944306CE0160E270E044E1A3
:107CA00050E00E9459C481E090E00E94430686E5BE
:107CB0000E949B12BC01FC0101900020E9F7319762
:107CC000E81BF90BCE01AF010E9450C489E50E9468
:107CD0009B12BC01FC0101900020E9F73197E81BE1
:107CE000F90B98012E1B3F0B369527952C0F3D1F46
:107CF000C901AF010E9450C488E50E949B12BC01DB
:107D0000FC0101900020E9F73197E81BF90B0E1BED
:107D10001F0B0C0F1D1FC801AF010E9450C482E051
:107D200090E00E944306CE0160E270E044E150E042
:107D30000E9459C485E50E949B12BC01FC01019080
:107D40000020E9F73197E81BF90B9E012E5F3F4FAA
:107D5000C901AF010E9450C487E50E949B12BC017B
:107D6000FC0101900020E9F73197E81BF90BCE1BCD
:107D7000DF0B6296CE01AF010E9450C483E090E019
:107D80000E9443060E94571289E80E949B1290931A
:107D9000391B8093381B8FE80E949B1290933B1BEA
:107DA00080933A1B8DE80E949B1290933D1B809319
:107DB0003C1B80E90E949B1290933F1B80933E1BCB
:107DC0008EE80E949B129093411B8093401B81EF91
:107DD0009AE10E94054ADF91CF911F910F91FF9088
:107DE000EF9008958CE08093F61A81E08093F81A62
:107DF000089588E18093F61A81E08093F81A089537
:107E000084E28093F61A81E08093F81A08958091B5
:107E1000F31A823030F081508093F31A81E080931E
:107E2000F81A08958091F31A803230F48F5F8093AE
:107E3000F31A81E08093F81A08958091F91A9091CD
:107E4000FA1A2FEF843F9207F0F40A969093FA1AE9
:107E50008093F91A8091F21A85508230E0F085E023
:107E60008093F21A8091A30D9091A40DA091A50D7D
:107E7000B091A60D8093FD1A9093FE1AA093FF1A5D
:107E8000B093001B08C01092F21A8EEF9FEF9093F0
:107E9000FA1A8093F91A81E08093F81A0895809174
:107EA000F91A9091FA1A8A309105F0F00A97909396
:107EB000FA1A8093F91A8091F21A87508230D0F022
:107EC00087E08093F21A8091A30D9091A40DA09168
:107ED000A50DB091A60D8093FD1A9093FE1AA09364
:107EE000FF1AB093001B06C01092F21A1092FA1AF1
:107EF0001092F91A81E08093F81A08958091F91A86
:107F00009091FA1A2FEF8D3F9207F0F4019690931B
:107F1000FA1A8093F91A8091F21A81508230E0F0B7
:107F200081E08093F21A8091A30D9091A40DA0910D
:107F3000A50DB091A60D8093FD1A9093FE1AA09303
:107F4000FF1AB093001B08C01092F21A8EEF9FEF39
:107F50009093FA1A8093F91A81E08093F81A0895A1
:107F60008091F91A9091FA1A0097F1F00197909385
:107F7000FA1A8093F91A8091F21A83508230D0F065
:107F800083E08093F21A8091A30D9091A40DA091AB
:107F9000A50DB091A60D8093FD1A9093FE1AA093A3
:107FA000FF1AB093001B06C01092F21A1092FA1A30
:107FB0001092F91A81E08093F81A0895EF92FF92D7
:107FC0000F931F93CF93DF938091F21A882309F4C4
:107FD00099C00E944E09882309F494C08091F21A36
:107FE000853030F4833050F4813008F48BC00BC0FE
:107FF000873070F0893008F085C00FC080E490E0D1
:10800000C0EBDFE30EC080E290E0CEE7DFE309C023
:1080100080E091E0CDE1DFE304C080E890E0CFE4D0
:10802000DFE30E945909882309F46EC08091F21A97
:10803000843009F43FC0853040F48230D9F1833078
:1080400070F4813009F05EC00AC0863099F1863044
:1080500030F0873021F0883009F054C02BC0809177
:10806000A30D9091A40DA091A50DB091A60D209106
:10807000FD1A3091FE1A4091FF1A5091001B7C01AD
:108080008D01E21AF30A040B150BA801970125369E
:10809000310541055105C0F18093FD1A9093FE1AF8
:1080A000A093FF1AB093001B8091F21A8F5F809308
:1080B000F21A2AC08091A30D9091A40DA091A50D54
:1080C000B091A60D2091FD1A3091FE1A4091FF1A31
:1080D0005091001B7C018D01E21AF30A040B150B71
:1080E000A80197012B3031054105510568F08093B7
:1080F000FD1A9093FE1AA093FF1AB093001BFE0185
:10810000099502C01092F21AC091F91AD091FA1A88
:108110008091FB1A9091FC1AC817D90761F182E08F
:1081200061E00E949F04CE0160EC75E045E00E9492
:1081300058068BE061E00E949F04BE0180E090E061
:108140000E9423C120E030E040E752E40E94D9C100
:1081500020E030E04AE754E40E948AC044EC55E055
:1081600028E00E949D068091F91A9091FA1A909346
:10817000FC1A8093FB1ADF91CF911F910F91FF9012
:10818000EF900895CF92DF92EF92FF920F931F939B
:10819000CF93DF9381E08093F11A1092F21A8FEF60
:1081A0009FEF9093FC1A8093FB1A1092F81A90910B
:1081B000651B8BE1989FC00111243091671B2DE056
:1081C000329F90011124820F931F449640E050E0AB
:1081D000BA0100E21EEF2FE63AE40F2EF0E0CF2EB8
:1081E000F0E8DF2EFBEBEF2EF5E4FF2EF02D0E94E2
:1081F000172B20E030E040E752E40E948AC07B0168
:108200008C017F2D912F20E030E0A9010E9486C0D3
:1082100018162CF01092FA1A1092F91A1FC06E2D2F
:108220007F2D802F912F20E03FEF4FE757E40E94F2
:10823000D5C118163CF48EEF9FEF9093FA1A8093F5
:10824000F91A0CC06E2D7F2D802F912F0E943CC2F9
:108250000E94F7C07093FA1A6093F91A0CED1AE1B4
:10826000C80160E270E044E150E00E9459C487E632
:108270000E949B12BC01FC0101900020E9F731979C
:10828000E81BF90B2AE030E02E1B3F0B36952795B3
:10829000200F311FC901AF010E9450C488E60E941F
:1082A0009B12BC01FC0101900020E9F73197E81B0B
:1082B000F90BC4E1D0E09E012E1B3F0B200F311FB4
:1082C000C901AF010E9450C480E090E00E944306C3
:1082D000C80160E270E044E150E00E9459C481E0CE
:1082E00090E00E9443068CE20E949B12BC01FC01BC
:1082F00001900020E9F73197E81BF90BC801AF01A5
:108300000E9450C48AE20E949B12BC01FC010190B1
:108310000020E9F73197E81BF90BCE1BDF0BC00FEC
:10832000D11FCE01AF010E9450C482E090E00E94B4
:108330004306C80160E270E044E150E00E9459C485
:108340008DE20E949B12BC01FC0101900020E9F724
:108350003197E81BF90B0E5F1F4FC801AF010E9458
:1083600050C48BE20E949B12BC01FC0101900020D2
:10837000E9F73197E81BF90B2EEE3AE12E1B3F0B84
:10838000C901AF010E9450C483E090E00E944306FF
:10839000DF91CF911F910F91FF90EF90DF90CF90E1
:1083A00008950F931F938091F81A882361F16091CB
:1083B000651B0BE1609FB00111248091671B1DE0DC
:1083C000819FC0011124680F791F605F7F4F8091EA
:1083D000F31A0E94ED296091651B609FB001112482
:1083E0008091671B819FC0011124680F791F6F5E08
:1083F0007F4F8091F61A0E94ED298091651B609154
:10840000671B0E945B591F910F9108951F93DF9383
:10841000CF9300D000D0CDB7DEB7182F8091F11ADE
:10842000882319F08130B9F503C00E94D14133C0CF
:108430008091F81A882379F12091F91A3091FA1A6B
:108440008CE390E0289FB001299F700D389F700D3C
:10845000112480E090E00E9423C169837A838B839A
:108460009C836091651B8BE1689FB0011124909102
:10847000671B8DE0989FC0011124680F791F6C5E07
:108480007F4FCE0101960E94542A8091651B609116
:10849000671B0E945B59812F0E94E9050F900F9086
:1084A0000F900F90CF91DF911F9108958091F11A55
:1084B000813011F083E001C084E10E9406420895FA
:1084C0008091F11A882311F086E101C085E10E94B4
:1084D000064208950F931F938091651B0BE1809FC7
:1084E000C00111242091671B1DE0219F90011124E0
:1084F000820F931F409661E040E221E00E94FA293A
:108500008093F31A8091651B809FC00111242091F4
:10851000671B219F90011124820F931F41966CE0ED
:1085200044E22CE00E94FA298093F61A1092F81A7D
:108530001F910F9108958091671B882361F48091AA
:10854000F51A882391F00E94D14181E08093671B46
:108550000E946A4208958091F41A882331F00E94A3
:10856000D1411092671B0E946A420895EF92FF92D8
:108570000F931F93DF93CF93CDB7DEB729970FB635
:10858000F894DEBF0FBECDBF82E160E00E949F0481
:108590008091F31A90E06BEC75E042E00E9458067F
:1085A0000CED1AE1C80160E270E044E150E00E9485
:1085B00059C48091651B2BE1829FC0011124409119
:1085C000671B3DE0439FA0011124840F951F429635
:1085D00060E044E020E039870E94FA29E82FF0E0CB
:1085E000EE0FFF1FE65CF44E60817181DB01FD013F
:1085F00001900020E9F73197EA1BFB0BC801AF019E
:108600000E9450C48DB79EB708970FB6F8949EBFCE
:108610000FBE8DBFEDB7FEB731967E010894E11C09
:10862000F11CADB7BEB71296FC92EE92119788E09E
:1086300090E0938382838091321B9091331B9583CA
:1086400084838091651B90E00196978386830E94C6
:10865000B6C4F70101900020E9F73197EE19FF0940
:1086600004E110E0A8014E1B5F0B5695479544525C
:10867000554E8DB79EB708960FB6F8949EBF0FBEA5
:108680008DBFCA01B701AF010E9450C48091651B24
:10869000ABE18A9FC00111242091671B3985239F7C
:1086A00090011124820F931F439660E043E020E085
:1086B0000E94FA29E82FF0E0EE0FFF1FEC5BF44E6A
:1086C00060817181DB01FD0101900020E9F73197A4
:1086D000EA1BFB0B0E1B1F0B0452154EC801AF010A
:1086E0000E9450C481E090E00E94430688E063E06D
:1086F0000E949F048091F61A90E06BEC75E042E0D6
:108700000E9458068091F71A882329F40091341B9F
:108710009091351B09C0E091671BF0E0EE0FFF1F41
:10872000EA5CF44E00819181E02FF92FDF010D907A
:108730000020E9F7EA1B8E2F8B5E62E099870E948A
:108740009F04802F99850E94550629960FB6F894AC
:10875000DEBF0FBECDBFCF91DF911F910F91FF9074
:10876000EF900895EF92FF92CF93DF931092F11A5A
:108770008091651B6EE00E94CB69929591709093F9
:10878000F41A8091651B6CE00E94CB699295917000
:108790009093F51A8091F41A292F280F2093F71A35
:1087A000992311F0882319F01092671B03C081E010
:1087B0008093671B0E946A42CCEDDAE1CE0160E251
:1087C00070E044E150E00E9459C486E60E949B128A
:1087D000BC01FC0101900020E9F73197E81BF90B7F
:1087E000CE01AF010E9450C480E090E00E94430699
:1087F000CE0160E270E044E150E00E9459C48FE392
:108800000E949B12BC01FC0101900020E9F7319706
:10881000E81BF90B9E01295F3F4FC901AF010E9480
:1088200050C481E090E00E944306CE0160E270E017
:1088300044E150E00E9459C481E90E949B12BC01AE
:10884000FC0101900020E9F73197E81BF90BCE01FC
:10885000AF010E9450C482E090E00E944306CE0126
:1088600060E270E044E150E00E9459C482E90E9455
:108870009B12BC01FC0101900020E9F73197E81B35
:10888000F90B2296CE01AF010E9450C483E90E94E9
:108890009B12BC01FC0101900020E9F73197E81B15
:1088A000F90B2EEE3AE12E1B3F0BC901AF010E94DE
:1088B00050C486E58093E61A83E090E00E94430668
:1088C0000E9457128BE00E949B129093331B80935F
:1088D000321B89E50E949B129093351B8093341BB9
:1088E00087E80E949B129093371B8093361B88E881
:1088F0000E949B129093391B8093381BCAE3D2E0ED
:10890000D0933B1BC0933A1B89E60E949B12909325
:108910003D1B80933C1B8BE60E949B1290933F1B58
:1089200080933E1B8AE60E949B129093411B80938A
:10893000401B8CE60E949B129093431B8093421B2A
:10894000D093451BC093441B8FE60E949B129093CB
:10895000471B8093461B8EE60E949B129093491BF7
:108960008093481B80E70E949B1290934B1B80933F
:108970004A1BDF91CF91FF90EF9008951F93809154
:108980000A1B813021F08230B1F511E001C010E006
:108990009091081B8091651B4091F61A5091F71A2F
:1089A0006091F81A7091F91A992399F090E0212FAB
:1089B0000E943F6D4091FA1A5091FB1A6091FC1A87
:1089C0007091FD1A8091651B90E0212F0E94256D0A
:1089D00012C090E0212F0E94736D4091FA1A5091BD
:1089E000FB1A6091FC1A7091FD1A8091651B90E052
:1089F000212F0E94596D1F9108951F9380910A1B8A
:108A0000813021F08230B1F511E001C010E0909189
:108A1000081B8091651B992399F090E0612F0E94BB
:108A2000656A6093F61A7093F71A8093F81A909318
:108A3000F91A8091651B90E0612F0E94596A12C05B
:108A400090E0612F0E947D6A6093F61A7093F71A86
:108A50008093F81A9093F91A8091651B90E0612F2A
:108A60000E94716A6093FA1A7093FB1A8093FC1A41
:108A70009093FD1A1F9108950E94BE4480910A1B95
:108A8000823021F085E10E94E905089581E080931C
:108A90000A1B10920B1B1092091B0E94FD440895A3
:108AA0000E94BE4480910A1B823051F082E0809384
:108AB0000A1B10920B1B1092091B0E94FD44089583
:108AC00087E10E94E90508951F93DF93CF930F92EA
:108AD000CDB7DEB70E94EF2680E060E00E949F04E1
:108AE000E091091BF0E0EE0FFF1FEF5EF44E808176
:108AF00091810E94550680910A1B813029F41091C2
:108B0000321B9091331B04C01091341B9091351B84
:108B1000E12FF92FDF010D900020E9F79F012A1BBB
:108B20003B0B255F3F4F36952795822F61E0998358
:108B30000E949F04812F99810E9455068BE061E07D
:108B40000E949F04E091091BF0E0EE0FFF1FEE0F63
:108B5000FF1FEF50F54E658176818781908540E05B
:108B600056E027E00E949D0682E161E00E949F049A
:108B700086E50E94B2040F90CF91DF911F91089576
:108B8000EF92FF92CF93DF9381E080930A1B1092C4
:108B90000B1B1092091B8091651B6CE00E94CB6936
:108BA000929591709093081B10920C1B80E090E0BE
:108BB000DC018093FE1A9093FF1AA093001BB093E0
:108BC000011B80E090E0A8E4B2E48093021B909344
:108BD000031BA093041BB093051B0E94FD44CCED26
:108BE000DAE1CE0160E270E044E150E00E9459C455
:108BF0008EE50E949B12BC01FC0101900020E9F768
:108C00003197E81BF90B2AE030E02E1B3F0B36951D
:108C10002795265F3F4F2C0F3D1FC901AF010E94D2
:108C200050C480E090E00E944306CE0160E270E014
:108C300044E150E00E9459C481E090E00E94430664
:108C40008EE20E949B12BC01FC0101900020E9F71A
:108C50003197E81BF90BCE01AF010E9450C480E3AD
:108C60000E949B12BC01FC0101900020E9F73197A2
:108C7000E81BF90B9E012E1B3F0B2C5E3F4FC901D9
:108C8000AF010E9450C482E090E00E944306CE01F2
:108C900060E270E044E150E00E9459C48FE20E941B
:108CA0009B12BC01FC0101900020E9F73197E81B01
:108CB000F90B9E012E5F3F4FC901AF010E9450C4C6
:108CC00081E30E949B12BC01FC0101900020E9F7A6
:108CD0003197E81BF90BCE1BDF0B6296CE01AF017B
:108CE0000E9450C483E090E00E9443060E94571205
:108CF0000E94222484E90E949B129093331B80934C
:108D0000321B85E90E949B129093351B8093341B84
:108D1000DF91CF91FF90EF900895EF92FF920F9324
:108D20001F93CF93DF931092F61ACCEDDAE1CE01C8
:108D300060E270E044E150E00E9459C489E60E947C
:108D40009B12BC01FC0101900020E9F73197E81B60
:108D5000F90BCE01AF010E9450C485E10E949B1225
:108D6000BC01FC0101900020E9F73197E81BF90BE9
:108D700004E110E098012E1B3F0B369527952C0F30
:108D80003D1FC901AF010E9450C48AE60E949B1298
:108D9000BC01FC0101900020E9F73197E81BF90BB9
:108DA0000E1B1F0B0C0F1D1FC801AF010E9450C4EA
:108DB00082E090E00E944306CE0160E270E044E170
:108DC00050E00E9459C48BE60E949B12BC01FC013A
:108DD00001900020E9F73197E81BF90B9E012E5F07
:108DE0003F4FC901AF010E9450C48CE60E949B1204
:108DF000BC01FC0101900020E9F73197E81BF90B59
:108E0000CE1BDF0B6296CE01AF010E9450C483E0FF
:108E100090E00E944306DF91CF911F910F91FF9048
:108E2000EF9008958091F61A882319F40E94C205E4
:108E300008950E948D460895EF92FF92CF93DF939D
:108E400081E08093F61ACCEDDAE1CE0160E270E0C9
:108E500044E150E00E9459C48DE60E949B12BC017F
:108E6000FC0101900020E9F73197E81BF90BCE01D6
:108E7000AF010E9450C48EE60E949B12BC01FC010F
:108E800001900020E9F73197E81BF90B9E012E1B9A
:108E90003F0B2C5E3F4FC901AF010E9450C482E0DE
:108EA00090E00E944306CE0160E270E044E150E0B1
:108EB0000E9459C48FE60E949B12BC01FC010190E4
:108EC0000020E9F73197E81BF90B9E012E5F3F4F19
:108ED000C901AF010E9450C480E70E949B12BC01EF
:108EE000FC0101900020E9F73197E81BF90BCE1B3C
:108EF000DF0B6296CE01AF010E9450C483E090E088
:108F00000E944306DF91CF91FF90EF9008958091EA
:108F1000F61A882349F48091F71A813029F40E94C7
:108F200057120E941C4708950E94070608950F9348
:108F30001F939091F61A6091651B8091671B99238E
:108F400011F593E09093F71A0BE1609FB0011124A3
:108F50001DE0819FC0011124680F791F6E5E7F4F55
:108F600083E00E94ED296091651B609FB001112490
:108F70008091671B819FC0011124680F791F6D5E6E
:108F80007F4F80E010C092E09093F81A9BE1699FB8
:108F9000B00111249DE0899FC0011124680F791F41
:108FA0006D5E7F4F82E00E94ED298091651B60918C
:108FB000671B0E945B590E9407061F910F9108953D
:108FC0000F931F939091F61A6091651B8091671B18
:108FD000992311F594E09093F71A0BE1609FB0018B
:108FE00011241DE0819FC0011124680F791F6E5E5E
:108FF0007F4F84E00E94ED296091651B609FB00166
:1090000011248091671B819FC0011124680F791F73
:109010006D5E7F4F80E010C093E09093F81A9BE163
:10902000699FB00111249DE0899FC0011124680F40
:10903000791F6D5E7F4F83E00E94ED298091651B53
:109040006091671B0E945B590E9407061F910F9158
:1090500008950F931F939091F61A6091651B80916C
:10906000671B992311F592E09093F71A0BE1609F2B
:10907000B00111241DE0819FC0011124680F791FE8
:109080006E5E7F4F82E00E94ED296091651B609FBC
:10909000B00111248091671B819FC0011124680FCA
:1090A000791F6D5E7F4F80E010C091E09093F81AB9
:1090B0009BE1699FB00111249DE0899FC0011124AB
:1090C000680F791F6D5E7F4F81E00E94ED298091CE
:1090D000651B6091671B0E945B590E9407061F91E8
:1090E0000F9108958091F61A882301F581E080930D
:1090F000F71A6091651B8BE1689FB0011124909174
:10910000671B8DE0989FC0011124680F791F6E5E68
:109110007F4F81E00E94ED298091651B6091671B64
:109120000E945B590E9457120E941C47089581EFCC
:109130009AE10E94C3490895EF92FF920F931F9303
:10914000DF93CF93CDB7DEB728970FB6F894DEBF85
:109150000FBECDBF8091651B1BE1819FC001112413
:109160002091671B0DE0209F90011124820F931F17
:10917000429660E044E020E00E94FA298093F71ACA
:109180006091651B2091671B813089F4619FC0014C
:109190001124209F80011124800F911F439660E0CD
:1091A00043E020E00E94FA298093F81A0FC0109241
:1091B000F81A619FB0011124209F80011124600FD3
:1091C000711F6D5E7F4F80E00E94ED298CED9AE16A
:1091D00060E270E044E150E00E9459C481E00E94E6
:1091E0009B12BC01FC0101900020E9F73197E81BBC
:1091F000F90B04E110E098012E1B3F0B36952795E3
:109200002452354EC901AF010E9450C480E090E065
:109210000E9443068CED9AE160E270E044E150E088
:109220000E9459C48BE00E949B122DB73EB7285074
:1092300030400FB6F8943EBF0FBE2DBFEDB7FEB75E
:1092400031967E010894E11CF11CADB7BEB71296B1
:10925000FC92EE92119728E030E0338322839583CD
:1092600084838091651B90E00196978386830E949A
:10927000B6C4F70101900020E9F73197EE19FF0914
:109280000E1B1F0B169507950452154E2DB73EB7B2
:10929000285F3F4F0FB6F8943EBF0FBE2DBFC801E9
:1092A000B701AF010E9450C481E090E00E944306E4
:1092B0000E948D4681EF9AE10E94054A28960FB6DA
:1092C000F894DEBF0FBECDBFCF91DF911F910F91FC
:1092D000FF90EF900895FF920F931F93082FF62EA3
:1092E0008430C0F4862F602F0E949F0410E0812FED
:1092F0000E942B041F5F1430D1F7033059F0602F08
:109300006F5F8F2D0E949F04812F0E942B041F5F8F
:109310001830D1F71F910F91FF900895AF92BF922F
:10932000CF92DF92EF92FF921F93CF93DF937C0156
:10933000162FC0E0D0E08C2F612F0E9490046E01A8
:1093400083E0CC0CDD1C8A95E1F7CE0CDF1CAA244F
:10935000BB24F60181916F010E942B040894A11C8B
:10936000B11CF8E0AF16B104A1F72196C830D105C1
:1093700011F7DF91CF911F91FF90EF90DF90CF9089
:10938000BF90AF900895CF93DF93EC016C81209153
:10939000A30D3091A40D4091A50D5091A60D88818B
:1093A0009981AA81BB81662371F4281B390B4A0B72
:1093B0005B0B203531054105510520F181E08C839F
:1093C00086E796E00CC0281B390B4A0B5B0B243157
:1093D000310541055105B0F01C8286E396E060E05E
:1093E0000E948E4980E060E00E946B498091A30D4D
:1093F0009091A40DA091A50DB091A60D888399839D
:10940000AA83BB83DF91CF910895CF93DF93EC01C3
:1094100086E396E060E00E948E4980E060E00E9472
:109420006B498091A30D9091A40DA091A50DB091D1
:10943000A60D88839983AA83BB831C82DF91CF9179
:10944000089580E060E041E00E941C6408958091EE
:10945000A30D9091A40DA091A50DB091A60D209102
:10946000F11A3091F21A4091F31A5091F41A821BBA
:10947000930BA40BB50B8D3221E0920720E0A207DD
:1094800020E0B20710F00E94214A0895EF92FF9267
:109490000F931F93CF93DF938091A30D9091A40D11
:1094A000A091A50DB091A60D8093F11A9093F21A98
:1094B000A093F31AB093F41ACCEDDAE1CE0160E296
:1094C00070E044E150E00E9459C482E10E949B1286
:1094D000BC01FC0101900020E9F73197E81BF90B72
:1094E0008E010B5F1F4FC801AF010E9450C480E086
:1094F00090E00E944306CE0160E270E044E150E05B
:109500000E9459C483E10E949B12BC01FC0101909E
:109510000020E9F73197E81BF90BC801AF010E9461
:1095200050C481E090E00E944306CE0160E270E00A
:1095300044E150E00E9459C485E40E949B12BC01A2
:10954000FC0101900020E9F73197E81BF90BCE01EF
:10955000AF010E9450C482E70E949B12BC01FC0133
:1095600001900020E9F73197E81BF90B9E012E1BB3
:109570003F0B2C5E3F4FC901AF010E9450C482E0F7
:1095800090E00E944306CE0160E270E044E150E0CA
:109590000E9459C483E090E00E94430686EB96E067
:1095A00060E00E948E4980E060E00E946B49DF919C
:1095B000CF911F910F91FF90EF9008958091621BC2
:1095C0008093E40D2091A30D3091A40D4091A50D41
:1095D0005091A60D28523040404050402093CF0D6E
:1095E0003093D00D4093D10D5093D20D90E00E9456
:1095F000B86A60937D1B70937E1B80937F1B909352
:10960000801B8091E40D90E00E94046B9B01AC01F3
:1096100060936D1B70936E1B80936F1B9093701BF8
:1096200060917D1B70917E1B80917F1B9091801BB0
:109630000E94D9C16093751B7093761B8093771B32
:109640009093781B8091E40D90E00E94B26A609341
:10965000811B7093821B8093831B9093841B80914A
:10966000E40D90E00E94FE6A9B01AC016093711BC7
:109670007093721B8093731B9093741B6091811B7A
:109680007091821B8091831B9091841B0E94D9C191
:109690006093791B70937A1B80937B1B90937C1B48
:1096A0001092D30D1092D40D1092D50D1092D60DAC
:1096B0001092D70D1092D80D1092D90D1092DA0D8C
:1096C0001092DB0D1092DC0D1092DD0D1092DE0D6C
:1096D0001092DF0D1092E00D1092E10D1092E20D4C
:1096E0001092E30D0895CF92DF92EF92FF920F93C5
:1096F0001F939091621B8091E40D981711F00E94C6
:10970000DE4A8091A30D9091A40DA091A50DB0917A
:10971000A60D2091CF0D3091D00D4091D10D5091DB
:10972000D20D7C018D01E21AF30A040B150BA8017E
:109730009701223331054105510508F4AEC18093EC
:10974000CF0D9093D00DA093D10DB093D20DE0909A
:10975000D30DF090D40D0091D50D1091D60D8091C0
:10976000E40D60E00E94CB69A0E0B0E09F70A070C3
:10977000B0708E0D9F1DA01FB11F8093D30D9093CD
:10978000D40DA093D50DB093D60DE090D70DF090E9
:10979000D80D0091D90D1091DA0D8091E40D64E09F
:1097A0000E94CB69A0E0B0E09F70A070B0708E0DF9
:1097B0009F1DA01FB11F8093D70D9093D80DA0932C
:1097C000D90DB093DA0DE090DB0DF090DC0D009137
:1097D000DD0D1091DE0D8091E40D65E00E94BE6A02
:1097E000AA2797FDA095BA2F8E0D9F1DA01FB11F10
:1097F0008093DB0D9093DC0DA093DD0DB093DE0D17
:10980000E090DF0DF090E00D0091E10D1091E20D80
:109810008091E40D62E00E94BE6AAA2797FDA095A0
:10982000BA2F8E0D9F1DA01FB11F8093DF0D909347
:10983000E00DA093E10DB093E20D8091E30D8F5FF9
:109840008093E30D843008F428C1C0908D04D0903B
:109850008E04E0908F04F09090048EE992E040E056
:1098600050E068E472EC00E010E028E432E40E948A
:10987000172B7B018C016091D30D7091D40D8091D9
:10988000D50D9091D60D0E9425C19B01AC01C80158
:10989000B7010E94D9C120E030E040E85EE30E94B9
:1098A000D9C160937D1B70937E1B80937F1B909327
:1098B000801BC0909104D0909204E0909304F090AB
:1098C000940482EA92E040E050E068E472EC00E048
:1098D00010E028E432E40E94172B7B018C01609198
:1098E000D70D7091D80D8091D90D9091DA0D0E940D
:1098F00025C19B01AC01C801B7010E94D9C120E07C
:1099000030E040E85EE30E94D9C16093811B709310
:10991000821B8093831B9093841BC0909504D090EE
:109920009604E0909704F090980486EA92E040E074
:1099300050E068E472EC00E010E028E432E40E94B9
:10994000172B7B018C016091DB0D7091DC0D8091F8
:10995000DD0D9091DE0D0E9425C19B01AC01C80177
:10996000B7010E94D9C120E030E040E85EE30E94E8
:10997000D9C160936D1B70936E1B80936F1B909386
:10998000701BC0909904D0909A04E0909B04F090D2
:109990009C048AEA92E040E050E068E472EC00E067
:1099A00010E028E432E40E94172B7B018C016091C7
:1099B000DF0D7091E00D8091E10D9091E20D0E941C
:1099C00025C19B01AC01C801B7010E94D9C120E0AB
:1099D00030E040E85EE30E94D9C17B018C01862F14
:1099E0009F2DA02FB12F8093711B9093721BA0937A
:1099F000731BB093741B60917D1B70917E1B8091D3
:109A00007F1B9091801B20916D1B30916E1B4091AC
:109A10006F1B5091701B0E94D9C16093751B70938E
:109A2000761B8093771B9093781B6091811B7091BC
:109A3000821B8091831B9091841B2E2D3F2D402FE4
:109A4000512F0E94D9C16093791B70937A1B809328
:109A50007B1B90937C1B1092D30D1092D40D10920F
:109A6000D50D1092D60D1092D70D1092D80D1092E0
:109A7000D90D1092DA0D1092DB0D1092DC0D1092C0
:109A8000DD0D1092DE0D1092DF0D1092E00D1092A0
:109A9000E10D1092E20D1092E30D1F910F91FF90D6
:109AA000EF90DF90CF9008952F923F924F925F9268
:109AB0006F927F928F929F92AF92BF92CF92DF92DE
:109AC000EF92FF920F931F935A016B017801890166
:109AD000E82FF0E0EE0FFF1FEE0FFF1FEB56F44EE6
:109AE000208031804280538060E070E088EC92E416
:109AF000A20191010E9421C09B01AC01C801B701E4
:109B00000E94D9C1A60195010E948AC020E030E0E0
:109B100048EC52E40E948AC0962E872E782E692E39
:109B2000A62EB72EC82ED92E8C2D880F8D2D881FCE
:109B30008F3FA9F0692D782D872D962D20E030E0FC
:109B4000A9010E9486C087FD0AC0692D782D872D46
:109B5000962DA80197010E94D5C1181684F4C8015A
:109B6000B701A20191010E94D9C120E030E048EC88
:109B700052E40E948AC0A62EB72EC82ED92E6A2D76
:109B80007B2D8C2D9D2D1F910F91FF90EF90DF90DD
:109B9000CF90BF90AF909F908F907F906F905F908D
:109BA0004F903F902F9008956F927F928F929F9247
:109BB000AF92BF92CF92DF92EF92FF920F931F93DB
:109BC0003B014C01CA01B901A80197010E94D9C10A
:109BD000A60195010E948AC09B01AC01C401B3019A
:109BE0000E9422C01F910F91FF90EF90DF90CF90C5
:109BF000BF90AF909F908F907F906F900895882333
:109C000059F48091621B6EE00E94CB6994FF17C0EB
:109C10008091621B62E00CC0813089F48091621BEC
:109C20006CE00E94CB6994FF0AC08091621B65E0E2
:109C30000E94CB69892F829586958170089580E076
:109C400008951F93CF93DF93182F0E94FF4D212F6C
:109C500030E0F901E651F24F8083220F331F220FCB
:109C6000331FF901E357F44E80E090E0DC0180837C
:109C70009183A283B383F901EB56F44E80839183E1
:109C8000A283B383F901EB57F44E2359344EE90113
:109C900088819981AA81BB8180839183A283B383C8
:109CA000DF91CF911F9108958091621B8093E90D00
:109CB00080E00E94214E81E00E94214E08954F9243
:109CC0005F926F927F928F929F92AF92BF92CF924C
:109CD000DF92EF92FF920F931F93CF93DF93B82EF3
:109CE0008091A30D9091A40DA091A50DB091A60D0A
:109CF0002091E50D3091E60D4091E70D5091E80D72
:109D00007C018D01E21AF30A040B150BA8019701DF
:109D1000243631054105510508F4D9C18093E50D7C
:109D20009093E60DA093E70DB093E80D0B2D10E096
:109D3000E801C651D24F8B2D0E94FF4D782E8881AD
:109D4000871521F08B2D0E94214E78828DE090E0C6
:109D5000089FE001099FD00D189FD00D112490910C
:109D6000621B8BE1989FC001112440968C0F9D1FB0
:109D700061E040E221E00E94FA29A82E882311F434
:109D8000AA24A3949091621B8BE1989FC001112497
:109D900044968C0F9D1F40E050E0BA0100E21EEF98
:109DA0002FE63AE40F2EF0E0CF2EF0E8DF2EFBEBAB
:109DB000EF2EF5E4FF2EF02D0E94172B7B018C0176
:109DC0002A2D30E0B901882777FD8095982F0E94D1
:109DD00025C1A80197010E94D9C120E030E040E7E9
:109DE00052E40E948AC0A62E172F082F692E8B2CB2
:109DF0009924E401CC0FDD1FCC0FDD1FFE01E359D8
:109E0000F44EC080D180E280F380E894F7F87720A8
:109E100009F435C18091621B62E00E94CB6996FF14
:109E200012C08091621B65E00E94CB6996FF0BC057
:109E3000CB56D44E80E090E0A8ECB2E488839983BE
:109E4000AA83BB8310C08091621B6B2D0E9499581E
:109E5000F401EE0FFF1FEE0FFF1FEB56F44E608371
:109E60007183828393838B2DB701A601F8010A2D9C
:109E70001F2F2E2F362D0E94544D2B013C01C70160
:109E8000B60120E030E040E85FE30E9486C088230E
:109E90002CF460E070E080E89FE3E5C0C701B60104
:109EA00020E030E040E251E40E9486C08823ECF4D8
:109EB000C701B60120E030E040E85FE30E9421C026
:109EC0007B018C0160E070E080E89FE32DEC3CECCE
:109ED0004CE45FEB0F2EF0E0AF2EF0E0BF2EF0E190
:109EE000CF2EF1E4DF2EF02DBCC0C701B60120E07B
:109EF00030E040E751E40E9486C088239CF4C7010B
:109F0000B60120E030E040E251E40E9421C07B0134
:109F10008C016DEC7CEC8CE49EE320E73EEC48E0A9
:109F20005DEB95C0C701B60120E030E040EA51E4A6
:109F30000E9486C088239CF4C701B60120E030E06F
:109F400040E751E40E9421C07B018C0161E379E983
:109F50008AE29EE328EB3CEF47E05DEB78C0C70167
:109F6000B60120E030E048EC51E40E9486C088232E
:109F70009CF4C701B60120E030E040EA51E40E94C1
:109F800021C07B018C0163E07AE988E09EE32CEA42
:109F900033E140ED5CEB5BC0C701B60120E030E08F
:109FA00040EF51E40E9486C088239CF4C701B601AB
:109FB00020E030E048EC51E40E9421C07B018C019C
:109FC0006BE17FE28DED9DE323E133E840E45DEB5F
:109FD0003EC0C701B60120E030E04CE052E40E94F0
:109FE00086C088239CF4C701B60120E030E040EF32
:109FF00051E40E9421C07B018C0163E27BED89E783
:10A000009DE324E430E645E65CE321C0C701B601E8
:10A0100020E030E040E252E40E9486C087FD05C0A7
:10A0200065E975E688E89DE31EC0C701B60120E03A
:10A0300030E04CE052E40E9421C07B018C016AE9CF
:10A0400079E989E99DE328E230EA49E05CEB0F2EEB
:10A05000F0E0AF2EF0E0BF2EF0EACF2EF0E4DF2EDE
:10A06000F02D0E94D44DE401CC0FDD1FCC0FDD1F7D
:10A07000C357D44EA30192010E94D9C124C080913C
:10A08000621B6B2D0E9499589B01AC0165E9862EDD
:10A090006BE1962E8C0E9D1E60E070E088EC92E4E1
:10A0A0000E9421C0F40160837183828393838B2D8E
:10A0B000B701A601F8010A2D1F2F2E2F362D0E9461
:10A0C000544DC357D44E688379838A839B83DF9131
:10A0D000CF911F910F91FF90EF90DF90CF90BF90A5
:10A0E000AF909F908F907F906F905F904F9008956A
:10A0F0009091E90D8091621B981711F00E94544EC7
:10A100008091621B6EE00E94CB6994FF03C080E0E7
:10A110000E945F4E8091621B6CE00E94CB6994FFAD
:10A1200003C081E00E945F4E0895249A2C9A0895FE
:10A1300080E58CBD8DB581608DBD2C9886E00E9438
:10A140000D052C9A089580E58CBD8DB581608DBD7F
:10A150002C9885E00E940D058FEF0E940D052C9A2A
:10A1600008951F931FB7F8940E94A35017FF01C0D2
:10A1700078941F9108951F93CF93DF931FB7F8949E
:10A180008091EC0D882381F0C0E0D0E4F8940E9427
:10A19000B15080FF02C0219719F41092EC0D04C059
:10A1A00017FFF4CF7894F2CF812FDF91CF911F91D9
:10A1B00008950F931F93082F0E94BB50182F0E94E1
:10A1C000985080E58CBD8DB581608DBD2C9881E067
:10A1D0000E940D05802F0E940D052C9A81E080932E
:10A1E000EC0D17FF01C078941F910F910895EF9225
:10A1F000FF920F931F93DF93CF9300D0CDB7DEB7BD
:10A20000182F7B014A8399830E94BB50082F80E559
:10A210008CBD8DB581608DBD2C9883E00E940D05AD
:10A220009981892F0E940D05812F0E940D05C7017C
:10A230004A81642F70E00E9413052C9A07FF01C029
:10A2400078940F900F90CF91DF911F910F91FF9015
:10A25000EF900895DF93CF930F92CDB7DEB7BE0195
:10A260006F5F7F4F41E00E94F75089810F90CF913F
:10A27000DF910895EF92FF921F93DF93CF9300D069
:10A28000CDB7DEB7182F7B014A8399830E9498507F
:10A2900080E58CBD8DB581608DBD2C9882E00E94DB
:10A2A0000D059981892F0E940D05812F0E940D05B2
:10A2B000C7014A81642F70E00E9423052C9A81E037
:10A2C0008093EC0D0F900F90CF91DF911F91FF9035
:10A2D000EF900895CF92DF92EF92FF920F931F932A
:10A2E000CF93DF93EC017B01142F80E4D82E20C0A4
:10A2F000CE018F73082F812F90E0800F911D813444
:10A30000910514F4012F03C09D2D901B092F0E946D
:10A31000BB50C82ECE01B701402F0E943A51C7FE54
:10A3200001C07894C05CDF4FC07CE00EF11C101BB4
:10A330001123F1F6DF91CF911F910F91FF90EF90D4
:10A34000DF90CF900895DF93CF930F92CDB7DEB714
:10A350006983BE016F5F7F4F41E00E946A510F9099
:10A36000CF91DF91089581E080930E0708951092B8
:10A37000E900E0EFF0E080818860808308951F921B
:10A380000F920FB60F920BB60F9211242F933F939B
:10A390004F935F936F937F938F939F93AF93BF93ED
:10A3A000EF93FF938091F40080FF0CC08091F40044
:10A3B0008E7F8093F4000E94A3578091E800877FEE
:10A3C0008093E8008091F40082FF1BC082E08093BC
:10A3D000E9008091E8008E7F8093E8008091F00092
:10A3E00080FF0FC08091F4008B7F8093F400609118
:10A3F000A21B7091A31B8091A01B9091A11B0E9496
:10A40000DE558091F40081FF35C081E08093E90042
:10A410008091F00082FF2EC08091F4008D7F8093A8
:10A42000F4008091E80085FF25C08091F2009091B2
:10A43000F3000097F9F08EEE9DE063E171E00E9479
:10A4400043558823B9F48EEE9DE061E07FE00E94E1
:10A45000BB2BBC01009771F082E08093E9008091F2
:10A46000E80085FF05C081E09FE00E94DE5502C044
:10A470000E949457FF91EF91BF91AF919F918F915F
:10A480007F916F915F914F913F912F910F900BBEF4
:10A490000F900FBE0F901F9018950E94945708952B
:10A4A000F8940E94735680919D1B10929D1B789486
:10A4B000882319F081E00E944B1B0895CF93DF930E
:10A4C0008091A61B833089F1843030F4813059F0BB
:10A4D000823009F082C060C08A3009F449C08B30F4
:10A4E00009F07BC02FC08091A51B813A09F075C08F
:10A4F000C1E0DFE08EEE9DE0BE010E94BB2BBC01FF
:10A50000181619060CF069C08091E800877F8093C7
:10A51000E800CE010E94815583E191E0FE019C019B
:10A52000119221503040E1F74FC08091A51B813A34
:10A5300009F053C08091E800877F8093E800809104
:10A540000E0735C08091A51B813209F046C080916D
:10A55000E800877F8093E80010920E078091A71B88
:10A560009091A81B009789F081E080930E070DC0A1
:10A570008091A51B813289F58091E800877F8093C7
:10A58000E8008091A81B8093ED0D0E946B5580918F
:10A59000E800982F9E7F1CC08091A51B813AE9F4AA
:10A5A0008091E800877F8093E8008091ED0D809393
:10A5B000F1008091E800982F9E7F9093E8008F77BC
:10A5C0008093E8000E9476558091E800982F9B7F49
:10A5D0009093E8008F778093E800DF91CF91089502
:10A5E00082E061EC46E30E94F15480E00E941B553A
:10A5F00081E060EC46E30E94F154E0EFF0E08081FE
:10A6000084608083089581E00E941B5508959330F3
:10A61000C1F0943030F4913051F0923009F03BC0E9
:10A620000BC0913271F1923209F035C02FC022E196
:10A6300030E08FEB94E033C029E230E081ED94E02C
:10A640002EC0813061F0813028F0823071F083308B
:10A6500011F510C08AEF94E0FC01249104C08EEF44
:10A6600094E0FC01249130E01AC084E295E0FC0102
:10A670002491F9CFECE4F5E0249130E08FE29CE105
:10A680000EC029E030E083EE94E009C024E330E01E
:10A690008BE894E004C020E030E080E090E0FA0134
:10A6A00091838083C9010895DF93CF9300D0CDB704
:10A6B000DEB7E5EAFBE18091F10081934BE1ED3AF1
:10A6C000F407C9F79091A51B8091A61B853009F46A
:10A6D00074C0863040F48130B9F1813070F083303D
:10A6E00009F033C131C0883009F4F6C0893009F46B
:10A6F00013C1863009F029C179C0903821F0923811
:10A7000009F023C108C080919E1B882311F083E0CB
:10A7100011C081E00FC08091A91B8093E900809156
:10A72000EB0090E025E0969587952A95E1F78170FA
:10A730001092E9009091E800977F9093E800809351
:10A74000F1001092F100D3C0923009F0FEC0909158
:10A75000A71B992331F59091A91B937009F4F7C0B9
:10A760009093E9002091EB0020FF1BC08130A1F401
:10A770008091EB0080618093EB0021E030E002C02B
:10A78000220F331F9A95E2F72093EA001092EA0015
:10A790008091EB00886003C08091EB008062809321
:10A7A000EB001092E9008091E800877F8093E80039
:10A7B0008091E800982F9E7FA9C0992309F0C5C019
:10A7C0008091E800877F8093E8008091E800982FCF
:10A7D0009E7F9093E8008F778093E8000E946B55EE
:10A7E0008091A71B80688093E300B1C0905892309D
:10A7F00008F0ABC08091A71B9091A81B6091A91B8A
:10A80000AE014F5F5F4F0E940753009709F49FC04E
:10A810002091E800277F2093E8002091AB1B309126
:10A82000AC1B8217930720F49093AC1B8093AB1B57
:10A830002091A71B3091A81B80E041C08091E800C7
:10A8400082FD60C08091E80080FFF8CF19C0E981E7
:10A85000FA8143E02330340731F44191FA83E983EC
:10A860004093F10008C0AF014F5F5F4F5A834983A7
:10A87000E491E093F10001979093AC1B8093AB1BA4
:10A880008091AB1B9091AC1B009739F04091F20086
:10A890005091F30048305105D0F24091F2005091B0
:10A8A000F30080E04830510509F481E09091E80020
:10A8B000492F4E7F4093E8009F779093E8004091A6
:10A8C000AB1B5091AC1B4115510509F0BBCF882340
:10A8D000B9F00E946B550BC09038B9F58091E80033
:10A8E000877F8093E80080919F1B8093F100809187
:10A8F000E800982F9E7F9093E8008F778093E80080
:10A900000E9476558091E800982F9B7F9093E800F5
:10A910008F778093E8001BC09923B9F49091A71B0F
:10A920009230A8F48091E800877F8093E8009093AC
:10A930009F1B8091E800982F9E7F9093E8008F776F
:10A940008093E8000E94F05202C00E945E52809103
:10A95000E80083FF0AC08091EB0080628093EB00E7
:10A960008091E800877F8093E8000F900F90CF914F
:10A97000DF9108959C019091E1009B7F9093E1000D
:10A980008091E80085FD1DC08091A41B882311F4EF
:10A9900082E008958091EB0085FF02C081E0089578
:10A9A0008091E10082FFECCF8091E1008B7F80936A
:10A9B000E1002115310511F483E008952150304064
:10A9C000DFCF80E00895AC0128E030E080E003C0F4
:10A9D0008F5F220F331F24173507D0F38295807FB6
:10A9E00008958093E9008091EB0081608093EB00F3
:10A9F0001092ED006093EC004093ED008091EE002A
:10AA0000881F8827881F08951092F40080E08093A3
:10AA1000E9001092F0001092E8009091ED009D7F07
:10AA20009093ED009091EB009E7F9093EB008F5FF1
:10AA3000873069F708952091A01B3091A11B211543
:10AA4000310501F19091E9001092A11B1092A01B19
:10AA50001092A31B1092A21B882341F081E08093E7
:10AA6000E9008091F00084608093F00082E08093A0
:10AA7000E9008091F0008E7F8093F000892F837031
:10AA80008093E90008950F931F93CF93DF938C0178
:10AA9000EB0184E690E00E94BA548823B9F4202F99
:10AAA000312FF90108C09091E80095FF06C0909100
:10AAB000F100919321972097B1F79091E800292F09
:10AAC0002B7F2093E8009F779093E800DF91CF9150
:10AAD0001F910F91089580E197E22091E80020FDF9
:10AAE00004C0009711F00197F8CF089580E197E234
:10AAF0002091E80022FD04C0009711F00197F8CFE3
:10AB00000895EF92FF920F931F93CF93DF93082F37
:10AB1000192F8091AB1B9091AC1BE62EE7017E01B3
:10AB2000F72EE7018E159F0508F4EC0180E023C0A5
:10AB30000E946B5507C0F80181918F018093F1004D
:10AB4000219739F08091F2009091F30088309105BF
:10AB500090F32091F2003091F30080E0283031052D
:10AB600009F481E09091E800292F2E7F2093E800DE
:10AB70009F779093E800209721F09091E80092FF52
:10AB8000D7CF9091E80092FF02C085E010C08823E3
:10AB900059F00E946B558091E800982F9E7F90930A
:10ABA000E8008F778093E8000E94765580E0DF917F
:10ABB000CF911F910F91FF90EF900895CF92DF9268
:10ABC000EF92FF920F931F93CF93DF938C01EB01D2
:10ABD00084E690E00E94BA54F82E882309F057C00A
:10ABE000CC24DD2408C0F80181918F018093F1000D
:10ABF0000894C11CD11CCC16DD0620F48091E8001D
:10AC000085FDF1CFC114D10411F00E94B49580915B
:10AC1000F4008B7F8093F4008091E800982F9E7F52
:10AC20009093E8008F778093E800CC19DD0949F410
:10AC3000C114D10461F1FFE3CF22DD24C114D1049A
:10AC400031F580E290E00E94BA54E82E882341F268
:10AC500083E0E816C9F41093A11B0093A01BD093C6
:10AC6000A31BC093A21B81E08093E9008091F000B8
:10AC70008B7F8093F00082E08093E9008091F00068
:10AC800081608093F00008C00E94945701C0EF2CAF
:10AC900081E00E941B55FE2C8F2DDF91CF911F91DB
:10ACA0000F91FF90EF90DF90CF9008950E94035393
:10ACB000E0EEF0E0808181608083E8EDF0E080816B
:10ACC0008062808319BCE7EDF0E080818E7F808315
:10ACD0001092A41B08950E94255781E08093A41B25
:10ACE0000E94B35108958091D90081709091A41B66
:10ACF000992329F4882319F00E946B5608959091A6
:10AD0000A41B992321F0882311F40E94565608951C
:10AD10001F920F920FB60F920BB60F9211242F9322
:10AD20003F934F935F936F937F938F939F93AF93D3
:10AD3000BF93EF93FF938091DA0080FF0BC0809167
:10AD4000D80080FF07C08091DA008E7F8093DA0000
:10AD50000E9473568091E10080FF19C08091E2004B
:10AD600080FF15C08091E1008E7F8093E10080918B
:10AD7000E2008E7F8093E2008091E2008061809308
:10AD8000E2008091D80080628093D80019BC809145
:10AD9000E10084FF20C08091E20084FF1CC08CE0B1
:10ADA00089BD89B5826089BD09B400FEFDCF80915F
:10ADB000D8008F7D8093D8008091E1008F7E8093B2
:10ADC000E1008091E2008F7E8093E2008091E200BA
:10ADD00081608093E2008091E10083FF23C0809135
:10ADE000E20083FF1FC08091E100877F8093E10034
:10ADF00010929F1B8091E1008E7F8093E1008091F3
:10AE0000E2008E7F8093E2008091E2008061809377
:10AE1000E2000E94045580E060E042E00E94F154AC
:10AE20000E94B751FF91EF91BF91AF919F918F9188
:10AE30007F916F915F914F913F912F910F900BBE3A
:10AE40000F900FBE0F901F9018958091D8008C7FA7
:10AE50008093D8001092E2001092DA001092E10084
:10AE60001092A41B10929F1B10929E1B80E00E94C8
:10AE70001B558CE089BD89B5826089BD09B400FE8F
:10AE8000FDCF8091D800982F9F779093D80080684D
:10AE90008093D8008091D70081608093D700809103
:10AEA000D8008F7D8093D8008091E0008B7F8093C5
:10AEB000E0008091D80081608093D8008091E0000C
:10AEC0008E7F8093E0008091E20081608093E200B9
:10AED0008091E20088608093E20008958091A41B35
:10AEE000882311F00E9403538091E00081608093D9
:10AEF000E0008091D8008C7F8093D8001092E2000F
:10AF00001092DA001092E1001092A41B10929F1B85
:10AF10008091D8008F778093D80019BC8091D80099
:10AF20008F7E8093D80008950E946E57E7EDF0E081
:10AF30008081806880830E942557E8EDF0E0808161
:10AF40008061808308950F931F938091A41B8823B1
:10AF500081F01091E9001092E9008091E80083FFF0
:10AF600005C00FB7F8940E9454530FBF137010938D
:10AF7000E9001F910F910895EF92FF920F931F9395
:10AF800090E0880F991F860F911DFC01EE0FFF1FA7
:10AF9000EE0FFF1FEC5EFF4EE080F1800281138117
:10AFA000FA01E082F1820283138388589F4EFC01EC
:10AFB0008081F90180831F910F91FF90EF90089598
:10AFC0009BE1899FC001112440962DE0629FB00152
:10AFD0001124860F971F61E040E221E00E94FA29C8
:10AFE000882309F481E00895AF92BF92CF92DF9257
:10AFF000EF92FF920F931F93B82EA62E2BE1829F04
:10B00000900111242C5E3F4F8DE0689FC0011124F8
:10B01000820F931F40E050E0BA0100E21EEF2FE6DE
:10B020003AE40F2EF0E0CF2EF0E8DF2EFBEBEF2E10
:10B03000F5E4FF2EF02D0E94172B7B018C018B2D48
:10B040006A2D0E94E057282F30E0B901882777FD4C
:10B050008095982F0E9425C19B01AC01C801B701C2
:10B060000E94D9C11F910F91FF90EF90DF90CF9078
:10B07000BF90AF900895BF92CF92DF92EF92FF9270
:10B080000F931F93082F162F0E94E057B82E2BE125
:10B09000029F900111242C5E3F4F8DE0189FC0014C
:10B0A0001124820F931F40E050E0BA0100E21EEF2E
:10B0B0002FE63AE40F2EF0E0CF2EF0E8DF2EFBEB88
:10B0C000EF2EF5E4FF2EF02D0E94172B7B018C0153
:10B0D00020E030E040E752E40E9486C087FD0AC0CD
:10B0E000C801B70120E030E64AEE56E40E94D5C11F
:10B0F000181654F40F2EF0E0EF2EF0E8FF2EFBEBC5
:10B100000F2FF5E41F2FF02D2B2D30E0B9018827EC
:10B1100077FD8095982F0E9425C1A80197010E9474
:10B12000D9C11F910F91FF90EF90DF90CF90BF900A
:10B130000895EF92FF920F931F93E82FF0E0EE0F28
:10B14000FF1FE60FF11DEE0FFF1FEE0FFF1FE35570
:10B15000F44EE080F180028113810E943B589B01F4
:10B16000AC01C801B7010E948AC07B018C01802F0D
:10B17000880F812F881F8F3F09F1C801B70120E098
:10B1800030E0A9010E9486C087FD18C0C801B70140
:10B1900020E030E040E85FE30E94D5C118162CF4AF
:10B1A00060E070E088EC92E40DC0C801B70120E0D7
:10B1B00030E048EC52E40E94D9C104C060E070E085
:10B1C00080E090E01F910F91FF90EF900895AF9273
:10B1D000BF92CF92DF92EF92FF920F931F93DF9374
:10B1E000CF9300D000D0CDB7DEB7082F162F8091B7
:10B1F000661B7E010894E11CF11C8330F9F080E0AD
:10B2000090E0DC0189839A83AB83BC836BE1069F6A
:10B21000B0011124685E7F4F8DE01802C001112437
:10B22000680F791FC7010E944F2A80E090E8ABE3C6
:10B23000B5E489839A83AB83BC8326C0802F0E94A8
:10B2400016605B016C01802F612F0E943B58A601A4
:10B2500095010E94D9C120E030E048EC52E40E9400
:10B260008AC069837A838B839C836BE1069FB001DC
:10B270001124685E7F4F8DE01802C0011124680F11
:10B28000791FC7010E944F2A59814A813B812C8135
:10B29000652F742F832F922F0F900F900F900F9088
:10B2A000CF91DF911F910F91FF90EF90DF90CF90A2
:10B2B000BF90AF9008950F931F93CF93DF93082F04
:10B2C00010E0C62FDD27C7FDD0950E94E7589B01EF
:10B2D000AC01000F111F0C0F1D1FC801880F991F13
:10B2E000880F991FFC01E355F44E2083318342837C
:10B2F00053838C5E9F4EFC01108211821282138256
:10B3000008581F4EF8011082DF91CF911F910F91C5
:10B3100008952F923F924F925F926F927F928F92F9
:10B320009F92AF92BF92CF92DF92EF92FF920F93D4
:10B330001F93DF93CF93CDB7DEB72A970FB6F8945C
:10B34000DEBF0FBECDBF8D836E834A013901170169
:10B350002801AF82B886C986DA86FA01E080F180DA
:10B3600002811381F9016081718182819381A80139
:10B3700097010E9421C0D62EC72EB82EA92EC20139
:10B38000B101D601F5012B2F3A2F4F2F5E2F0E94CE
:10B39000D9C19B01AC01C801B7010E9422C0F401D0
:10B3A00060837183828393836F81788589859A8591
:10B3B000D601F5012B2F3A2F4F2F5E2F0E94D9C1B6
:10B3C0009B01AC01C801B7010E9422C0B62EC72E56
:10B3D000D82EE92E862F9C2DAD2DBE2DF301808316
:10B3E0009183A283B3838D816E810E94E057282FC1
:10B3F00030E0B901882777FD8095982F0E9425C1FC
:10B400009B01AC016B2D7C2D8D2D9E2D0E948AC041
:10B4100069837A838B839C836BE1FD81F69FB00106
:10B4200011246C5E7F4F8DE02E81289FC001112476
:10B43000680F791FCE0101960E94542A2A960FB6F2
:10B44000F894DEBF0FBECDBFCF91DF911F910F915A
:10B45000FF90EF90DF90CF90BF90AF909F908F9034
:10B460007F906F905F904F903F902F9008952F9214
:10B470003F924F925F926F927F928F929F92AF9284
:10B48000BF92CF92DF92EF92FF920F931F93DF93C1
:10B49000CF93CDB7DEB72E970FB6F894DEBF0FBEB1
:10B4A000CDBFA82EB62E442E882E99246623E9F40B
:10B4B000C0909504D0909604E0909704F090980482
:10B4C00086EA92E040E050E068E472EC00E010E0D0
:10B4D00028E432E40E94172B7B018C01F40123E065
:10B4E000EE0FFF1F2A95E1F71FC0C0909904D0907E
:10B4F0009A04E0909B04F0909C048AEA92E040E079
:10B5000050E068E472EC00E010E028E432E40E94CD
:10B51000172B7B018C01F401EE0FFF1FEB0DF11DCA
:10B52000EE0FFF1FEE0FFF1FEC5EFF4E608171817B
:10B53000828193810E9425C19B01AC01C801B701A2
:10B540000E94D9C1962EC72ED82EE92E642D70E008
:10B5500080E090E00E9423C19B01AC01692D7C2D0D
:10B560008D2D9E2D0E948AC0D62EC72E982E892EF4
:10B570002A2C33242B2D30E03A872987C101880FEC
:10B58000991F820F931F9C01220F331F220F331F1D
:10B59000F901EC5EFF4E10821182128213828858EC
:10B5A0009F4EDC011C922355344EF901608171815C
:10B5B00082819381D601F4012B2F3A2F4F2F5E2FDA
:10B5C0000E9421C0262F372F482F592F29833A83D5
:10B5D0004B835C8320E030E0A9010E9486C0882371
:10B5E0003CF480E090E0DC0189839A83AB83BC83E8
:10B5F0008A2D6B2D0E943B582B013C016D837E836D
:10B600008F8398878A2D6B2D0E9416607B018C0199
:10B61000A6019401652F7C2D832F982D20E030E02A
:10B6200040E050E40E9486C088230CF04BC0898122
:10B630009A81AB81BC818B879C87AD87BE87C30114
:10B64000B2012FE832EC45EF5CE30E94D9C19B01C7
:10B65000AC016B857C858D859E850E9486C0181601
:10B66000CCF0C801B70120E030E040E450E40E9493
:10B6700086C018163CF5C801B7012D813E814F8167
:10B6800058850E94D9C120E030E048EC52E40E9485
:10B690008AC014C0C801B70120E030E040E450E4A3
:10B6A0000E9486C0181674F06B857C858D859E85FA
:10B6B0002DEC3CEC4CE45FE30E94D9C169837A83B2
:10B6C0008B839C8369817A818B819C812D813E81D2
:10B6D0004F8158850E94D5C1181654F5C801B7018D
:10B6E00020E030E042EC52E40E94D5C19E012B5F85
:10B6F0003F4FAE014F5F5F4F88231CF08A2D6B2DAB
:10B7000037C08A2D6B2D0F2EF6E6EF2EF6E6FF2EB4
:10B71000F6EE0F2FFEE31F2FF02D0F2EF3E3AF2ECB
:10B72000F3E3BF2EF3E7CF2EFFE3DF2EF02D34C07F
:10B73000A6019401652F7C2D832F982D20E030E009
:10B7400040E050EC0E94D5C1181644F5C801B7017D
:10B7500020E030E042EC52E40E94D5C18823F4F0AE
:10B760008A2D6B2DAE014F5F5F4F9E012B5F3F4FC8
:10B770000F2EFDECEF2EFCECFF2EFCE40F2FFEE372
:10B780001F2FF02D0F2EFDECAF2EFCECBF2EFCE496
:10B79000CF2EFFE3DF2EF02D0E948959F101EE0F2D
:10B7A000FF1FA985BA85EA0FFB1FEE0FFF1FEE0FE3
:10B7B000FF1FE355F44E89819A81AB81BC81808360
:10B7C0009183A283B3832E960FB6F894DEBF0FBE8B
:10B7D000CDBFCF91DF911F910F91FF90EF90DF9040
:10B7E000CF90BF90AF909F908F907F906F905F9021
:10B7F0004F903F902F9008954F925F927F928F923B
:10B800009F92AF92BF92CF92DF92EF92FF920F93EF
:10B810001F93DF93CF930F92CDB7DEB7823050F4F2
:10B820005DEAE52E5BE1F52E48E1842E912C44245F
:10B8300055242EC08430C1F5F3CFF80180818823D0
:10B8400059F0872D622F4CE329830E94375AC60195
:10B85000B5010E944F2A29812F5F0F5F1F4F84E09F
:10B8600090E0C80ED91EEDE0F0E0AE0EBF1E223013
:10B8700021F70894411C511C88E090E0E80EF91E65
:10B88000EBE1F0E08E0E9F1EFCE04F16510451F0EC
:10B89000742C8201000F111F08581F4E54016701BC
:10B8A00020E0CBCF109292100F90CF91DF911F919B
:10B8B0000F91FF90EF90DF90CF90BF90AF909F904F
:10B8C0008F907F905F904F90089580919210882381
:10B8D00009F58091661B8330E9F485EA9DE560E017
:10B8E00070E00E94BA5F8091A30D9091A40DA09189
:10B8F000A50DB091A60D8093741090937510A09330
:10B900007610B0937710109290101092911081E001
:10B910008093921008955F926F927F928F929F9280
:10B92000AF92BF92CF92DF92EF92FF920F931F934D
:10B93000CF93DF938091A30D9091A40DA091A50DBD
:10B94000B091A60D20917410309175104091761031
:10B95000509177107C018D01E21AF30A040B150B4C
:10B96000A8019701243631054105510508F468C046
:10B970008093741090937510A0937610B093771005
:10B980000E94655C80919210882309F459C080E37D
:10B990009DE560E070E00E94BA5F809190108F5F3B
:10B9A000809390108C3308F44BC0109290108091CB
:10B9B00091108F5F80939110893610F4EE2404C0AB
:10B9C00010929110EE24E394EDEACE2EEBE1DE2E00
:10B9D00078E1672E712CC0E0D0E028C0F8014081EA
:10B9E000442351F0852D6F2D0E94375AEE2021F00F
:10B9F000C501B4010E944F2AF3940F5F1F4F84E0EA
:10BA000090E0A80EB91EEDE0F0E08E0E9F1EF2E071
:10BA1000FF1621F7219608E010E0C00ED11E8BE141
:10BA200090E0680E791ECC30D10551F05C2E8E016D
:10BA3000000F111F08581F4E43015601FF24CECF9F
:10BA4000DF91CF911F910F91FF90EF90DF90CF90FA
:10BA5000BF90AF909F908F907F906F905F90089570
:10BA6000AF92BF92CF92DF92EF92FF921F93CF934C
:10BA7000DF93182F662319F421E030E05BC06EE0FD
:10BA80000E94CB6994FF26C0E12EFF24E70183E0EA
:10BA9000CC0FDD1F8A95E1F7CC5EDF4EA880B98020
:10BAA000CA80DB80812F65E00E94BE6AAA2797FDCD
:10BAB000A095BA2F8A0D9B1DAC1DBD1D888399834F
:10BAC000AA83BB83F701EE0FFF1FE858FF4E80816A
:10BAD0008F5F8083812F6CE00E94CB6994FF28C028
:10BAE000C12FD0E0CC0FDD1F7E01EE0CFF1CEE0C51
:10BAF000FF1C88E190E1E80EF91EF701A080B180FB
:10BB0000C280D380812F62E00E94BE6AAA2797FD7F
:10BB1000A095BA2F8A0D9B1DAC1DBD1DF70180831A
:10BB20009183A283B383C858DF4E89818F5F898355
:10BB300020E030E0C901DF91CF911F91FF90EF909D
:10BB4000DF90CF90BF90AF9008955F926F927F92F9
:10BB50008F929F92AF92BF92CF92DF92EF92FF921D
:10BB60000F931F93CF93DF93A82E562E8BE19A2D20
:10BB7000989FE00111246896CA2CDD24C60143E099
:10BB8000880F991F4A95E1F73DEA832E3BE1932EFA
:10BB9000880E991E24E1622E20E1722E680E791E15
:10BBA000CC0CDD1CE8E7F0E1CE0EDF1EBB24CE019D
:10BBB0000E94D72A7B018C0120E030E040E752E46C
:10BBC0000E9486C087FD0AC0C801B70120E030E6A8
:10BBD0004AEE56E40E94D5C118169CF4552059F43B
:10BBE0000F2EF0E0EF2EF0E8FF2EFBE30F2FF5E431
:10BBF0001F2FF02D06C08A2D6B2D0E94E7587B0168
:10BC00008C01F401E192F192019311934F01F30140
:10BC100011921192119211923F01F60111926F014E
:10BC2000B3942D96F2E0BF1611F680E090E0DF911C
:10BC3000CF911F910F91FF90EF90DF90CF90BF9029
:10BC4000AF909F908F907F906F905F9008958FEF4F
:10BC500080930D1C8FE780930E1C80930F1C08951A
:10BC6000FC018FEF80838FE7818382830895CF93D8
:10BC7000DF93C82FD0E0CC57DF4F84E0CC0FDD1F1F
:10BC80008A95E1F7CE0182579F4F0E94D367292FF3
:10BC900022952F7030E02230310511F090E00AC07B
:10BCA000CE018A579D4F0E94D36790E08F708F30EE
:10BCB00009F091E0892FDF91CF9108959091661B53
:10BCC000923010F480E0089590E024E0880F991FEE
:10BCD0002A95E1F78A53954F0E94D367892F9111D6
:10BCE00081E008951F93CF93DF93C4ECDAE010E076
:10BCF00080E00E945E5E882371F0CE010E94D367CF
:10BD000084FF09C0812F0E94375E882329F01F5FBE
:10BD10006096123069F781E0DF91CF911F9108950D
:10BD20000F931F93CF93DF93082F0E94725E882397
:10BD3000D9F010E015C0812F60E80E94CB69EC01BA
:10BD4000812F63E80E94CB69C070DE702EE0C030A6
:10BD5000D20729F48F7090708F30910529F01F5F02
:10BD6000101748F381E001C080E0DF91CF911F916F
:10BD70000F91089590E034E0880F991F3A95E1F70C
:10BD80008C53954F0E94D36785FD02C081E00895D2
:10BD90008CE00E94905E811181E00895CF92DF9245
:10BDA000EF92FF920F931F93CF93DF93EC017B01F0
:10BDB00080E00E94BA5E882341F080E00E945E5ECF
:10BDC000882319F081E090E002C080E090E0182F15
:10BDD00000E0802F612FA701FE0109956C0111235E
:10BDE000E1F00097C9F40023B9F480E00E94375EC7
:10BDF000182F882391F081E00E94BA5E882341F0D9
:10BE000081E00E945E5E882319F081E090E002C02C
:10BE100080E090E0182F01C011E00F5F023019F0B0
:10BE2000C114D104B1F2C601DF91CF911F910F91DE
:10BE3000FF90EF90DF90CF900895CF92DF92EF9236
:10BE4000FF921F93CF93DF93182FEB0160E80E94BE
:10BE5000CB696C01812F61E80E94CB697C01812F45
:10BE600063E80E94CB699883960165E03695279533
:10BE70006A95E1F72077382F3F70232B298354E010
:10BE8000969587955A95E1F78F70970145E036951D
:10BE900027954A95E1F7922F9077892B8A83DF9136
:10BEA000CF911F91FF90EF90DF90CF900895EF9288
:10BEB000FF920F931F938091A30D9091A40DA091D9
:10BEC000A50DB091A60D2091931030919410409142
:10BED0009510509196107C018D01E21AF30A040B23
:10BEE000150BA80197012B30310541055105E8F0EC
:10BEF0008093931090939410A0939510B093961004
:10BF00008091621B0E94905E882349F48FEF80939A
:10BF10000D1C8FE780930E1C80930F1C06C0809130
:10BF2000621B6DE07CE10E941D5F1F910F91FF90ED
:10BF3000EF9008951F93182F8091661B8230B8F000
:10BF4000812F6FE00E94BA69009789F0812F67E81E
:10BF50000E94CB69009759F0812F61E80E94CB695C
:10BF600080E092959F70191719F481E001C080E07C
:10BF70001F9108958F929F92AF92BF92CF92DF92BE
:10BF8000EF92FF920F931F93DF93CF9300D00F9206
:10BF9000CDB7DEB76C015B010E94725E882341F071
:10BFA00080E00E949A5F882319F001E010E002C04F
:10BFB00000E010E010E07E010894E11CF11C812FEC
:10BFC000602FA501F60109954C010023C1F00097EF
:10BFD000B1F41B30A1F0812F60E80E94CB6997FF7C
:10BFE0000DC0812FB7010E941D5F8A818F3730F409
:10BFF000812F8F5F0E949A5F082F01C000E01F5FB2
:10C000001C3019F081149104D1F2C4010F900F90EB
:10C010000F90CF91DF911F910F91FF90EF90DF90E4
:10C02000CF90BF90AF909F908F9008952F923F92A6
:10C030004F925F926F927F928F929F92AF92BF9238
:10C04000CF92DF92EF92FF920F931F93DF93CF93E4
:10C0500000D000D0CDB7DEB7182F062F662381F4AD
:10C060006EE00E94CB6994FF3CC1812F90E00E945A
:10C07000B86A6B017C01812F90E00E94046B0FC0B5
:10C080006CE00E94CB6994FF2CC1812F90E00E944C
:10C09000B26A6B017C01812F90E00E94FE6A2B0145
:10C0A0003C012BE1129F900111242F5E3F4F8DE048
:10C0B000089FC0011124820F931F6CE044E22CE022
:10C0C0000E94FA29082FC701B60120E030E040E1C4
:10C0D00051E40E9486C088230CF41EC1C701B6013A
:10C0E00020E030E048E851E40E9486C0882314F440
:10C0F00011E00FC0C701B60120E030E040EF51E48D
:10C100000E9486C0182F111F1127111F83E0811B69
:10C11000182F083189F0043219F00C30C1F522C013
:10C12000C701B60120E030E048ED51E40E94D5C1DE
:10C1300088236CF113E02BC0C701B60120E030E08A
:10C1400040E951E40E94D5C188230CF1C701B60132
:10C1500020E030E040EE51E40E9486C01816BCF0AA
:10C1600012E015C0C701B60120E030E040E151E423
:10C170000E94D5C188235CF0C701B60120E030E001
:10C1800040E651E40E9486C018160CF011E0212F01
:10C1900030E0B901882777FD8095982F0E9425C14E
:10C1A0004B015C01C701B601A50194010E948AC040
:10C1B000062F372E282E9983C301B2019F77A50140
:10C1C00094010E948AC0862EA72EC82E192F2DEC0E
:10C1D0003CEC40E051E40E94D5C188232CF08FE074
:10C1E00097E09C838B8315C0682D7A2D8C2D912F21
:10C1F00020E030E048EB50E40E94D5C187FF05C045
:10C20000A7E6B7E0BC83AB8304C0EBE3F7E0FC83B5
:10C21000EB838B809C80AA24BB2414E6D401CD90B0
:10C22000DD90ED90FC90C701B6017980202F332D71
:10C23000422D572D0E9486C018160CF447C0AA2024
:10C2400029F460E070E088EC92E44FC0612F70E068
:10C2500080E090E00E9423C1162F872E982E9A83AB
:10C26000C701B601A1013981402E552E642E732ECF
:10C27000A30192010E9421C020E030E040E251E49D
:10C280000E94D9C12B013C01F5013197EE0FFF1F30
:10C29000EE0FFF1F8B819C81E80FF91FC701B601CC
:10C2A00020813181428153810E9421C09B01AC01D8
:10C2B000C301B2010E948AC09B01AC01CA80612FF8
:10C2C000782D892D9C2D0E9422C00FC00894A11C9E
:10C2D000B11CA4E0B0E08A0E9B1E112311F01A508D
:10C2E0009DCF60E070E080E090E00F900F900F90A5
:10C2F0000F90CF91DF911F910F91FF90EF90DF9002
:10C30000CF90BF90AF909F908F907F906F905F90F5
:10C310004F903F902F90089510E0FBCE8091671BC7
:10C32000813039F48091F21A882319F01092671B3A
:10C3300008950E94C20508958091671B882341F4E7
:10C340008091F31A882321F081E08093671B089580
:10C350000E94C20508958091621B6091671B0E9434
:10C360005B5908958091621B8093F11A6EE00E94E0
:10C37000CB69929591709093F21A8091621B6CE058
:10C380000E94CB69929591709093F31A992321F0B2
:10C390008091F21A882319F01092671B089581E0AA
:10C3A0008093671B0895AF92BF92CF92DF92EF9276
:10C3B000FF920F931F93DF93CF9300D000D000D054
:10C3C000CDB7DEB79091621B8091F11A981711F0EA
:10C3D0000E94B2618AE060E00E949F04E091671BC6
:10C3E000F0E0EE0FFF1FEF50F54E838194810E9425
:10C3F000550682E160E00E949F048091621B90E0FC
:10C40000019663E977E042E00E94580684E060E02C
:10C410000E949F046091671BE62FF0E0EF50F54EFD
:10C420008181882309F457C08091621B0E94F457D0
:10C4300020E030E040E752E40E948AC08B01B82E31
:10C44000A92E9501712F832F922F48E957E026E0FE
:10C450000E949D0684E061E00E949F048091671B1A
:10C46000E091621BF0E0EE0FFF1FE80FF11DEE0FF1
:10C47000FF1FEE0FFF1FE355F44E60817181828133
:10C48000938120E030E040E752E40E948AC06B01D3
:10C490007C017D2D9F2D48E957E026E00E949D06F6
:10C4A0008BE061E00E949F046C2D7D2D8E2D9F2DD1
:10C4B00020E030E048EC52E40E94D9C1F501202F81
:10C4C000312F4F2F5E2F0E948AC04EE957E025E0A2
:10C4D0000E949D0614C087E392E00E94550684E006
:10C4E00061E00E949F0487E392E00E9455068BE082
:10C4F00061E00E949F0488E392E00E9455069091BB
:10C50000671B8091621B992349F40E94046B7B0195
:10C510008C01C090F81AD090F91A09C090E00E94DE
:10C52000FE6A7B018C01C090FA1AD090FB1A80E061
:10C5300062E00E949F04C6010E94550684E062E00A
:10C540000E949F04E091671BF0E0EF50F54E81815F
:10C55000882309F470C0C801B70148E957E026E014
:10C560000E949D068EE062E00E949F048091621B03
:10C570006091671B0E9416604EE957E025E00E941B
:10C580009D068091621B6091671BAE014E5F5F4FFD
:10C590009E012F5F3F4F0E94BC578091671B8823ED
:10C5A00059F4C0909504D0909604E0909704F090D0
:10C5B000980486EA92E00AC0C0909904D0909A0448
:10C5C000E0909B04F0909C048AEA92E040E050E006
:10C5D00068E472EC00E010E028E432E40E94172BDB
:10C5E0007B018C016A817B818C819D810E9425C1A8
:10C5F0009B01AC01C801B7010E94D9C1F62E072FDB
:10C60000182F84E063E09E830E949F049E816F2D1B
:10C61000702F812F48E957E026E00E949D068BE0AD
:10C6200063E00E949F04898190E064EA77E042E041
:10C630000E9458061CC087E392E00E9455068EE0D7
:10C6400062E00E949F0488E392E00E94550684E025
:10C6500063E00E949F0487E392E00E9455068BE00E
:10C6600063E00E949F048BE392E00E9455062696A9
:10C670000FB6F894DEBF0FBECDBFCF91DF911F91F3
:10C680000F91FF90EF90DF90CF90BF90AF90089503
:10C69000CF92DF92EF92FF920F931F93CF93DF938E
:10C6A00084EF91E00E9489050E94B261CCEDDAE14D
:10C6B000CE0160E270E044E150E00E9459C48EE493
:10C6C0000E949B12BC01FC0101900020E9F7319708
:10C6D000E81BF90BCE01AF010E9450C44AE3F42ECF
:10C6E000F092DF1A8FE30E949B12BC01FC010190C3
:10C6F0000020E9F73197E81BF90B8E01015F1F4F0E
:10C70000C801AF010E9450C480E090E00E9443063F
:10C71000CE0160E270E044E150E00E9459C485E738
:10C720000E949B12BC01FC0101900020E9F73197A7
:10C73000E81BF90BCE01AF010E9450C4F092DF1A42
:10C7400035E2E32EE092EC1A81E090E00E9443068D
:10C75000CE0160E270E044E150E00E9459C4F092E2
:10C76000DF1A81E48093E61AE092EF1A82E090E00B
:10C770000E944306CE0160E270E044E150E00E9476
:10C7800059C484E70E949B12BC01FC010190002067
:10C79000E9F73197E81BF90BCE01AF010E9450C4B5
:10C7A000F092DF1A84E20E949B12BC01FC0101900E
:10C7B0000020E9F73197E81BF90BC801AF010E948F
:10C7C00050C483E090E00E94430687E80E949B12D9
:10C7D0009093F51A8093F41A88E80E949B12909324
:10C7E000F71A8093F61A85E30E949B129093F91A28
:10C7F0008093F81A86E30E949B129093FB1A809311
:10C80000FA1A0E94D361DF91CF911F910F91FF908F
:10C81000EF90DF90CF900895E8ECF7E008C020811A
:10C8200031812817390711F462830895339627E080
:10C83000EA3DF207A1F708956093981091E0909374
:10C84000971083FD02C090E401C090E68770892BA9
:10C8500098E10FB6F894A895909360000FBE80936E
:10C86000600078944111FFCF08951F93CF93DF9319
:10C87000182FC0ECD7E004C0E991F991812F0995F8
:10C8800087E0C83CD807C1F7DF91CF911F91089589
:10C8900080919710882319F4A8950E94DB9508953C
:10C8A0000F931F93CF93DF9384B780932E1C98E14F
:10C8B0000FB6F89490936000109260000FBE20E0D5
:10C8C00090E80FB6F89490936100209361000FBE3A
:10C8D00080FF06C08FE493EC0197F1F700C00000E1
:10C8E00018E101E60FB6F894A895109360000FBE0A
:10C8F0000093600078940E9438650E9400050E94B1
:10C900009F180E944D520E9495508CE00E943F0457
:10C910008FE39DE0A3E081509040A040E1F700C08C
:10C9200000008CE00E943F040E94AA090E94073A7E
:10C930000E946F130E94C5290E9411090E94E59070
:10C940000E949395129A129A14BE78940E948D6D4B
:10C950008EEB9AE161EF72E04EE150E00E94592ABD
:10C960000FB6F894A895109360000FBE0093600076
:10C970007894C8ECD7E007C08A81813019F4E88147
:10C98000F9810995239697E0CA3DD907A9F70E9436
:10C99000486482B1847082B98BB184708BB962971C
:10C9A000F2CF1F920F920FB60F920BB60F92112477
:10C9B0002F933F934F935F936F937F938F939F93A7
:10C9C000AF93BF93CF93DF93EF93FF9381E00E94E8
:10C9D000356480919810882319F4C0E0D0E008C035
:10C9E00083E094E065E570E00E94A46BC0E0D0EFC6
:10C9F00084B7877F84BF88E10FB6F8948093600086
:10CA0000109260000FBE0E94BE180E946E578FE306
:10CA10009DE0A3E081509040A040E1F700C00000FD
:10CA2000FE01099583FD03C020E030E002C020E054
:10CA300038E0613069F4B90160507E4F43FF03C0B4
:10CA4000B90160587D4F47705070462B572B04C07A
:10CA50004F785070422B532B9C012770307084E02C
:10CA6000220F331F8A95E1F7242B352BC901089536
:10CA7000209A2898089588E58CBD8DB581608DBD7C
:10CA8000289A089528980895CF92DF92EF92FF9206
:10CA90000F931F93CF93DF93EC01C0909D04D09030
:10CAA0009E04E0909F04F090A0048EEA92E040E0A3
:10CAB00050E068E472EC00E010E028E432E40E9408
:10CAC000172B6B017C01DF70BE0180E090E00E94BB
:10CAD00023C1A70196010E94D9C1DF91CF911F9177
:10CAE0000F91FF90EF90DF90CF900895CF92DF925B
:10CAF000EF92FF920F931F93CF93DF93EC01C090BF
:10CB00009904D0909A04E0909B04F0909C048AEAE7
:10CB100092E040E050E068E472EC00E010E028E4CD
:10CB200032E40E94172B6B017C01BE01882777FD40
:10CB30008095982F0E9425C19B01AC01C701B601C9
:10CB40000E94D9C1DF91CF911F910F91FF90EF907B
:10CB5000DF90CF900895CF92DF92EF92FF920F93E4
:10CB60001F93CF93DF93EC01C0909504D09096046F
:10CB7000E0909704F090980486EA92E040E050E05C
:10CB800068E472EC00E010E028E432E40E94172B25
:10CB90006B017C01BE01882777FD8095982F0E944C
:10CBA00025C19B01AC01C701B6010E94D9C1DF912B
:10CBB000CF911F910F91FF90EF90DF90CF9008954C
:10CBC000CF92DF92EF92FF920F931F93CF93DF9359
:10CBD000EC01C0909104D0909204E0909304F09006
:10CBE000940482EA92E040E050E068E472EC00E0F5
:10CBF00010E028E432E40E94172B6B017C01DF7007
:10CC0000BE0180E090E00E9423C1A70196010E942E
:10CC1000D9C1DF91CF911F910F91FF90EF90DF90DD
:10CC2000CF900895CF92DF92EF92FF920F931F93D0
:10CC3000CF93DF93EC01C0908D04D0908E04E090F0
:10CC40008F04F09090048EE992E040E050E068E4B8
:10CC500072EC00E010E028E432E40E94172B6B0134
:10CC60007C01DF70BE0180E090E00E9423C1A7013B
:10CC700096010E94D9C1DF91CF911F910F91FF9032
:10CC8000EF90DF90CF9008958F929F92AF92BF92D6
:10CC9000CF92DF92EF92FF920F931F934B015C01B3
:10CCA00020E030E0A9010E9486C088231CF460E0E7
:10CCB00070E02BC0C501B40120E030EF4FE755E430
:10CCC0000E94D5C118161CF46FEF7FE01EC0C09003
:10CCD0009D04D0909E04E0909F04F090A0048EEA02
:10CCE00092E040E050E068E472EC00E010E028E4FC
:10CCF00032E40E94172B9B01AC01C501B4010E94D4
:10CD00008AC00E943CC20E94F7C0CB011F910F91C4
:10CD1000FF90EF90DF90CF90BF90AF909F908F905B
:10CD200008958F929F92AF92BF92CF92DF92EF922F
:10CD3000FF920F931F934B015C01C0909904D09018
:10CD40009A04E0909B04F0909C048AEA92E040E010
:10CD500050E068E472EC00E010E028E432E40E9465
:10CD6000172B9B01AC01C501B4010E948AC00E942F
:10CD70003CC20E94F2C0CB011F910F91FF90EF9037
:10CD8000DF90CF90BF90AF909F908F9008958F923B
:10CD90009F92AF92BF92CF92DF92EF92FF920F934A
:10CDA0001F934B015C01C0909504D0909604E090D5
:10CDB0009704F090980486EA92E040E050E068E43E
:10CDC00072EC00E010E028E432E40E94172B9B0193
:10CDD000AC01C501B4010E948AC00E943CC20E94FD
:10CDE000F2C0CB011F910F91FF90EF90DF90CF9099
:10CDF000BF90AF909F908F9008958F929F92AF9227
:10CE0000BF92CF92DF92EF92FF920F931F934B014D
:10CE10005C0120E030E0A9010E9486C018161CF0D9
:10CE200060E070E02BC0C501B40120E030EF4FE7B7
:10CE300055E40E94D5C188231CF06FEF7FE01EC02F
:10CE4000C0909104D0909204E0909304F0909404E8
:10CE500082EA92E040E050E068E472EC00E010E02A
:10CE600028E432E40E94172B9B01AC01C501B401F8
:10CE70000E948AC00E943CC20E94F7C0CB011F9151
:10CE80000F91FF90EF90DF90CF90BF90AF909F9069
:10CE90008F9008958F929F92AF92BF92CF92DF9220
:10CEA000EF92FF920F931F934B015C0120E030E063
:10CEB000A9010E9486C018161CF060E070E02BC02B
:10CEC000C501B40120E030EF4FE755E40E94D5C121
:10CED00088231CF06FEF7FE01EC0C0908D04D090BF
:10CEE0008E04E0908F04F09090048EE992E040E090
:10CEF00050E068E472EC00E010E028E432E40E94C4
:10CF0000172B9B01AC01C501B4010E948AC00E948D
:10CF10003CC20E94F7C0CB011F910F91FF90EF9090
:10CF2000DF90CF90BF90AF909F908F9008951F9308
:10CF30001FB7F89488E58CBD8DB581608DBD289AAA
:10CF400082E094E00E943405289817FF01C078948D
:10CF50001F9108950E949767892F82958695817009
:10CF60000895EF92FF921F93CF93DF93EB017A0125
:10CF70001FB7F89428E52CBD2DB521602DBD289A4A
:10CF80009F770E943405CE01B7010E94370528988B
:10CF900017FF01C0789488819981DF91CF911F910B
:10CFA000FF90EF900895DF93CF9300D0CDB7DEB719
:10CFB000BE016F5F7F4F41E050E00E94B167898101
:10CFC0009A810F900F90CF91DF9108950E94126582
:10CFD0000E94D3670895462F90E061E050E00E94E0
:10CFE000E667009729F460E070E080E090E00DC013
:10CFF000BC0180E090E00E9423C19B01AC0160E095
:10D0000070EA8CE09AE40E948AC008956DE00E9464
:10D01000EB6708956CE00E94EB6708958F929F92F2
:10D02000AF92BF92CF92DF92EF92FF920F931F9336
:10D0300061E046E050E00E94E667BC017F7180E05D
:10D0400090E00E9423C10E9460C24B015C01C0902D
:10D05000C904D090CA04E090CB04F090CC048AEDCF
:10D0600092E040E050E068E472EC00E010E028E478
:10D0700032E40E94172B9B01AC01C501B4010E9450
:10D08000D9C11F910F91FF90EF90DF90CF90BF908B
:10D09000AF909F908F9008958F929F92AF92BF9282
:10D0A000CF92DF92EF92FF920F931F9361E043E0E4
:10D0B00050E00E94E667BC0180E090E00E9423C13E
:10D0C0000E9460C24B015C01C090C104D090C204B8
:10D0D000E090C304F090C40482ED92E040E050E0A0
:10D0E00068E472EC00E010E028E432E40E94172BC0
:10D0F0009B01AC01C501B4010E94D9C11F910F91E0
:10D10000FF90EF90DF90CF90BF90AF909F908F9067
:10D1100008958F929F92AF92BF92CF92DF92EF923B
:10D12000FF920F931F9361E044E050E00E94E66796
:10D13000BC0180E090E00E9423C10E9460C24B01CC
:10D140005C01C090BD04D090BE04E090BF04F0909C
:10D15000C0048EEC92E040E050E068E472EC00E045
:10D1600010E028E432E40E94172B9B01AC01C501BA
:10D17000B4010E94D9C11F910F91FF90EF90DF90F1
:10D18000CF90BF90AF909F908F900895CF92DF92F5
:10D19000EF92FF920F931F93CF93DF9361E042E0F2
:10D1A00050E00E94E667EC01DF7796FDD068C09002
:10D1B000B104D090B204E090B304F090B40482ECD7
:10D1C00092E040E050E068E472EC00E010E028E417
:10D1D00032E40E94172B6B017C01BE01882777FD8A
:10D1E0008095982F0E9425C19B01AC01C701B60113
:10D1F0000E94D9C1DF91CF911F910F91FF90EF90C5
:10D20000DF90CF900895CF92DF92EF92FF920F932D
:10D210001F93CF93DF9361E041E050E00E94E66707
:10D22000EC01DF7796FDD068C090AD04D090AE04DD
:10D23000E090AF04F090B0048EEB92E040E050E05C
:10D2400068E472EC00E010E028E432E40E94172B5E
:10D250006B017C01BE01882777FD8095982F0E9485
:10D2600025C19B01AC01C701B6010E94D9C1DF9164
:10D27000CF911F910F91FF90EF90DF90CF90089585
:10D280008F929F92AF92BF92CF92DF92EF92FF92D6
:10D290000F931F9361E045E050E00E94E667BC01F8
:10D2A00080E090E00E9423C10E9460C24B015C01BB
:10D2B000C090B904D090BA04E090BB04F090BC04D4
:10D2C0008AEC92E040E050E068E472EC00E010E0AC
:10D2D00028E432E40E94172B9B01AC01C501B40184
:10D2E0000E94D9C11F910F91FF90EF90DF90CF90D6
:10D2F000BF90AF909F908F9008958F929F92AF9222
:10D30000BF92CF92DF92EF92FF920F931F9361E053
:10D3100040E050E00E94E667BC0180E090E00E949F
:10D3200023C10E9460C24B015C01C090B504D09043
:10D33000B604E090B704F090B80486EC92E040E0C8
:10D3400050E068E472EC00E010E028E432E40E946F
:10D35000172B9B01AC01C501B4010E94D9C11F91DB
:10D360000F91FF90EF90DF90CF90BF90AF909F9084
:10D370008F900895462F90E061E050E00E94E667AC
:10D3800008956BE00E94BA699C012F773070295094
:10D390003040C9010895462F90E060E050E00E94BF
:10D3A000E667089569E00E94CB699C0194E0369598
:10D3B00027959A95E1F780E0922F9F700E9444652F
:10D3C000089569E00E94CB699C012F70307080E065
:10D3D000922F0E944465089569E00E94CB6980E025
:10D3E00092959F700E944465089569E00E94CB6900
:10D3F00080E09F700E9444650895662319F46FE0F1
:10D4000070E002C06FE870E00E94CB69292F30E025
:10D4100045E0220F331F4A95E1F7C9019F7034FDA3
:10D42000906F0E9476650895662319F46FE070E0AE
:10D4300002C06FE870E00E94CB69282F30E055E011
:10D44000220F331F5A95E1F7C9019F7034FD906F89
:10D450000E9476650895662319F46DE070E002C0BD
:10D460006DE870E00E94CB69292F30E065E0220F63
:10D47000331F6A95E1F7C9019F7034FD906F0E94D8
:10D48000AB650895662319F46DE070E002C06DE8A5
:10D4900070E00E94CB69282F30E075E0220F331F27
:10D4A0007A95E1F7C9019F7034FD906F0E94AB65DA
:10D4B0000895662319F46BE070E002C06BE870E039
:10D4C0000E94CB690E94E0650895662319F46CE020
:10D4D00070E002C06CE870E00E94CB690E94E065D9
:10D4E0000895662319F46EE070E002C06EE870E003
:10D4F0000E94CB690E9412660895662319F468E0C1
:10D5000070E002C068E870E00E94CB690E94126679
:10D51000089566E00E94CB69BC0160707F70672F40
:10D52000772780E090E00E9423C120E030E048ECC3
:10D5300052E40E94D9C120E030E040E751E40E946B
:10D540008AC0089566E00E94CB699C012F773070F5
:10D5500029503040C901089561E00E94CB690E94C2
:10D560004465089564E00E94CB690E94E0650895D7
:10D5700060E00E94CB690E94126608950E94CB6908
:10D580009C013F7094FD306FC9010895CF92DF92E6
:10D59000EF92FF920F931F93CF93DF9363E00E946C
:10D5A000BE6AEC01C090A104D090A204E090A30454
:10D5B000F090A40482EB92E040E050E068E472EC6A
:10D5C00000E010E028E432E40E94172B6B017C019C
:10D5D000BE01882777FD8095982F0E9425C19B0169
:10D5E000AC01C701B6010E94D9C1DF91CF911F9153
:10D5F0000F91FF90EF90DF90CF90089562E00E942E
:10D60000BE6A0E947665089565E00E94BE6A0E9427
:10D61000AB65089590E060E044E850E00E94E66762
:10D62000089594600E94D36708958F929F92AF925D
:10D63000BF92CF92DF92EF92FF920F931F93DF93EF
:10D64000CF9300D0CDB7DEB78C017B014A018CE2CD
:10D6500094EB9A838983DB01BC901196CC9011974F
:10D66000AFB6F894F8E5DF2EDCBC8DB581608DBDDA
:10D67000289AB4E000301B07F8F48EE094E80E948A
:10D680003405CE01019661E070E00E944F05E3EFA2
:10D69000F1E03197F1F700C0000028988FE79AE198
:10D6A000A6E081509040A040E1F700C00000DCBC43
:10D6B0008DB581608DBD289AC80190680E9434059F
:10D6C000C701B4010E944F05A3EFB1E01197F1F734
:10D6D00000C000002898B4E000301B0708F5E7E818
:10D6E000F3E13197F1F700C0000088E58CBD8DB5FE
:10D6F00081608DBD289A8EE094E80E9434058EEFFB
:10D700009AEC9A838983CE01019661E070E00E94D1
:10D710004F0583EF91E00197F1F700C000002898D2
:10D72000A7FE01C078948B2D9C2D0F900F90CF9168
:10D73000DF911F910F91FF90EF90DF90CF90BF90FE
:10D74000AF909F908F900895DF93CF9300D0CDB787
:10D75000DEB77A836983BE016F5F7F4F41E050E09F
:10D760000E94156B0F900F90CF91DF9108951F933A
:10D77000182F84E094E00E94D367BC017F73912F3F
:10D780009295907F80E0682B792B84E094E00E9452
:10D79000A46B1F91089594600E94A46B0895CF928A
:10D7A000DF92EF92FF921F93CF93DF93EC017B0107
:10D7B0006A011FB7F8940E94D367B601609570950F
:10D7C000682379236E297F29CE010E94A46B17FF5D
:10D7D00001C07894DF91CF911F91FF90EF90DF907F
:10D7E000CF9008950F931F93CF93DF93762FEA0185
:10D7F000890190E060E0472F50E00E941265BE0171
:10D80000A8010E94CF6BDF91CF911F910F910895D6
:10D810001F93182FCB01BA010E94446680E0492F64
:10D82000582F4031510510F04FE050E0A4E0440F74
:10D83000551FAA95E1F7812F69E020EF30E00E94A3
:10D84000F26B1F9108951F93182FCB01BA010E940C
:10D85000446680E0492F582F4031510510F04FE0C9
:10D8600050E0812F69E02FE030E00E94F26B1F91C1
:10D8700008951F93182FCB01BA010E94446680E0DF
:10D88000492F582FCA018031910510F08FE090E0A8
:10D89000582F5295507F812F69E040E020E030EF13
:10D8A0000E94F26B1F9108951F93182FCB01BA01AC
:10D8B0000E94446680E0492F582F9A01203131059B
:10D8C00010F02FE030E0812F69E040E0522F20E09F
:10D8D0003FE00E94F26B1F9108951F93CF93DF9357
:10D8E000182FCB01BA01222319F4CFE0D0E002C0F7
:10D8F000CFE8D0E00E9491669C01B5E03595279570
:10D90000BA95E1F74FEF203834071CF420E830E0F7
:10D9100007C0203831051CF02FE730E001C030701F
:10D92000812F6C2F40E0522F20E03FEF0E94F26BDE
:10D93000DF91CF911F9108951F93CF93DF93182FFD
:10D94000CB01BA01222319F4CFE0D0E002C0CFE826
:10D95000D0E00E949166AC0185E0559547958A9587
:10D96000E1F72FEF403852071CF440E850E007C0C1
:10D97000403851051CF04FE750E001C05070812F36
:10D980006C2F2FEF30E00E94F26BDF91CF911F914F
:10D9900008951F93CF93DF93182FCB01BA01222351
:10D9A00019F4CDE0D0E002C0C8E8D0E00E94C7661C
:10D9B0009C0195E0359527959A95E1F74FEF203832
:10D9C00034071CF420E830E007C0203831051CF093
:10D9D0002FE730E001C03070812F6C2F40E0522FD4
:10D9E00020E03FEF0E94F26BDF91CF911F910895ED
:10D9F0001F93CF93DF93182FCB01BA01222319F481
:10DA0000CDE0D0E002C0C8E8D0E00E94C766AC011B
:10DA100025E0559547952A95E1F72FEF40385207B5
:10DA20001CF440E850E007C0403851051CF04FE7B7
:10DA300050E001C05070812F6C2F2FEF30E00E941A
:10DA4000F26BDF91CF911F9108951F93CF93DF93D6
:10DA5000182FCB01BA01222319F4CBE0D0E002C089
:10DA6000CBE8D0E00E94FD66AC01812F6C2F2FEF38
:10DA70003FE00E94F26BDF91CF911F9108951F93B9
:10DA8000CF93DF93182FCB01BA01222319F4CCE0F6
:10DA9000D0E002C0CCE8D0E00E94FD66AC01812F4E
:10DAA0006C2F2FEF3FE00E94F26BDF91CF911F911F
:10DAB00008951F93CF93DF93182FCB01BA01222330
:10DAC00019F4CEE0D0E002C0CEE8D0E00E944A6770
:10DAD000AC01812F6C2F2FEF3FE00E94F26BDF91A2
:10DAE000CF911F9108951F93CF93DF93182FCB01F0
:10DAF000BA01222319F4C8E0D0E002C0C8E8D0E09F
:10DB00000E944A67AC01812F6C2F2FEF3FE00E94EB
:10DB1000F26BDF91CF911F910895CF93DF93C0E017
:10DB2000D0E00E94B11A0E94CC1A80E00E944B1BE8
:10DB3000009729F0219681E0C43FD80791F7DF9143
:10DB4000CF9108958091F61A882319F087E20E94F8
:10DB5000E90508958091631C882319F088E20E94EA
:10DB6000E90508950F931F93DF93CF93CDB7DEB7E9
:10DB700028970FB6F894DEBF0FBECDBF81EF9AE1B4
:10DB80000E94C3498DB79EB708970FB6F8949EBF01
:10DB90000FBE8DBFEDB7FEB731968E010F5F1F4FE1
:10DBA000ADB7BEB712961C930E93119788E090E024
:10DBB000938382838091321B9091331B958384835E
:10DBC0008091621B90E00196978386830E94B6C481
:10DBD000F80101900020E9F78DB79EB708960FB6BF
:10DBE000F8949EBF0FBE8DBFC8018E1B9F0B45963C
:10DBF0009695879561E00E949F04C8010E94550692
:10DC00000CED1AE1C80160E270E044E150E00E94CE
:10DC100059C48091631C882381F06091361B7091F8
:10DC2000371BDB01FD0101900020E9F73197EA1B6A
:10DC3000FB0BC801AF010E9450C46091341B70916E
:10DC4000351BDB01FD0101900020E9F73197EA1B4C
:10DC5000FB0B24E130E02E1B3F0B36952795245219
:10DC6000354EC901AF010E9450C482E090E00E948D
:10DC700043068091621B6EE00E94CB69192F809150
:10DC8000621B6CE00E94CB699295917012951170A5
:10DC9000910F092F9093F61A8CED9AE160E270E0F3
:10DCA00044E150E00E9459C4002391F060913A1B76
:10DCB00070913B1BDB01FD0101900020E9F73197DA
:10DCC000EA1BFB0B2EED3AE1C901AF010E9450C4E3
:10DCD00083E090E00E94430628960FB6F894DEBFDA
:10DCE0000FBECDBFCF91DF911F910F910895CF93BC
:10DCF000DF9388EC90E00E948905CCEDDAE1CE015B
:10DD000060E270E044E150E00E9459C481E00E946A
:10DD10009B12BC01FC0101900020E9F73197E81B40
:10DD2000F90B24E130E02E1B3F0B369527952C0F85
:10DD30003D1FC901AF010E9450C480E090E00E94E5
:10DD40004306CE0160E270E044E150E00E9459C415
:10DD500081E090E00E94430682E090E00E9443064A
:10DD600083E090E00E9443060E9457128BE00E94DD
:10DD70009B129093331B8093321B8FE00E949B1267
:10DD80009093351B8093341B83E70E949B129093E2
:10DD9000371B8093361B87E60E949B1290933B1B98
:10DDA00080933A1B81EF9AE10E94054A0E94B26D6E
:10DDB000DF91CF91089588E00E94E905089586E0FB
:10DDC0000E94E90508958AE00E94E905089587E028
:10DDD0000E94E905089585E00E94E9050895EF9203
:10DDE000FF920F931F93DF93CF93CDB7DEB72897A2
:10DDF0000FB6F894DEBF0FBECDBF81EF9AE10E944F
:10DE0000C3498DB79EB708970FB6F8949EBF0FBE53
:10DE10008DBFEDB7FEB731968E010F5F1F4FADB7C7
:10DE2000BEB712961C930E93119788E0E82EF12C42
:10DE3000F382E2828091321B9091331B958384831D
:10DE40008091681B90E00D96978386830E94B6C4EC
:10DE50008DB79EB708960FB6F8949EBF0FBE8DBFC4
:10DE600085E061E00E949F04C8010E945506ADB79D
:10DE7000BEB718970FB6F894BEBF0FBEADBFEDB7D3
:10DE8000FEB7319612961C930E931197F382E2829D
:10DE90008091341B9091351B958384838091631B03
:10DEA00090E00196978386830E94B6C48DB79EB793
:10DEB00008960FB6F8949EBF0FBE8DBF8AE061E052
:10DEC0000E949F04C8010E9455069091691B86EA32
:10DED000989FC00111243091631B21E1329F900172
:10DEE0001124820F931F8E569E4F60E04BE022E07C
:10DEF0000E94FA2981FD03C002EF17E002C002E090
:10DF000018E082E063E00E949F04C8010E94550669
:10DF100028960FB6F894DEBF0FBECDBFCF91DF912C
:10DF20001F910F91FF90EF900895EF92FF920F9342
:10DF30001F93DF93CF93CDB7DEB728970FB6F89432
:10DF4000DEBF0FBECDBF81EF9AE10E94C3498DB7FE
:10DF50009EB708970FB6F8949EBF0FBE8DBFEDB762
:10DF6000FEB731968E010F5F1F4FADB7BEB7129649
:10DF70001C930E93119798E0E92EF12CF382E28224
:10DF80008091321B9091331B958384838091681B11
:10DF900090E00D96978386830E94B6C48DB79EB796
:10DFA00008960FB6F8949EBF0FBE8DBF85E061E066
:10DFB0000E949F04C8010E945506ADB7BEB71897CE
:10DFC0000FB6F894BEBF0FBEADBFEDB7FEB731962A
:10DFD00012961C930E931197F382E2828091341B68
:10DFE0009091351B958384838091641B90E001960A
:10DFF000978386830E94B6C48DB79EB708960FB6E6
:10E00000F8949EBF0FBE8DBF8AE061E00E949F041E
:10E01000C8010E94550628960FB6F894DEBF0FBEC1
:10E02000CDBFCF91DF911F910F91FF90EF90089599
:10E030000F931F93DF93CF93CDB7DEB728970FB61B
:10E04000F894DEBF0FBECDBF81EF9AE10E94C349B5
:10E050008DB79EB708970FB6F8949EBF0FBE8DBFC1
:10E06000EDB7FEB731968E010F5F1F4FADB7BEB74C
:10E0700012961C930E93119788E090E0938382830D
:10E080008091321B9091331B958384838091681B10
:10E0900090E00D96978386830E94B6C4F8010190A4
:10E0A0000020E9F78DB79EB708960FB6F8949EBF8B
:10E0B0000FBE8DBFC8018E1B9F0B45969695879509
:10E0C00061E00E949F04C8010E94550628960FB681
:10E0D000F894DEBF0FBECDBFCF91DF911F910F919E
:10E0E00008950F931F93CF93DF9388EC90E00E94E5
:10E0F0008905CCEDDAE1CE0160E270E044E150E068
:10E100000E9459C481E00E949B12BC01FC01019055
:10E110000020E9F73197E81BF90B04E110E09801C2
:10E120002E1B3F0B369527952C0F3D1FC901AF01C4
:10E130000E9450C480E090E00E944306CE0160E25D
:10E1400070E044E150E00E9459C481E090E00E94F8
:10E15000430681E10E949B12BC01FC01019000205A
:10E16000E9F73197E81BF90B0E1B1F0B1695079566
:10E170000C0F1D1FC801AF010E9450C482E090E047
:10E180000E944306CE0160E270E044E150E00E944C
:10E1900059C483E090E00E94430681EF9AE10E9417
:10E1A000054ADF91CF911F910F910895CF93DF938F
:10E1B0000E9471708FE50E949B12EC0180E062E08A
:10E1C0000E949F04CE010E94550680E60E949B1289
:10E1D000EC0182E063E00E949F04CE010E9455069C
:10E1E0000E9457128CE00E949B129093331B8093E5
:10E1F000321B8EE00E949B129093351B8093341B40
:10E20000DF91CF9108959091691B86EA989FC00194
:10E2100011243091631B21E1329F90011124820F60
:10E22000931F8E569E4F60E04BE022E00E94FA2939
:10E2300081FF02C08D7001C082606091691B96EA07
:10E24000699FB00111242091631B91E1299F9001E6
:10E250001124620F731F6E567E4F0E94ED290E949B
:10E26000D6700895CF93DF930E9471708FE50E945E
:10E270009B12EC0180E062E00E949F04CE010E94AC
:10E2800055060E9457128CE00E949B129093331BFC
:10E290008093321B8DE00E949B129093351B8093DC
:10E2A000341BDF91CF910895CF93DF930E9471705B
:10E2B00087E70E949B12EC0180E062E00E949F04CD
:10E2C000CE010E94550688E70E949B12EC0182E075
:10E2D00063E00E949F04CE010E9455060E945712DF
:10E2E0008CE00E949B129093331B8093321BDF9132
:10E2F000CF9108958FE10E94E90508958EE10E9473
:10E30000E90508958DE10E94E90508958CE10E94D8
:10E31000E90508950F931F93DF93CF93CDB7DEB731
:10E3200028970FB6F894DEBF0FBECDBF81EF9AE1FC
:10E330000E94C3498DB79EB708970FB6F8949EBF49
:10E340000FBE8DBFEDB7FEB731968E010F5F1F4F29
:10E35000ADB7BEB712961C930E93119788E090E06C
:10E36000938382838091321B9091331B95838483A6
:10E370008091691B90E00D96978386830E94B6C4B6
:10E38000F80101900020E9F78DB79EB708960FB607
:10E39000F8949EBF0FBE8DBFC8018E1B9F0B459684
:10E3A0009695879561E00E949F04C8010E945506DA
:10E3B00028960FB6F894DEBF0FBECDBFCF91DF9188
:10E3C0001F910F910895EF92FF920F931F93CF9398
:10E3D000DF9388EC90E00E948905CCEDDAE1CE0174
:10E3E00060E270E044E150E00E9459C481E00E9484
:10E3F0009B12BC01FC0101900020E9F73197E81B5A
:10E40000F90B04E110E098012E1B3F0B3695279580
:10E410002C0F3D1FC901AF010E9450C480E090E065
:10E420000E944306CE0160E270E044E150E00E94A9
:10E4300059C481E090E00E94430687E70E949B1246
:10E44000BC01FC0101900020E9F73197E81BF90BB2
:10E45000CE01AF010E9450C48FE00E949B12BC010C
:10E46000FC0101900020E9F73197E81BF90B9801B6
:10E470002E1B3F0B369527952C0F3D1FC901AF0171
:10E480000E9450C489E70E949B12BC01FC010190CC
:10E490000020E9F73197E81BF90B0E1B1F0B0C0F3F
:10E4A0001D1FC801AF010E9450C482E090E00E948D
:10E4B0004306CE0160E270E044E150E00E9459C49E
:10E4C00082E798E00E946612BC01FC0101900020E6
:10E4D000E9F73197E81BF90B9E012E1B3F0B2E5ECF
:10E4E0003F4FC901AF010E9450C488E70E949B12B0
:10E4F000BC01FC0101900020E9F73197E81BF90B02
:10E500002296CE01AF010E9450C483E090E00E94A9
:10E51000430681EF9AE10E94054A0E9457128CE05F
:10E520000E949B129093331B8093321BDF91CF91FB
:10E530001F910F91FF90EF900895382F262F862F6F
:10E5400063E00E940BC390E0880F991F86599A4F91
:10E55000FC01A591B4912150253010F020E005C0B8
:10E56000E22FF0E0E057F74F2081832F90E08C57A7
:10E570009F4F34E0880F991F3A95E1F7642F70E0C0
:10E580006F707070022E02C0660F771F0A94E2F758
:10E590004FE050E002C0440F551F2A95E2F78A0F62
:10E5A0009B1F0E94CF6B08951F93382F262F862F15
:10E5B00063E00E940BC390E0880F991F86599A4F21
:10E5C000FC01459154912150253010F010E005C018
:10E5D000E22FF0E0E057F74F1081832F90E08C5747
:10E5E0009F4F64E0880F991F6A95E1F7840F951F8C
:10E5F0000E94D36702C0969587951A95E2F78F70AF
:10E600001F91089570E0660F771F62597A4FFB01E2
:10E610002591349190E08C579F4FE4E0880F991F2B
:10E62000EA95E1F7820F931F0E94D3670895663041
:10E6300018F020E030E015C070E0660F771F640F1F
:10E64000751FFB012591349190E08C579F4FA4E0FA
:10E65000880F991FAA95E1F7820F931F0E94D36735
:10E660009C01C9010895643018F020E030E015C025
:10E6700070E0660F771F640F751FFB0125913491C1
:10E6800090E08C579F4F44E0880F991F4A95E1F71F
:10E69000820F931F0E94D3679C01C901089560E017
:10E6A0004AEC55E00E943373BC01009729F460E006
:10E6B00070E080E090E00CC080E090E00E9423C118
:10E6C0009B01AC0160E070EA8CE09AE40E948AC091
:10E6D000089542ED55E00E9433730895DF93CF9380
:10E6E0000F92CDB7DEB7E62FF0E0EE0FFF1FEE5131
:10E6F000FA4F8591949169830E94D367282F69818D
:10E70000862F63E00E940BC341E050E002C0440F3B
:10E71000551F9A95E2F7822F84230F90CF91DF91B6
:10E720000895CF92DF92EF92FF920F931F93CF93B2
:10E73000DF93182FC62E0E943373EC01DF7796FD0E
:10E74000D06826EA129F90011124225A3E4F8C2D48
:10E7500090E0B4E0880F991FBA95E1F7C090D50416
:10E76000D090D604E090D704F090D804820F931F85
:10E7700040E050E068E472EC00E010E028E432E4AD
:10E780000E94172B6B017C01BE01882777FD8095C5
:10E79000982F0E9425C19B01AC01C701B6010E94C0
:10E7A000D9C1DF91CF911F910F91FF90EF90DF9032
:10E7B000CF90089542E955E00E949173089542ED8B
:10E7C00055E00E9491730895CF92DF92EF92FF92ED
:10E7D0000F931F93CF93DF93082F162F42EB55E033
:10E7E0000E941773EC01DF7796FDD06826EA029F3E
:10E7F0009001112429563E4F81E1189FC001112438
:10E80000C090DD04D090DE04E090DF04F090E004DE
:10E81000820F931F40E050E068E472EC00E010E0EB
:10E8200028E432E40E94172B6B017C01BE0188278B
:10E8300077FD8095982F0E9425C1A70196010E941F
:10E84000D9C1DF91CF911F910F91FF90EF90DF9091
:10E85000CF9008956F927F928F929F92AF92BF92C6
:10E86000CF92DF92EF92FF920F931F93CF93DF939C
:10E87000A82EB62EEA013801490126EA829F9001AE
:10E8800011242D563E4F81E1689FC0011124C09094
:10E89000D904D090DA04E090DB04F090DC04820F1D
:10E8A000931F40E050E068E472EC00E010E028E4E0
:10E8B00032E40E94172B9B01AC0185E08B15A0F17F
:10E8C0008B2D90E0880F991F8C0F9D1FFC01C59127
:10E8D000D491C401B3010E948AC00E94F2C0669F15
:10E8E0009001679F300D769F300D1124B90180E0B3
:10E8F00090E00E9423C10E943CC29B01AC018A2D82
:10E9000090E08C579F4F14E0880F991F1A95E1F7FC
:10E91000C80FD91FCA01B9010E94F7C09B01AC0101
:10E92000CE01B9010E94A46BDF91CF911F910F918D
:10E93000FF90EF90DF90CF90BF90AF909F908F901F
:10E940007F906F9008950F931F9389019A014AE772
:10E9500055E00E942A741F910F9108950F931F9301
:10E9600089019A0146E855E00E942A741F910F918F
:10E970000895FF920F931F93CF93DF93F82E643087
:10E9800020F5862F90E0880F991F840F951FFC01BA
:10E99000C591D491C901B8010E943CC29B01AC0150
:10E9A0008F2D90E08C579F4F64E0880F991F6A95D8
:10E9B000E1F7C80FD91FCA01B9010E94F7C09B0136
:10E9C000AC01CE01B9010E94A46BDF91CF911F91E0
:10E9D0000F91FF9008956F927F928F929F92AF92C6
:10E9E000BF92CF92DF92EF92FF920F931F93B82EB8
:10E9F000A62E39014A0186EA2B2D289FC001112439
:10EA0000825A9E4F262F30E0E4E0220F331FEA9512
:10EA1000E1F7C090D504D090D604E090D704F090F0
:10EA2000D804820F931F40E050E068E472EC00E0ED
:10EA300010E028E432E40E94172B9B01AC01C401D2
:10EA4000B3010E948AC00E94F7C080E090E00E945B
:10EA500023C18B019C018B2D6A2D42E955E00E9458
:10EA6000B9741F910F91FF90EF90DF90CF90BF90FE
:10EA7000AF909F908F907F906F9008956F927F924C
:10EA80008F929F92AF92BF92CF92DF92EF92FF92BE
:10EA90000F931F93B82EA62E39014A0186EA2B2D1B
:10EAA000289FC0011124865A9E4F262F30E0F4E0A3
:10EAB000220F331FFA95E1F7C090D104D090D20411
:10EAC000E090D304F090D404820F931F40E050E014
:10EAD00068E472EC00E010E028E432E40E94172BB6
:10EAE0009B01AC01C401B3010E948AC0562F472F7D
:10EAF000382F292FDA01F9016B2F7A2F8F2F9E2FB4
:10EB00002B2F3A2F4F2F5E2F0E94D9C10E94F7C0A2
:10EB100080E090E00E9423C18B019C018B2D6A2D27
:10EB20004AE955E00E94B9741F910F91FF90EF9050
:10EB3000DF90CF90BF90AF909F908F907F906F901D
:10EB400008956F927F928F929F92AF92BF92CF92D1
:10EB5000DF92EF92FF920F931F93CF93DF93B82E24
:10EB6000A62EEA013801490186EA2B2D289FC00113
:10EB700011248A5A9E4F262F30E0A4E0220F331F23
:10EB8000AA95E1F7C090CD04D090CE04E090CF04D8
:10EB9000F090D004820F931F40E050E068E472ECE4
:10EBA00000E010E028E432E40E94172B9B01AC0146
:10EBB000C401B3010E948AC0562F472F382F292F36
:10EBC000DA01F9016B2F7A2F8F2F9E2F2B2F3A2FDF
:10EBD0004F2F5E2F0E94D9C10E94F7C080E090E0C5
:10EBE0000E9423C18B019C018B2D6A2DAE010E94D6
:10EBF000B974DF91CF911F910F91FF90EF90DF904B
:10EC0000CF90BF90AF909F908F907F906F9008951E
:10EC10000F931F9389019A0142EA55E00E94A17562
:10EC20001F910F9108950F931F9389019A014AEA4A
:10EC300055E00E94A1751F910F910895EF92FF92E8
:10EC40001F93DF93CF930F92CDB7DEB7162F862F8A
:10EC500090E0880F991F8E519A4FFC01E590F49037
:10EC6000C70149830E94D3679C01812F63E00E9402
:10EC70000BC361E070E002C0660F771F9A95E2F760
:10EC8000CB0180959095282339234981442311F0A5
:10EC9000262B372BC701B9010E94A46B0F90CF918F
:10ECA000DF911F91FF90EF9008952F923F924F9226
:10ECB0005F926F927F928F929F92AF92BF92CF920C
:10ECC000DF92EF92FF920F931F93DF93CF930F92F8
:10ECD000CDB7DEB7182F062F29830E9417734C017A
:10ECE000AA24BB242981222359F5C501B4010E941D
:10ECF00023C10E9460C24B015C0126EA129F900171
:10ED000011242D563E4F81E1089FC0011124C0906F
:10ED1000D904D090DA04E090DB04F090DC04820F98
:10ED2000931F40E050E068E472EC00E010E028E45B
:10ED300032E40E94172B9B01AC01C501B4014EC007
:10ED400081E1089F1001112486EA189FC001112457
:10ED5000280E391EC090E504D090E604E090E70448
:10ED6000F090E804C10181569E4F40E050E068E415
:10ED700072EC00E010E028E432E40E94172B2B0133
:10ED80003C01C090E104D090E204E090E304F090F4
:10ED9000E404C10185569E4F40E050E068E472EC07
:10EDA00000E010E028E432E40E94172B7B018C0184
:10EDB000C501B4010E9423C14B015C01C301B20132
:10EDC00020E030E44CE156EC0E94D9C19B01AC013B
:10EDD000C501B4010E9422C0A80197010E94D9C1B7
:10EDE0000F90CF91DF911F910F91FF90EF90DF90E7
:10EDF000CF90BF90AF909F908F907F906F905F90DB
:10EE00004F903F902F9008954AE755E020E00E94F0
:10EE10005576089546E855E020E00E94557608951D
:10EE2000242F4EEB55E00E94557608958F929F92C5
:10EE3000AF92BF92CF92DF92EF92FF920F931F9308
:10EE4000082F162F0E943373BC0180E090E00E94CF
:10EE500023C10E9460C24B015C0126EA029F90011F
:10EE60001124265A3E4F812F90E014E0880F991FFD
:10EE70001A95E1F7C090D104D090D204E090D30469
:10EE8000F090D404820F931F40E050E068E472ECED
:10EE900000E010E028E432E40E94172B9B01AC0153
:10EEA000C501B4010E94D9C11F910F91FF90EF904D
:10EEB000DF90CF90BF90AF909F908F9008954AE9D8
:10EEC00055E00E94167708954AED55E00E941677A6
:10EED00008958F929F92AF92BF92CF92DF92EF925E
:10EEE000FF920F931F93082F162F0E943373BC01BC
:10EEF00080E090E00E9423C10E9460C24B015C014F
:10EF000026EA029F900111242A5A3E4F812F90E059
:10EF100004E0880F991F0A95E1F7C090CD04D090C6
:10EF2000CE04E090CF04F090D004820F931F40E015
:10EF300050E068E472EC00E010E028E432E40E9463
:10EF4000172B9B01AC01C501B4010E94D9C11F91CF
:10EF50000F91FF90EF90DF90CF90BF90AF909F9078
:10EF60008F90089542EA55E00E94697708954AEA31
:10EF700055E00E94697708954EEE55E00E9469774A
:10EF800008958EE10E94DF0508958F929F92AF92BF
:10EF9000BF92CF92DF92EF92FF920F931F93DF9376
:10EFA000CF93CDB7DEB764970FB6F894DEBF0FBE30
:10EFB000CDBF8091661B882309F479C080910D1C18
:10EFC0008F3F09F474C080910F1C8F3708F06FC019
:10EFD0009091F11A8091621B992351F50E9440692A
:10EFE0006093F61A7093F71A8093F81A9093F91AAF
:10EFF0008091621B90E00E944C686093FA1A7093B3
:10F00000FB1A8093FC1A9093FD1A8091621B90E08A
:10F010000E94C6686093FE1A7093FF1A8093001BCB
:10F020009093011B8091621B90E00E940A682AC0A5
:10F0300090E00E947D696093F61A7093F71A8093AE
:10F04000F81A9093F91A8091621B90E00E948968E7
:10F050006093FA1A7093FB1A8093FC1A9093FD1A2E
:10F060008091621B90E00E9403696093FE1A709386
:10F07000FF1A8093001B9093011B8091621B90E00C
:10F080000E94066860930A1B70930B1B80930C1BF5
:10F0900090930D1B8091621B90E00E940E6860931C
:10F0A0000E1B70930F1B8093101B9093111B80916C
:10F0B000661B882309F431C18091691B90916B1BF9
:10F0C000891708F02AC16091641B0E94BC77609385
:10F0D000F11A7093F21A8093F31A9093F41A8091B4
:10F0E000691B6091641B0E9464776093F51A7093AA
:10F0F000F61A8093F71A9093F81A8091691B609121
:10F10000641B0E94DF736093FD1A7093FE1A809354
:10F11000FF1A9093001B8091691B6091641B0E94F1
:10F120004F736093F91A7093FA1A8093FB1A9093B5
:10F13000FC1A6091F11A7091F21A8091F31A909171
:10F14000F41A2091F51A3091F61A4091F71A50915D
:10F15000F81A0E94D9C1D62EC72EB82EA92EA60104
:10F160009501652F742F832F922F20E030E040EA25
:10F1700050E40E94D5C118165CF00F2EF0E0EF2E7F
:10F18000F0E0FF2EF0E00F2FF0E01F2FF02D33C046
:10F190006091FD1A7091FE1A8091FF1A9091001BE8
:10F1A000D601F5012B2F3A2F4F2F5E2F0E948AC0D8
:10F1B000E62EF72E082F192F20E030E0A9010E943B
:10F1C00086C0882324F417FB109517F91095C80101
:10F1D000B70120E030E040E85FE30E94D5C1181697
:10F1E00054F40F2EF0E0EF2EF0E0FF2EF0E80F2F9A
:10F1F000FFE31F2FF02D80E060E00E949F048DB799
:10F200009EB70E970FB6F8949EBF0FBE8DBFEDB799
:10F21000FEB731964E010894811C911CADB7BEB764
:10F2200012969C928E92119784E190E09383828350
:10F2300085E998E0958384838091641B90E0019632
:10F2400097838683E086F186028713878091691B06
:10F2500090E00D96958784870E94B6C48DB79EB7BF
:10F260000E960FB6F8949EBF0FBE8DBFC4010E94CC
:10F27000550680E061E00E949F046091F11A709150
:10F28000F21A8091F31A9091F41A4DEA58E025E0B1
:10F290000E949D0687E061E00E949F046091F91A38
:10F2A0007091FA1A8091FB1A9091FC1A43EB58E086
:10F2B00025E00E949D068EE061E00E949F0460911F
:10F2C000F51A7091F61A8091F71A9091F81A4DEA92
:10F2D00058E025E00E949D0683E062E00E949F04C2
:10F2E0006091FD1A7091FE1A8091FF1A9091001B97
:10F2F00049EB58E027E00E949D068BE062E00E9407
:10F300009F04A6019501652F7C2D832F9A2D49EB33
:10F3100058E027E00E949D0630C087E060E00E9430
:10F320009F0486E392E00E94550680E061E00E941F
:10F330009F0488E392E00E9455068EE061E00E94FF
:10F340009F0488E392E00E94550683E062E00E94F9
:10F350009F0486E392E00E9455068BE062E00E94E3
:10F360009F0486E392E00E9455068BE060E00E94D5
:10F370009F0486E392E00E94550664960FB6F894C7
:10F38000DEBF0FBECDBFCF91DF911F910F91FF90D8
:10F39000EF90DF90CF90BF90AF909F908F900895A7
:10F3A000EF92FF92CF93DF9381E08093F11A84EF85
:10F3B00091E00E948905CCEDDAE1CE0160E270E0D7
:10F3C00044E150E00E9459C480E090E00E9443066E
:10F3D000CE0160E270E044E150E00E9459C481E453
:10F3E0000E949B12BC01FC0101900020E9F73197BB
:10F3F000E81BF90B9E01245F3F4FC901AF010E943A
:10F4000050C486E58093E11A81E48093EF1A81E08D
:10F4100090E00E944306CE0160E270E044E150E0DB
:10F420000E9459C483E40E949B12BC01FC0101901C
:10F430000020E9F73197E81BF90BCE01AF010E94DC
:10F4400050C487E58093E61A82E40E949B12BC01B7
:10F45000FC0101900020E9F73197E81BF90B9E01B0
:10F460002E5E3F4FC901AF010E9450C482E090E080
:10F470000E944306CE0160E270E044E150E00E9449
:10F4800059C483E090E00E9443060E94C577DF9153
:10F49000CF91FF90EF9008958091511C882371F4D3
:10F4A00080E090E0DC018093F91A9093FA1AA0931F
:10F4B000FB1AB093FC1A0E94662808958091521C92
:10F4C000882311F080E001C083E08093521C1092E9
:10F4D000991080E090E0DC0180939A1090939B104B
:10F4E000A0939C10B0939D1008958091511C882387
:10F4F00071F480E090E0DC018093F91A9093FA1A9D
:10F50000A093FB1AB093FC1A0E945C280895809186
:10F51000521C882311F080E001C083E08093521CCC
:10F520001092991080E090E0DC0180939A10909303
:10F530009B10A0939C10B0939D1008958091661B22
:10F54000882349F110924E1C10924D1C8091691B2A
:10F550006091631B0E94D47280FF05C0482F4E7FCC
:10F560001092151B07C0482F416081E08093151B46
:10F5700010929F1085E080939E108091691B60918E
:10F58000631B0E949D728EEC98E00E94D36790935B
:10F59000541C8093531C08958091161B882331F4CA
:10F5A0008091691B6091631B41E005C08091691BDC
:10F5B0006091631B40E00E941E760895CF93DF9315
:10F5C0008091511C882389F58CE060E00E949F04A3
:10F5D00086E392E00E94550687E060E00E949F0467
:10F5E00086E392E00E94550680E061E00E949F045D
:10F5F00088E392E00E9455068EE061E00E949F043D
:10F6000088E392E00E94550683E062E00E949F0436
:10F6100086E392E00E9455068BE062E00E949F0420
:10F6200086E392E00E94550616C0C0E0D0E08CE070
:10F630006C2F0E949F0486E392E00E94550682E0B0
:10F640006C2F0E949F0486E392E00E94550621964B
:10F65000C430D10561F7DF91CF910895CF93DF9347
:10F660001092511C1092521C84EF91E00E94890567
:10F67000CCEDDAE1CE0160E270E044E150E00E94BE
:10F6800059C480E090E00E944306CE0160E270E041
:10F6900044E150E00E9459C481E090E00E9443069A
:10F6A000CE0160E270E044E150E00E9459C482E083
:10F6B00090E00E944306CE0160E270E044E150E039
:10F6C0000E9459C483E090E00E9443060E945712B2
:10F6D0008CE00E949B129093331B8093321B8EE030
:10F6E0000E949B129093351B8093341B87ED98E00A
:10F6F0000E9466129093371B8093361B86E90E9406
:10F700009B129093391B8093381B8EED98E00E94DA
:10F71000661290933B1B80933A1B85EE98E00E9403
:10F72000661290933D1B80933C1B87E90E949B12BD
:10F7300090933F1B80933E1B8CEE98E00E946612D4
:10F740009093431B8093421B8FEE98E00E946612B9
:10F750009093411B8093401BDF91CF910895CF92EE
:10F76000DF92EF92FF920F931F93CF93DF93EC0101
:10F77000162F042F862F642F0E946E73482F8DA39F
:10F78000812F602F0E941077688379838A839B83FF
:10F790008091511C882349F0812F602F0E94E473CF
:10F7A000688779878A879B873DC0C0909A10D090E0
:10F7B0009B10E0909C10F0909D10812F602F0E9474
:10F7C000E4739B01AC01C701B6010E9422C0262F41
:10F7D000372F482F592F20939A1030939B10409326
:10F7E0009C1050939D1020919910322F3F5F3093C1
:10F7F00099102430B8F020E030E040EA50E40E9454
:10F800008AC0688779878A879B871092991080E0E1
:10F8100090E0DC0180939A1090939B10A0939C1031
:10F82000B0939D10812F602F0E940273292F30E02A
:10F8300039A328A3013031F0013090F0802F84509B
:10F84000823070F4C90144E0969587954A95E1F7B6
:10F8500083708BA396E0369527959A95E1F707C0BC
:10F86000822F83708BA33695279536952795237025
:10F870002AA30330D8F4812F60E00E94BC776B018B
:10F880007C016C837D838E839F83812F60E00E9447
:10F8900064779B01AC01C701B6010E94D9C16C8B92
:10F8A0007D8B8E8B9F8B812F60E01AC0812F61E052
:10F8B0000E94BC776B017C016C837D838E839F8368
:10F8C000812F61E00E9464779B01AC01C701B60102
:10F8D0000E94D9C16C8B7D8B8E8B9F8B812F61E0B9
:10F8E0000E94DF73688F798F8A8F9B8F812F602FA3
:10F8F0000E94D47281708CA3EC88FD880E891F89C8
:10F90000C801B7012AE037ED43E25CE30E94D5C1AC
:10F9100018160CF03CC0688D798D8A8D9B8DA801DE
:10F9200097010E948AC0562F472F382F292FE62E85
:10F93000F72E082F192F862F942FA32FB22F8C8FDD
:10F940009D8FAE8FBF8F652F742F832F922F20E056
:10F9500030E0A9010E9486C0882344F417FB10956B
:10F9600017F91095EC8EFD8E0E8F1F8F6C8D7D8D8F
:10F970008E8D9F8D20E030E040E85FE30E94D5C18E
:10F98000181664F480E090E0A0E8BFE303C080E0D4
:10F9900090E0DC018C8F9D8FAE8FBF8F6C817D815D
:10F9A0008E819F81288139814A815B810E94D9C1E2
:10F9B0007B018C01862F9F2DA02FB12F888B998BD7
:10F9C000AA8BBB8B6E2D7F2D802F912F20E030E0F6
:10F9D00040EA50E40E94D5C118160CF03EC068857C
:10F9E00079858A859B852E2D3F2D402F512F0E9492
:10F9F0008AC0562F472F382F292FE62EF72E082F93
:10FA0000192F862F942FA32FB22F8C879D87AE8717
:10FA1000BF87652F742F832F922F20E030E0A9013C
:10FA20000E9486C0882344F417FB109517F910959F
:10FA3000EC86FD860E871F876C857D858E859F856C
:10FA400020E030E040E85FE30E94D5C1181664F47E
:10FA500080E090E0A0E8BFE303C080E090E0DC013C
:10FA60008C879D87AE87BF87DF91CF911F910F91C4
:10FA7000FF90EF90DF90CF9008951F93DF93CF9387
:10FA8000CDB7DEB72A970FB6F894DEBF0FBECDBF55
:10FA9000182F81EF9AE16091691B412F0E94AF7B83
:10FAA0008091151B882321F08091131B80FD38C0A5
:10FAB0004091161B9E012F5F3F4F812F90E0442302
:10FAC000C9F44DB75EB74C5050400FB6F8945EBFC6
:10FAD0000FBE4DBFEDB7FEB73196ADB7BEB71296AC
:10FAE0003C932E9311972AE030E03383228322EF58
:10FAF00038E04AC0ADB7BEB71C970FB6F894BEBF8A
:10FB00000FBEADBFEDB7FEB7319612963C932E9364
:10FB100011972AE030E0338322832EEF38E034C09F
:10FB20004091161B9E012F5F3F4F812F90E0442391
:10FB3000B1F4ADB7BEB71C970FB6F894BEBF0FBEF9
:10FB4000ADBFEDB7FEB7319612963C932E93119749
:10FB50002AE030E03383228329E039E015C0ADB7D5
:10FB6000BEB71C970FB6F894BEBF0FBEADBFEDB7C2
:10FB7000FEB7319612963C932E9311972AE030E00F
:10FB80003383228325E139E03583248301969783EB
:10FB900086838091F11A9091F21AA091F31AB09194
:10FBA000F41A80879187A287B3870E94B6C44DB7A5
:10FBB0005EB7445F5F4F0FB6F8945EBF0FBE4DBF98
:10FBC000CE0101960E9455062A960FB6F894DEBF24
:10FBD0000FBECDBFCF91DF911F9108951F93DF938B
:10FBE000CF93CDB7DEB72A970FB6F894DEBF0FBE1E
:10FBF000CDBF182F81EF9AE16091691B412F0E94C0
:10FC0000AF7B8091151B882321F08091131B80FD11
:10FC100038C04091161B9E012F5F3F4F812F90E00F
:10FC20004423C9F44DB75EB74C5050400FB6F8941A
:10FC30005EBF0FBE4DBFEDB7FEB73196ADB7BEB7D5
:10FC400012963C932E9311972AE030E0338322835F
:10FC500020E239E04AC0ADB7BEB71C970FB6F894A2
:10FC6000BEBF0FBEADBFEDB7FEB7319612963C9347
:10FC70002E9311972AE030E0338322832CE239E07F
:10FC800034C04091161B9E012F5F3F4F812F90E0A3
:10FC90004423B1F4ADB7BEB71C970FB6F894BEBFFE
:10FCA0000FBEADBFEDB7FEB7319612963C932E93C3
:10FCB00011972AE030E03383228327E339E015C02F
:10FCC000ADB7BEB71C970FB6F894BEBF0FBEADBFA1
:10FCD000EDB7FEB7319612963C932E9311972AE01A
:10FCE00030E03383228323E439E035832483019693
:10FCF000978386838091F91A9091FA1AA091FB1A42
:10FD0000B091FC1A80879187A287B3870E94B6C4FE
:10FD10004DB75EB7445F5F4F0FB6F8945EBF0FBE3E
:10FD20004DBFCE0101960E9455062A960FB6F89453
:10FD3000DEBF0FBECDBFCF91DF911F910895CF924F
:10FD4000DF92EF92FF921F93DF93CF93CDB7DEB791
:10FD50002B970FB6F894DEBF0FBECDBF182F81EFE3
:10FD60009AE16091691B412F0E94AF7B8091151B26
:10FD7000882321F08091131B80FD37C08091161BD2
:10FD80007E010894E11CF11C8823C9F48DB79EB74D
:10FD90000C970FB6F8949EBF0FBE8DBFEDB7FEB7A0
:10FDA0003196ADB7BEB71296FC92EE9211976BE00A
:10FDB000C62ED12CD382C2828EE499E035C0ADB775
:10FDC000BEB71C970FB6F894BEBF0FBEADBFEDB760
:10FDD000FEB731961296FC92EE9211978AE090E06F
:10FDE0009383828384E699E07CC08091161B7E0118
:10FDF0000894E11CF11C882309F05EC0ADB7BEB7C2
:10FE00001C970FB6F894BEBF0FBEADBFEDB7FEB7DF
:10FE100031961296FC92EE9211975BE0C52ED12C92
:10FE2000D382C28281E799E0958384831683178207
:10FE30008091F91A9091FA1AA091FB1AB091FC1ACC
:10FE400080879187A287B3870E94B6C48DB79EB77B
:10FE50000C960FB6F8949EBF0FBE8DBFC7010E94CF
:10FE600055068BE062E00E949F04ADB7BEB71A97BB
:10FE70000FB6F894BEBF0FBEADBFEDB7FEB731965B
:10FE80001296FC92EE921197D382C2828BE599E092
:10FE9000958384838091FD1A9091FE1AA091FF1A98
:10FEA000B091001B86839783A087B1870E94B6C458
:10FEB0008DB79EB70A962AC0ADB7BEB71C970FB6CE
:10FEC000F894BEBF0FBEADBFEDB7FEB73196129628
:10FED000FC92EE9211978AE090E0938382838EE702
:10FEE00099E095838483168317828091F91A909103
:10FEF000FA1AA091FB1AB091FC1A80879187A28709
:10FF0000B3870E94B6C48DB79EB70C960FB6F8940F
:10FF10009EBF0FBE8DBFCE0101960E9455062B9647
:10FF20000FB6F894DEBF0FBECDBFCF91DF911F910A
:10FF3000FF90EF90DF90CF900895EF92FF920F9394
:10FF40001F93DF93CF93CDB7DEB7A8970FB6F89482
:10FF5000DEBF0FBECDBF8091511C823009F486C038
:10FF6000833009F419C1813009F0BCC180E060E040
:10FF70000E949F0480E00E943D7D8AE060E00E9434
:10FF80009F0481E00E943D7D80E061E00E949F042B
:10FF900082E00E943D7D8AE061E00E949F0483E050
:10FFA0000E943D7D80E062E00E949F0484E00E9408
:10FFB0003D7D8AE062E00E949F0485E00E943D7DD5
:10FFC00080E063E00E949F048091691B60E00E94D2
:10FFD00064772DB73EB72A5030400FB6F8943EBF35
:10FFE0000FBE2DBFEDB7FEB731968E010B5E1F4FD2
:10FFF000ADB7BEB712961C930E931197BAE0EB2ED5
:020000021000EC
:10000000F12CF382E2822BE839E035832483668386
:100010007783808791870E94B6C42DB73EB7265F4D
:100020003F4F0FB6F8943EBF0FBE2DBFC8010E94D0
:1000300055068AE063E00E949F048091691B61E09D
:100040000E946477ADB7BEB71A970FB6F894BEBFDB
:100050000FBEADBFEDB7FEB7319612961C930E934F
:100060001197F382E28225E939E07CC080E060E00C
:100070000E949F0480E00E94EE7D8AE060E00E9482
:100080009F0481E00E94EE7D80E061E00E949F0479
:1000900082E00E94EE7D8AE061E00E949F0483E09E
:1000A0000E94EE7D80E062E00E949F0484E00E9456
:1000B000EE7D8AE062E00E949F0485E00E94EE7D72
:1000C00080E063E00E949F048091691B60E00E94D1
:1000D000DF73ADB7BEB71A970FB6F894BEBF0FBEA9
:1000E000ADBFEDB7FEB731968E010B5E1F4F129676
:1000F0001C930E931197AAE0EA2EF12CF382E28270
:100100002FE939E03583248366837783808791875D
:100110000E94B6C42DB73EB7265F3F4F0FB6F89486
:100120003EBF0FBE2DBFC8010E9455068AE063E0A6
:100130000E949F048091691B61E00E94DF73ADB74C
:10014000BEB71A970FB6F894BEBF0FBEADBFEDB7DE
:10015000FEB7319612961C930E931197F382E282AA
:1001600029EA39E035832483668377838087918702
:100170000E94B6C42DB73EB7265F3F4F0FB6F89426
:100180003EBF0FBE2DBFC8010E9455068091661B61
:10019000882309F09FC083C21091521C1111125084
:1001A00081EF9AE16091691B412F0E94AF7B80E053
:1001B00060E00E949F04812F8F5F0E949F7E412FED
:1001C0004E5F81EF9AE16091691B0E94AF7B80E0F6
:1001D00061E00E949F04812F8D5F0E949F7E412FCE
:1001E0004C5F81EF9AE16091691B0E94AF7B80E0D8
:1001F00062E00E949F04812F8B5F0E949F7E80E0BF
:1002000063E00E949F048DB79EB70C970FB6F894D9
:100210009EBF0FBE8DBFEDB7FEB731968E010B5E50
:100220001F4FADB7BEB712961C930E9311977BE08C
:10023000E72EF12CF382E28283EB99E095838483AD
:100240008091521C90E08170907001969783868314
:100250008091091B90910A1BA0910B1BB0910C1B64
:1002600080879187A287B3870E94B6C42DB73EB717
:10027000245F3F4F0FB6F8943EBF0FBE2DBFC8019D
:100280000E9455068BE063E00E949F048DB79EB7E5
:100290000A970FB6F8949EBF0FBE8DBFEDB7FEB79D
:1002A0003196ADB7BEB712961C930E931197F38299
:1002B000E2828BE599E09583848380910D1B909178
:1002C0000E1BA0910F1BB091101B86839783A087F4
:1002D000B1874ECF9091691B80916B1B981708F0E6
:1002E000DEC1DFC181EF9AE16091691B4091631B20
:1002F0000E94AF7B8CED9AE160E270E044E150E057
:100300000E9459C481E48093EF1A8091161B8823C0
:1003100019F486E58093E11A81E090E00E9443069B
:1003200080E061E00E949F0400D000D000D0EDB7D3
:10033000FEB731968E010F5F1F4FADB7BEB7129655
:100340001C930E93119784E190E09383828380EC59
:1003500099E0958384830E94B6C42DB73EB72A5F87
:100360003F4F0FB6F8943EBF0FBE2DBFC8010E948D
:1003700055068CED9AE160E270E044E150E00E94A5
:1003800059C48091161B882379F480E58093DC1A88
:100390008AE38093DD1A87E58093E61A86E58093E9
:1003A000EE1A81E48093EF1A82E090E00E94430607
:1003B0008091661B882309F472C19091691B80911A
:1003C0006B1B981708F06BC180E060E00E949F04EF
:1003D0008091151B882321F08091131B80FD32C072
:1003E0002091161BCE0145962223B1F4ADB7BEB7BE
:1003F0001E970FB6F894BEBF0FBEADBFEDB7FEB7E8
:10040000319612969C938E93119784E190E093839A
:10041000828383ED99E031C0ADB7BEB71A970FB6AE
:10042000F894BEBF0FBEADBFEDB7FEB731961296C2
:100430009C938E93119784E190E0938382838BEE5B
:1004400099E051C02091161BCE0145962223B1F5AB
:10045000ADB7BEB71E970FB6F894BEBF0FBEADBF07
:10046000EDB7FEB7319612969C938E93119784E167
:1004700090E09383828382E09AE0958384838091E5
:10048000631B90E00196978386838091FD1A90917B
:10049000FE1AA091FF1AB091001B80879187A28756
:1004A000B3878091691B90E00D96958784870E94A1
:1004B000B6C42DB73EB7225F3F4F29C0ADB7BEB718
:1004C0001A970FB6F894BEBF0FBEADBFEDB7FEB71B
:1004D000319612969C938E93119784E190E09383CA
:1004E00082838AE19AE0958384838091631B90E004
:1004F0000196978386838091691B90E00D96918782
:1005000080870E94B6C42DB73EB7265F3F4F0FB617
:10051000F8943EBF0FBE2DBFCE0145960E945506F2
:100520000091361B1091371B8091151B882391F485
:1005300080919F10882329F48091381B9091391B5A
:1005400004C080913C1B90913D1B9093501C809364
:100550004F1C31C08091131B80FF05C080913E1B52
:1005600090913F1BF2CF80919E1090919F10882315
:1005700089F4992301F580913A1B90913B1B90934C
:10058000501C80934F1C84E080939E1081E08093E8
:100590009F1011C0815080939E10992361F081308B
:1005A00051F480913C1B90913D1B9093501C809383
:1005B0004F1C0E949E7A8091161B8823A9F4E0901C
:1005C000401BF090411B61E00E949F046091F51A6E
:1005D0007091F61A8091F71A9091F81A41E35AE057
:1005E00025E00E949D0604C0E090421BF090431B52
:1005F0008EE061E00E949F046091F11A7091F21AFE
:100600008091F31A9091F41A41E35AE025E00E9498
:100610009D068091161B882311F583E062E00E94FD
:100620009F046091F91A7091FA1A8091FB1A9091C7
:10063000FC1A47E35AE027E00E949D068BE062E047
:100640000E949F046091011B7091021B8091031B0B
:100650009091041B47E35AE027E00E949D0687E043
:1006600063E00E949F0480914F1C9091501C0E9457
:10067000550682E063E00E949F04C7010E94550670
:10068000F801D8010D900020E9F7EA1B8E2F8B5E50
:1006900063E00E949F04C8010E94550602C00E94A8
:1006A000DE7AA8960FB6F894DEBF0FBECDBFCF910D
:1006B000DF911F910F91FF90EF9008950F931F937B
:1006C0001091511C1F5F1093511C143021F48DE1C7
:1006D0000E94DF050AC00091521C0E942E7B1093DD
:1006E000511C0093521C0E949D7F1F910F910895F1
:1006F00080910A1B813019F40E941E21089581E027
:100700008093091B089580910B1B882309F45FC017
:1007100080910A1B833081F18430E9F18230E9F065
:100720002091F61A3091F71A4091F81A5091F91A5F
:100730008091681B6091641B0E9408762091FA1AD0
:100740003091FB1A4091FC1A5091FD1A8091681B60
:100750006091641B0E9413763AC02091FA1A30917E
:10076000FB1A4091FC1A5091FD1A8091681B609110
:10077000641B0E943E752BC02091FA1A3091FB1A1F
:100780004091FC1A5091FD1A8091681B6091641B86
:100790000E94EB741CC02091F61A3091F71A409118
:1007A000F81A5091F91A8091681B6091631B0E949E
:1007B000A3742091FA1A3091FB1A4091FC1A5091BF
:1007C000FD1A8091681B6091631B0E94AE741092A9
:1007D0000B1B08950E9483830E94C2050895EF9227
:1007E000FF920F931F9380910A1B833009F45AC024
:1007F000843009F484C0823061F18091681B60917B
:10080000641B0E94B2776093F61A7093F71A809374
:10081000F81A9093F91A8091681B6091641B0E94EA
:10082000B7776093FA1A7093FB1A8093FC1A90932F
:10083000FD1A80E090E0DC018093FE1A9093FF1A8D
:10084000A093001BB093011B80E090E0A0E7B3E40D
:1008500082C00F2EF0E0EF2EF0E0FF2EF6E90F2F12
:10086000F3EC1F2FF02DE092F61AF092F71A009396
:10087000F81A1093F91A8091681B6091641B0E940A
:100880005F776093FA1A7093FB1A8093FC1A909327
:10089000FD1AE092FE1AF092FF1A0093001B1093CB
:1008A000011B55C00F2EF0E0EF2EF0E0FF2EFAE70F
:1008B0000F2FF4EC1F2FF02DE092F61AF092F71A9A
:1008C0000093F81A1093F91A8091681B6091641BC9
:1008D0000E94DA736093FA1A7093FB1A8093FC1AE1
:1008E0009093FD1AE092FE1AF092FF1A0093001BFB
:1008F0001093011B80E090E0AAE7B4E42CC0809143
:10090000681B6091631B0E9404776093F61A7093D2
:10091000F71A8093F81A9093F91A8091681B6091E6
:10092000631B0E940A776093FA1A7093FB1A8093F4
:10093000FC1A9093FD1A80E090E0A6E9B3EC809356
:10094000FE1A9093FF1AA093001BB093011B80E046
:1009500090E0A6E9B3E48093021B9093031BA0935D
:10096000041BB093051B1F910F91FF90EF9008950A
:10097000EF92FF92CF93DF9380930A1B1092091B93
:100980001092081B10920C1B10920B1B88EC90E02D
:100990000E9489050E94EF83CCEDDAE1CE0160E28E
:1009A00070E044E150E00E9459C48EE50E949B1221
:1009B000BC01FC0101900020E9F73197E81BF90B1D
:1009C0002AE030E02E1B3F0B36952795265F3F4FE0
:1009D0002C0F3D1FC901AF010E9450C480E090E080
:1009E0000E944306CE0160E270E044E150E00E94C4
:1009F00059C481E090E00E9443068EE20E949B125F
:100A0000BC01FC0101900020E9F73197E81BF90BCC
:100A1000CE01AF010E9450C480E30E949B12BC0132
:100A2000FC0101900020E9F73197E81BF90B9E01CA
:100A30002E1B3F0B2C5E3F4FC901AF010E9450C4DB
:100A400082E090E00E944306CE0160E270E044E163
:100A500050E00E9459C48FE20E949B12BC01FC012D
:100A600001900020E9F73197E81BF90B9E012E5FFA
:100A70003F4FC901AF010E9450C481E30E949B1205
:100A8000BC01FC0101900020E9F73197E81BF90B4C
:100A9000CE1BDF0B6296CE01AF010E9450C483E0F3
:100AA00090E00E9443060E9457120E942224DF9188
:100AB000CF91FF90EF90089584E00E94B8848EE07B
:100AC0000E949B129093331B8093321B8EE30E94F3
:100AD0009B129093351B8093341B089581E00E94F4
:100AE000B8848DE00E949B129093331B8093321B3D
:100AF0008BE30E949B129093351B8093341B8CE3F5
:100B00000E949B129093371B8093361B8DE30E94AB
:100B10009B129093391B8093381B08950E94838306
:100B200080910A1B823029F0833049F00E94C2056F
:100B3000089581E080930A1B1092091B06C082E091
:100B400080930A1B81E08093091B0E94EF83089524
:100B50000E94838380910A1B813019F0823071F4E6
:100B600004C092E090930A1B04C083E080930A1BA8
:100B700081E08093091B0E94EF8308950E94C205C3
:100B80000895EF92FF920F931F93DF93CF93CDB70A
:100B9000DEB728970FB6F894DEBF0FBECDBF0E9418
:100BA000EF2680E060E00E949F04E091091BF0E0E6
:100BB000EE0FFF1FEF5EF44E808191810E9455067B
:100BC00080910A1B8E010F5F1F4F843009F042C0D5
:100BD00080E061E00E949F048DB79EB708970FB632
:100BE000F8949EBF0FBE8DBFEDB7FEB73196ADB77F
:100BF000BEB712961C930E93119788E090E09383F2
:100C000082838091321B9091331B958384838091E2
:100C1000631B90E00196978386830E94B6C48DB7CC
:100C20009EB708960FB6F8949EBF0FBE8DBFC80141
:100C30000E94550686E061E00E949F048091341B6B
:100C40009091351B0E94550682E161E00E949F044D
:100C500081E453C080E061E00E949F04ADB7BEB75D
:100C600018970FB6F894BEBF0FBEADBFEDB7FEB775
:100C7000319612961C930E93119788E090E093831F
:100C800082838091321B9091331B95838483809162
:100C9000641B90E00196978386830E94B6C48DB74B
:100CA0009EB708960FB6F8949EBF0FBE8DBFC801C1
:100CB0000E94550680910A1B823041F0833061F01A
:100CC000E090341BF090351B06E50BC0E090361B1E
:100CD000F090371B01E405C0E090381BF090391B01
:100CE00007E585E061E00E949F04C7010E94550668
:100CF00082E161E00E949F04802F0E94B2048BE099
:100D000061E00E949F04E091091BF0E0EE0FFF1FDD
:100D1000EE0FFF1FEF50F54E65817681878190853C
:100D200045E55AE027E00E949D0628960FB6F89404
:100D3000DEBF0FBECDBFCF91DF911F910F91FF900E
:100D4000EF900895772767FD7095E82FF0E0EE0F9C
:100D5000FF1FEE0FFF1FE60FF71FEE0FFF1FEE0F37
:100D6000FF1FE056FF4E5081418132812381652F64
:100D7000742F832F922F0895EF92FF920F931F935A
:100D8000262F332727FD3095482F50E0CA01880FC2
:100D9000991F880F991F820F931F880F991F880F23
:100DA000991F80569F4E0F2EF0E0EF2EF0E0FF2EA1
:100DB000F0E00F2FF0E01F2FF02DFC01E082F18218
:100DC00002831383E6EAF0E04E9FB0014F9F700D5F
:100DD0005E9F700D11246E5A7E4F44E0220F331F28
:100DE0004A95E1F7620F731F0E944F2A1F910F91DE
:100DF000FF90EF9008952F923F924F925F926F92E3
:100E00007F928F929F92AF92BF92CF92DF92EF929A
:100E1000FF920F931F93DF93CF9300D00F92CDB724
:100E2000DEB74983682E7724A62EBB249301220FB8
:100E3000331F220F331F2A0D3B1D220F331F220F9A
:100E4000331F3B832A8310EA812E10E1912E820EFC
:100E5000931EF401208031804280538096EA899F5E
:100E6000C0011124825A9E4F9501B4E0220F331F16
:100E7000BA95E1F7C090D504D090D604E090D7049D
:100E8000F090D804820F931F40E050E068E472ECC9
:100E900000E010E028E432E40E94172B6B017C0193
:100EA0000A811B8100541F4EF8016081718182818B
:100EB00093810E9425C19B01AC01C701B6010E942C
:100EC000D9C16B017C01F9812F2F30E0B90188274E
:100ED00077FD8095982F0E9425C19B01AC01C70129
:100EE000B6010E948AC020E030E64AE657E40E943C
:100EF0008AC09B01AC01C201B1010E9422C0F40171
:100F00006083718382839383F8011082118212823D
:100F10001382F301EE0FFF1FEA0DFB1DEC51FF4E94
:100F200010820F900F900F90CF91DF911F910F9132
:100F3000FF90EF90DF90CF90BF90AF909F908F90F9
:100F40007F906F905F904F903F902F9008954F92B9
:100F50005F927F928F929F92AF92BF92CF92DF92D9
:100F6000EF92FF920F931F93DF93CF930F92CDB722
:100F7000DEB7823058F440EAE42E40E1F42E32E548
:100F8000832E31E0932E442455242CC08430B1F5B7
:100F9000F2CFF8018081882359F0872D622F4CE32E
:100FA00029830E94FB86C601B5010E944F2A298130
:100FB0002F5F0F5F1F4F84E090E0C80ED91EE0E165
:100FC000F0E0AE0EBF1E243021F70894411C511CE6
:100FD000EE0EFF1E86EA90E0880E991E92E04916FA
:100FE000510451F0742C8201000F111F0C511F4E3F
:100FF0005401670120E0CDCF1092FE100F90CF91E9
:10100000DF911F910F91FF90EF90DF90CF90BF90F5
:10101000AF909F908F907F905F904F9008958F92A8
:101020009F92AF92BF92CF92DF92FF920F931F9346
:10103000DF93CF930F92CDB7DEB7F82E662319F466
:1010400021E030E034C0882E9924840164E0000F50
:10105000111F6A95E1F700541F4E880C991C84EE0D
:1010600090E1880E991E20E0F801A080B180C28036
:10107000D3808F2D622F29830E946973AA2797FD41
:10108000A095BA2F8A0D9B1DAC1DBD1DF801819343
:101090009193A193B1938F01F40180818F5F81932C
:1010A0004F0129812F5F2430F9F620E030E0C9019B
:1010B0000F90CF91DF911F910F91FF90DF90CF9014
:1010C000BF90AF909F908F9008956F927F928F9274
:1010D0009F92AF92BF92CF92DF92EF92FF920F93C7
:1010E0001F93CF93DF938091FE10882309F060C097
:1010F0008091661B833009F05BC002E511E0C0E01F
:10110000D0E01FC0C7010E94D72AF40161937193F8
:10111000819391934F01F5011192119211921192C5
:101120005F01F60111926F0180E190E0E80EF91E77
:10113000E614F70439F721960A551F4FC230D1053E
:1011400001F1CE01B4E0880F991FBA95E1F7A0EA4A
:101150008A2EA0E19A2E880E991EF0ECAF2EF0E1B7
:10116000BF2EA80EB91E6E01CC0CDD1CE4EEF0E122
:10117000CE0EDF1E70E4672E712C600E711E78019A
:10118000C1CF8091A30D9091A40DA091A50DB09118
:10119000A60D8093E0109093E110A093E210B0931D
:1011A000E3101092FC101092FD1081E08093FE106D
:1011B000DF91CF911F910F91FF90EF90DF90CF9033
:1011C000BF90AF909F908F907F906F9008955F92A7
:1011D0006F927F928F929F92AF92BF92CF92DF9247
:1011E000EF92FF920F931F93CF93DF938091A30D04
:1011F0009091A40DA091A50DB091A60D2091E010A5
:101200003091E1104091E2105091E3107C018D018A
:10121000E21AF30A040B150BA801970124363105D5
:101220004105510508F469C08093E0109093E110E6
:10123000A093E210B093E3100E9465888091FE10A5
:10124000882309F45AC08FE098E860E070E00E94BB
:10125000CE5E8091FC108F5F8093FC108C3308F47D
:101260004CC01092FC108091FD108F5F8093FD1098
:10127000893610F4EE2404C01092FD10EE24E3949D
:1012800020EAC22E20E1D22E92E5692E91E0792E3D
:10129000C0E0D0E028C0F8014081442351F0852D02
:1012A0006F2D0E94FB86EE2021F0C501B4010E9443
:1012B0004F2AF3940F5F1F4F84E090E0A80EB91EF1
:1012C000E0E1F0E08E0E9F1EF4E0FF1621F721967C
:1012D00000E110E0C00ED11E86EA90E0680E791E93
:1012E000C230D10551F05C2E8E01000F111F0C5140
:1012F0001F4E43015601FF24CECFDF91CF911F91A6
:101300000F91FF90EF90DF90CF90BF90AF909F90A4
:101310008F907F906F905F9008958091691B60918E
:10132000641B0E94BC860895CF92DF92EF92FF92D9
:101330000F931F93DF93CF93CDB7DEB728970FB6E8
:10134000F894DEBF0FBECDBF81EF9AE10E94C34982
:101350008091691B6091641B0E94A2866B017C01D5
:101360008DB79EB708970FB6F8949EBF0FBE8DBF7E
:10137000EDB7FEB731968E010F5F1F4FADB7BEB709
:1013800012961C930E93119788E090E093838283CA
:101390008091321B9091331B958384838091641BD1
:1013A00090E00196978386830E94B6C48DB79EB75E
:1013B00008960FB6F8949EBF0FBE8DBF8AE061E01D
:1013C0000E949F04C8010E9455068091661B8823D5
:1013D00079F18091F61A843130F462E00E949F0422
:1013E00080E20E94B2048091F61A8F5F8093F61A11
:1013F000883210F01092F61A0091F61A102F1E5F24
:10140000183210F0185206C0043120F4143128F0BC
:1014100013E103C0143160F400E0802F62E00E9409
:101420009F0404C08BED0E94B2040F5F1017D0F729
:1014300083E063E00E949F04C701B6014BE85AE0D5
:1014400027E00E949D0628960FB6F894DEBF0FBED7
:10145000CDBFCF91DF911F910F91FF90EF90DF9063
:10146000CF900895EF92FF920F931F93DF93CF9346
:10147000CDB7DEB728970FB6F894DEBF0FBECDBF4D
:1014800084E690E00E94890585E28093F61A0CEDCF
:101490001AE1C80160E270E044E150E00E9459C4E2
:1014A00081E00E949B12BC01FC0101900020E9F741
:1014B0003197E81BF90B24E130E02E1B3F0B3695EA
:1014C0002795200F311FC901AF010E9450C480E051
:1014D00090E00E944306C80160E270E044E150E001
:1014E0000E9459C48CE00E949B122DB73EB7285031
:1014F00030400FB6F8943EBF0FBE2DBFEDB7FEB71C
:1015000031967E010894E11CF11CADB7BEB712966E
:10151000FC92EE92119728E030E03383228395838A
:1015200084838091691B90E00D96978386830E9447
:10153000B6C4F70101900020E9F73197EE19FF09D1
:1015400098012B5F3F4F8DB79EB708960FB6F89462
:101550009EBF0FBE8DBFC901B701AF010E9450C42D
:1015600081E090E00E944306C80160E270E044E13F
:1015700050E00E9459C482E090E00E94430689E74F
:101580000E949B12BC01FC0101900020E9F73197F9
:10159000E81BF90BC801AF010E9450C484E20E940D
:1015A0009B12BC01FC0101900020E9F73197E81B78
:1015B000F90B0E1B1F0B0E5E1F4FC801AF010E94DF
:1015C00050C483E090E00E94430681EF9AE10E94BC
:1015D000054A0E9457128DE00E949B129093331B84
:1015E0008093321B0E94948928960FB6F894DEBF30
:1015F0000FBECDBFCF91DF911F910F91FF90EF9064
:101600000895CF93DF9384E060E00E949F04C8E3D5
:10161000D2E0CE010E94550680E160E00E949F0466
:10162000CE0102960E94550684E061E00E949F046C
:10163000CE010E945506DF91CF910895EF92FF925F
:101640000F931F93DF93CF93CDB7DEB728970FB6D5
:10165000F894DEBF0FBECDBF8DB79EB708970FB60B
:10166000F8949EBF0FBE8DBFEDB7FEB731968E01C9
:101670000F5F1F4FADB7BEB712961C930E93119715
:1016800088E090E0938382838091321B9091331B9A
:10169000958384838091621B90E001969783868373
:1016A0000E94B6C48DB79EB708960FB6F8949EBF39
:1016B0000FBE8DBF8BE060E00E949F04C8010E94B6
:1016C00055068091661B882309F439C180910D1C51
:1016D0008F3F09F434C18091621B90E00E94A26A9E
:1016E0009093FC1A8093FB1A8091621B90E00E94F9
:1016F000B86A6093FD1A7093FE1A8093FF1A909354
:10170000001B8091621B90E00E94B26A6093011BF3
:101710007093021B8093031B9093041B8091621BA8
:1017200090E00E94046B6093051B7093061B8093EE
:10173000071B9093081B8091621B90E00E94FE6A39
:101740006093091B70930A1B80930B1B90930C1BD7
:101750008091621B90E00E94AC6A60930D1B7093B5
:101760000E1B80930F1B9093101B8091621B90E0C7
:101770000E94896A6093111B7093121B8093131B44
:101780009093141B80E161E00E949F046091111B03
:101790007091121B8091131B9091141B49EA5AE01F
:1017A00023E00E949D066091FD1A7091FE1A8091BF
:1017B000FF1A9091001B2091051B3091061B409150
:1017C000071B5091081B0E94D9C10E943CC27B019B
:1017D0008C0184E062E00E949F04C801B7010E946E
:1017E000F2C0DC01CB016FEA7AE045E00E945806C6
:1017F00080E162E00E949F048091FB1A9091FC1AA4
:1018000063EB7AE043E00E9458066091011B7091FF
:10181000021B8091031B9091041B2091091B3091A6
:101820000A1B40910B1B50910C1B0E94D9C10E94B6
:101830003CC27B018C0184E063E00E949F04C801EC
:10184000B7010E94F2C0DC01CB016FEA7AE045E00B
:101850000E9458068FE063E00E949F0460910D1B78
:1018600070910E1B80910F1B9091101B47EB5AE05B
:1018700024E00E949D0680910F1C8F3708F087C0DE
:101880008091621B90E00E94C6686093F11A709389
:10189000F21A8093F31A9093F41A8091621B90E0ED
:1018A0000E9403696093F51A7093F61A8093F71AF1
:1018B0009093F81A8091621B90E00E94C169909306
:1018C000FA1A8093F91A84E060E00E949F04609104
:1018D000F51A7091F61A8091F71A9091F81A0E94F1
:1018E0003CC20E94F2C0DC01CB016FEA7AE045E025
:1018F0000E94580680E160E00E949F048091F91ADE
:101900009091FA1A63EB7AE043E00E94580684E073
:1019100061E00E949F046091F11A7091F21A809127
:10192000F31A9091F41A0E943CC20E94F2C0DC01AA
:10193000CB016FEA7AE045E00E9458062AC080E1B8
:1019400061E00E949F048AE392E00E94550684E0D1
:1019500062E00E949F0488E392E00E94550680E1C5
:1019600062E00E949F048AE392E00E94550684E0B0
:1019700063E00E949F0488E392E00E9455068FE096
:1019800063E00E949F048AE392E00E9455060E9451
:10199000018B28960FB6F894DEBF0FBECDBFCF9156
:1019A000DF911F910F91FF90EF900895CF92DF92FA
:1019B000EF92FF920F931F93CF93DF9384EF91E009
:1019C0000E948905CCEDDAE1CE0160E270E044E1ED
:1019D00050E00E9459C481E60E949B12BC01FC01A8
:1019E00001900020E9F73197E81BF90BCE01AF0118
:1019F0000E9450C417E51093E51A03E40093EF1A10
:101A000080E090E00E944306CE0160E270E044E195
:101A100050E00E9459C48AE50E949B12BC01FC015F
:101A200001900020E9F73197E81BF90BCE01AF01D7
:101A30000E9450C482E60E949B12BC01FC010190EE
:101A40000020E9F73197E81BF90B8BE0E82EF12C29
:101A5000EC0EFD1EC701AF010E9450C41093E51AA1
:101A600085E28093EF1A81E090E00E944306CE0168
:101A700060E270E044E150E00E9459C483E60E94B5
:101A80009B12BC01FC0101900020E9F73197E81B93
:101A9000F90BCE01AF010E9450C41093E51A0093D8
:101AA000EF1A82E090E00E944306CE0160E270E00F
:101AB00044E150E00E9459C484E60E949B12BC019C
:101AC000FC0101900020E9F73197E81BF90BCE01EA
:101AD000AF010E9450C485E60E949B12BC01FC012C
:101AE00001900020E9F73197E81BF90BC701AF011E
:101AF0000E9450C41093E51A86E58093EF1A83E0A4
:101B000090E00E9443060E9457128BE00E949B12B5
:101B10009093331B8093321B0E941E8BDF91CF91D9
:101B20001F910F91FF90EF90DF90CF9008958091DB
:101B3000F11A882321F08091F21A813019F00E9465
:101B4000B41108951092F11A08958091F11A81301C
:101B500021F08091F31A813019F00E94A0110895AC
:101B60008093F11A08958091621B60E00E946A36AA
:101B70008093F21A8091621B61E00E946A36809322
:101B8000F31A80E09091F21A913009F481E090E02C
:101B90002091F31A213009F491E0890F8093F41A0F
:101BA00008956F927F928F929F92AF92BF92CF9241
:101BB000DF92EF92FF920F931F93CF93DF930E94D8
:101BC000B38D81E060E00E949F04E091F21AF0E0A2
:101BD000EE0FFF1FEE5CF44E808191810E9455064E
:101BE00081E061E00E949F04E091F31AF0E0EE0FC3
:101BF000FF1FEE5CF44E808191810E94550680E0CB
:101C00006091F11A0E949F048091F41A882311F4C4
